:020000040038C2
:07FF000018FB785C560216A5
:0FFF60008B0B48DA5A220000167AFA682BAB4056
:20FFE0005C56021610FF20FF30FF40FF000060FF5C56021610FF20FF30FF40FF00FF60FF78
:020000040000FA
:200500000000000000000000000000000000000000000000000000000000000000000000DB
:200520000000000000000000000000000000000000000000000000000008000000000000B3
:2005400000000000000000000000000200040000060000000000000000000000000000008F
:2005600000000000000000000000000000000000000000000000000000000000000000007B
:200580000000313233343536373839302D3D080951574552545955494F505B5D0D00415351
:2005A000444647484A4B4C3B2760005C5A584356424E4D2C2E2F002A002000000000000028
:2005C00000000000000000000000000000000000000000000000000000000000000000001B
:2005E0000000000000000000000000000000000000000000000000000000000000000000FB
:020000040016E4
:200000004808C220A900005B2868A90048ABE220AD4001F03CAD40012901C901D0068D40DD
:2000200001200E01AD40012904C904D0068D400120AB01AD40012908C908D0068D40012084
:20004000AF01AD40012980C980D0068D400120CD01E220AD4101F00FAD41012901C901D0DB
:20006000068D4101206F00E220AD4201F0006BE210AF87E8AF2907D006AF6010AF8004AF09
:200080000318AFC97FB07AAAAF540216C905F016BD0005AAE000F069AF540216C903F061AE
:2000A000C210FC040160E00EF010E01CF011BD8005C900F04C201C0280472031028042A51C
:2000C00092C906F00E186590AAA9209FF51B16E69280ECC21020B410A9018F540216A01885
:2000E000AA8417A00700A21E00A9008717E617CAD0F9C220A517186932008517E22088D036
:20010000E5C21060F8064F087908A308CD08AF87E8AF2907D006AF6410AF8004AF0718AFCC
:200120008901F014AF87E8AF2907D006AF6010AF8004AF0318AF80D6200C08AF540216D01E
:20014000052019068064C901D02EA5811A8581C93CD057A9008581F8A58038E9018580D872
:2001600020390DA580C900D041A9048F54021622A8100020880F8032C903D00520A90B803A
:2001800029C904D005203B0F8020C905D01CA028AA8417A9AF8519A923851EC220A9F51BC3
:2001A0001865908570E220203E0C6020811160A57AF0198901F00320D417A57A8902F00312
:2001C000202218A57A8904F00320701860E220AF40010029808F400100AF87E8AF2907D0E6
:2001E00006AF6010AF8004AF0318AFA20000E210A6E09F0607AFE8E003D01CAF0207AF8516
:20020000E1AF0307AF85E2AF0407AF85E3AF0507AF85E4E220A20086E0C2106048A592C906
:2002200006F00CE692186590AA689FF51B16606860A592F00DC6923A186590AAA95F9FF51F
:200240001B166000000000000500000000000000000000000401E220C210A9008D870F8FD4
:200260000007AF8F1000AF857A85928F0500AF8F0600AF8F0700AFA9018F5502168F04005F
:20028000AFA9208F0800AF8F0900AFA9208F0020AEA9108F0040AEA9208F6420AEA9108F2B
:2002A0006440AEA9208FC820AEA9108FC840AEA9208F2C21AEA9108F2C41AEA9208F902141
:2002C000AEA9108F9041AEA9208FF421AEA9108FF441AEA9208F5822AEA9108F5842AEA9AA
:2002E000208FBC22AEA9108FBC42AEA9208F2023AEA9108F2043AEA9208F8423AEA9108F38
:200300008443AEA9208FE823AEA9108FE843AEA9208F4C24AEA9108F4C44AEA9208FB0240E
:20032000AEA9108FB044AEA9208F1425AEA9108F1445AEA9208F7825AEA9108F7845AEA998
:20034000208FDC25AEA9108FDC45AEA9208F4026AEA9108F4046AEA9208FA426AEA9108F28
:20036000A446AEA9208F0827AEA9108F0847AEA9208F6C27AEA9108F6C47AEA9208FD027DA
:20038000AEA9108FD047AEA9208F3428AEA9108F3448AEA9208F9828AEA9108F9848AEA989
:2003A000208FFC28AEA9108FFC48AEA9208F6029AEA9108F6049AEA9208FC429AEA9108F19
:2003C000C449AEA9208F282AAEA9108F284AAEA9208F8C2AAEA9108F8C4AAEA9208FF02AA8
:2003E000AEA9108FF04AAEA9208F542BAEA9108F544BAEA9208FB82BAEA9108FB84BAEA97A
:20040000208F1C2CAEA9108F1C4CAEA9208F802CAEA9108F804CAEA9208FE42CAEA9108F07
:20042000E44CAEA9208F482DAEA9108F484DAEA9208FAC2DAEA9108FAC4DAEA9208F102E74
:20044000AEA9108F104EAEA9208F742EAEA9108F744EAEA9208FD82EAEA9108FD84EAEA969
:20046000208F3C2FAEA9108F3C4FAEA9208FA02FAEA9108FA04FAEA9208F0430AEA9108FF7
:200480000450AEA9208F6830AEA9108F6850AEA9208FCC30AEA9108FCC50AEA9208F303141
:2004A000AEA9108F3051AEA9208F9431AEA9108F9451AEA9208FF831AEA9108FF851AEA95A
:2004C000208F5C32AEA9108F5C52AEA9208FC032AEA9108FC052AEA9208F2433AEA9108FE8
:2004E0002453AEA9208F8833AEA9108F8853AEA9208FEC33AEA9108FEC53AEA9208F50340F
:20050000AEA9108F5054AEA9208FB434AEA9108FB454AEA9208F1835AEA9108F1855AEA948
:20052000208F7C35AEA9108F7C55AEA9208FE035AEA9108FE055AEA9208F4436AEA9108FD8
:200540004456AEA9208FA836AEA9108FA856AEA9208F0C37AEA9108F0C57AEA9208F7037DA
:20056000AEA9108F7057AEA9208FD437AEA9108FD457AEA9208F3838AEA9108F3858AEA939
:20058000208F9C38AEA9108F9C58AEC220A905008F84E8AF8F480216E220A9018F001EAE10
:2005A000A9418FC820AEA9108FC840AE20C50D20FD18201A10A9048F5402162003102011B1
:2005C00017A91F8F0000AFA9018F86E8AF22A81000A9F28F4C0100A9FE8F4D0100AF5402CE
:2005E00016C904D00620880F58801678AF84E8AF29078F470216C907F0F220CE06207D0AF0
:2006000058EAEAEAAF540216C902D00BA9008F54021620B10E80B680E8AF4302161A8F43EC
:200620000216CF4E0216D00FAF4A02161A8F4A0216A9008F430216206509AF4D0216F07BD2
:20064000AF4A0216D0034C5A0C20BE18201209C220F818AF5002166925008F500216900CA9
:2006600018AF5202166901008F520216D8E22020F906A9058F480216A9008F4A02168F4DDA
:2006800002168F4C02168F43021620CE06207D0AAF4F02161A8F4F0216C90AD01EA9008FAB
:2006A0004F0216F818AF55021669018F550216D8AF4E021638E9028F4E021620BF0920151F
:2006C0000A20060B20D90A20630B20870B60AF4702168F460216AF84E8AF29078F47021659
:2006E000C907F0F2608717C220A51718690020851FE220A51E871F6060647364746475A014
:2007000000006472C220AF4A02163A8D0001A90E008D0201AD0401AAE220BFCF1A16F00FE6
:20072000E672E8C8C00E00D0F1A572C90EF016E673AF4A02161A8F4A0216C915F006A573CD
:20074000C904D0BB60E674A9038F540216C220AF4A02163A8D0001A90E008D0201AD04012C
:20076000AAE220E8E8A00000A9099FCF1A16E8C8A90A9FCF1A16E8C8C00900D0F5A90B9F7B
:20078000CF1A1680AAA900EBAF4C0216D005BF5F1A1660C901D02BDA8A29F085738A290316
:2007A000AA38A90CE00000F005E904CA80F68572A3014A4A29031865726573AABF5F1A1686
:2007C000FA60C902D01ADA8A29F085738A290F857238A90FE572186573AABF5F1A16FA6053
:2007E000DA8A29F085738A290C4A4A8572A3012903AAA903E00000F006186904CA80F53842
:20080000E572186573AABF5F1A16FA60A5831A8583C906D0396483AF00E8AF8902D007642A
:200820007D20A30880288904D007647D204F08801D8908D007647D20790880128910D00C7E
:20084000A57DD00AA901857D20CD0860647D60AF540216C901F021AF4802163A8F4802162C
:20086000206509AF4D0216F00FAF4802161A8F480216A9008F4D021660AF540216C901F0ED
:2008800021AF4802161A8F480216206509AF4D0216F00FAF4802163A8F480216A9008F4DC1
:2008A000021660AF540216C901F021AF4A02161A8F4A0216206509AF4D0216F00FAF4A0212
:2008C000163A8F4A0216A9008F4D021660AF540216C901F004C904D007A9028F5402166057
:2008E000AF4C02161AC904D002A9008F4C0216206509AF4D0216F016A9008F4D0216AF4C50
:200900000216F0033A8002A9038F4C02166020E81860AF4602160A0A0A0AAAC220AF4A02D5
:20092000163A8D0001A90E008D0201AD0401186F480216A8A90000E220208507C900F00E33
:20094000DABB18AF46021669029FCF1A16FAE8C88A2903D0E4C2209818690A00A8E2208A87
:20096000290FD0D560A900EBAF4602160A0A0A0AAAC220AF4A02168D0001A90E008D0201FF
:20098000AD0401186F480216A8A90000E220208507C900F00BDABBBFCF1A16FAC900D018FD
:2009A000E8C88A2903D0E7C2209818690A00A8E2208A290FD0D88006A9018F4D021660A2DB
:2009C0009C128617A9B08519A20000A9008F450216A9008F440216BFCF1A16C923D004A9E3
:2009E0000180008717E8E617A9008717E617AF4402161A8F440216C90ED0DCC220A5171866
:200A00006964008517E220AF4502161A8F450216C915D0BD60A9B08519C220A99C12186FD7
:200A20004802166F4802168517A980008D0001AF4A02168D0201AD04011865178517E220AF
:200A4000A900EBAF4602160A0A0A0AAA208507C900F009AF4602161869028717E8E617A9F9
:200A6000008717E6178A2903D0E2C220A5171869780085178A290F00E220D0D060A038A5FF
:200A80008417A9AF8519A920851EA091198470203E0CA2C0158617A9B08519A900EBAF471C
:200AA00002160A0A0A0AAABF5F1A16C900F007AF4702161869028717E8E617A9008717E6FD
:200AC000178A2903D0E1C220A5171869780085178A290F00E220D0CF60A0C8A18417A9AFA6
:200AE0008519A920851EA071198470203E0CE617AF52021620540DAF51021620540DAF5035
:200B0000021620540D60A093A18417A9AF8519A920851EA0071A8470203E0CA0E3A184172D
:200B2000A0F51B8470A20000203E0CE617E220BFFE1B1620540DBFFD1B1620540DBFFC1B53
:200B40001620540DC2208A18690A00AA1869F51B8570A517186943008517BFFC1B16E220CD
:200B6000D0C660A068A28417A9AF8519A920851EA078198470203E0C18A51769058517AFBC
:200B800055021620540D60A048A48417A9AF8519A920851EA088198470203E0CE617A579C4
:200BA00020540DA57820540D60AF4302161A8F430216C901D02AA0A8A38417A9AF8519A9BF
:200BC00020851EA07F198470203E0CE617A674BF62191620540DA90020540D20D318805DC2
:200BE000C932D059A0A8A38417A900A000009717C8C01000D0F8A674BF621916EBA900C234
:200C000020F8186F5002168F500216900C18AF5202166901008F520216A57418657885789B
:200C2000E220900BAF5202161869018F520216D8207C0DA9008F4302168F54021660DA8BAF
:200C4000A91648ABB270F00F20E506A617E88617A670E8867080EDABFA6020FB10A57EC9F7
:200C60000AF004A9058002A9018F540216A9008581A9308580A9008F0002AF8F0C02AFA936
:200C800018858A8586C220A955C68584E22020A91622A81000A03FA88417A9AF8519A923D4
:200CA000851EA067198470203E0CA08DA88417A920851EA071198470203E0CE617AF5202AF
:200CC0001620540DAF51021620540DAF50021620540DAF540216C905D02BA058AB8417A08A
:200CE000231A8470203E0CA0A8AB8417A03B1A8470203E0CA018AA8417A923851EA0121A40
:200D00008470203E0C20390DA9008F4A0216A20200A00000A9009FCF1A16E8C8C00A00D0A0
:200D2000F5E8E8E8E8AF4A02161A8F4A0216C914D0DFA9008F4A021660A02DA98417A9AF13
:200D40008519A920851EA09D198470203E0CA58020540D60DA48EBA900EB29F04A4A4A4AED
:200D6000AABF52191620E506E617A900EB68290FAABF52191620E506E617FA608BC220A5EF
:200D800074290F00F03BA90A018F521A16AAE8E8BFCF1A16C9090AD01EDAAF521A16AABF41
:200DA000CF1A169FDD1A16CAD0F5FAA574290F003A8574D0DB800AAF521A1638E90E008066
:200DC000C8E220AB608BA9808F0000AFA9008F0302AF8F0F02AF8F8202AF8F0001AFA90166
:200DE0008F0B01AFA9088F8302AF8F8702AFC220A900008F0901AF8F0802AF8F0A02AF8F7A
:200E00001402AF8F1602AF8F8002AFA900108F0102AFA900188F0D02AFA940008F0402AFC2
:200E20008F1002AFA920008F0602AF8F1202AFA9FF0FA2131EA0000054B016A9FF03A20F61
:200E400032A0002054AF16A9FF03A2132EA0002454AF16A9FFFFA20000A0000054B11AA96B
:200E6000FFFFA20000A0000054B21BA9FFFFA20000A0000054B31CA9FFFFA20000A000001C
:200E800054B41DA9FFAFA20000A0000054B51EA9FF07A20F3EA0008054AF16E220ABA90040
:200EA0008F0C02AFA9018F0002AFA9038F0801AF60A9288F4E0216A9008F1000AF8F4A0211
:200EC000168F4D02168F4302168F5002168F5102168F520216857885798F0500AF8F060063
:200EE000AF8F0700AFA9018F550216A9508511A9FF8F4801008F4901008F4A01008F4B01BB
:200F000000A9FF8F4C01008F4D01008F4E01008F4F0100200310A9018F0002AFA9008F0C52
:200F200002AFA917858A8586C220A9C3CC8584E22020A916A91F8F0000AF60AF4302161A98
:200F40008F430216C914D03FA9008F430216A20000A5821A8582A20000A9B08519A00018ED
:200F60008417A20000A00000BF0F3616F00D1AC909D002A9029F0F36169717E8C8A900977C
:200F800017C8E0C005D0E160A9008F0002AFA916858A8586C220A90D478584E22020A91631
:200FA000A08AAD8417A9AF8519A970851EA0A9198470203E0CA024AE8417A970851EA0C024
:200FC000198470203E0CA0C4AE8417A970851EA0E3198470203E0CA9008582A9B08519A0F0
:200FE00000188417A20000A00000BF0F36169717E8C8A9009717C8E00008D0EEA9018F0C7A
:2010000002AF60A200108617A9B08519A900A000009717C8C00010D0F860A53FD0034CA31C
:2010200010C220A9F51D8D4003A916008D4203A9541A8FF71D16A916008FF91D16A9F51B9F
:201040008D5403A916008D5603A900008F031E16A91F008F051E16E220A9028FF61D162281
:20106000181100B002803CAD2E03D037A94F8FF421AEA9108FF441AE22F8100060AD2E0317
:20108000F021C220AFFF1D168FFB1D16AF011E168FFD1D16E220A9598F5822AEA9108F58C1
:2010A00042AE60AD2E031869308F7825AEA9108F7845AE60A53FF042C220A9F51D8D4003E1
:2010C000A9541A8FF71D16A964008F071E16A900008F091E16A9F51B8F031E16A916008F27
:2010E000051E16E220A9028FF61D16A9168D4203A9168FF91D1622FC100060A900EBA9007C
:20110000857E85928590A20000BFFE1B16CF5202169029D016BFFD1B16CF510216901DD096
:201120000ABFFC1B16CF5002169011E67E8A18690A8590AAA57EC90AD0CF8044A25A00BF95
:20114000F41B169FFE1B16CAE490D0F3A900A00600EBA590AAA95F9FF51B16E888D0F8A9D4
:20116000009FF51B16E8AF5002169FF51B16E8AF5102169FF51B16E8AF5202169FF51B165B
:2011800060A68CE00000F004CA868C60A900EBA788857FC220E688D002E68AE22029F04AEF
:2011A0004A4AAA7CA71160C711C711C711CA11CA112C14231675168316A6167B12D711EA67
:2011C00011EA1103125C124C8111C220E688D002E68AE2204C8111C220E688D002E68AE6B8
:2011E00088D002E68AE2204C8111C220E688D002E68AE688D002E68AE688D002E68AE22051
:201200004C8111A57FC9E0D053C220A7888D2001C220E688D002E68AE220C220E688D0028B
:20122000E68AE220C220A7888D2201C220E688D002E68AE220C220E688D002E68AE220C291
:2012400020AD00808D2401AD02808D2601AD2801858AAD2A01858CE2204CA611C220E68889
:20126000D002E68AE688D002E68AE688D002E68AE688D002E68AE2204C8111A57FC9A0F0BF
:20128000034CD711A788C220E688D002E68AE220C900D04CA590C9089019A9878F00F1AF61
:2012A000A93F8F00F1AFC220E688D002E68AE2204C8111EBA788C220E688D002E68AE220F7
:2012C000C2204AE22048290F09808F00F1AF68C2204A4A4A4AE220293F8F00F1AF4C8111BF
:2012E000C901D013A788C220E688D002E68AE220290F85904C8111C902D04CA592C90890D4
:2013000019A9A78F00F1AFA93F8F00F1AFC220E688D002E68AE2204C8111EBA788C220E6CA
:2013200088D002E68AE220C2204AE22048290F09A08F00F1AF68C2204A4A4A4AE220293F7F
:201340008F00F1AF4C8111C903D013A788C220E688D002E68AE220290F85924C8111C90414
:20136000D04CA594C9089019A9C78F00F1AFA93F8F00F1AFC220E688D002E68AE2204C8187
:2013800011EBA788C220E688D002E68AE220C2204AE22048290F09C08F00F1AF68C2204A54
:2013A0004A4A4AE220293F8F00F1AF4C8111C905D013A788C220E688D002E68AE220290F2C
:2013C00085944C8111C908D01AA90F38E788C220E688D002E68AE220290F09908F00F1AF68
:2013E0004C8111C909D01AA90F38E788C220E688D002E68AE220290F09B08F00F1AF4C8173
:2014000011C90AD01AA90F38E788C220E688D002E68AE220290F09D08F00F1AF4C8111C22B
:2014200020E688D002E68AE2204C8111A57FC950D013A7888F00F1AFC220E688D002E68AEC
:20144000E2204CA611C951D023A900EBA788AAC220E688D002E68AE220A7889F00E6AFC254
:2014600020E688D002E68AE2204C8111C952D023A900EBA788AAC220E688D002E68AE220AD
:20148000A7889F00F2AFC220E688D002E68AE2204CA611C953D023A900EBA788AAC220E602
:2014A00088D002E68AE220A7889F00F3AFC220E688D002E68AE2204CA611C954D023A900A0
:2014C000EBA788AAC220E688D002E68AE220A7889F00F0AFC220E688D002E68AE2204C81E6
:2014E00011C955D01FA900EBA788AAC220E688D002E68AE220A788C220E688D002E68AE22A
:20150000204C8111C956D02AA900EBA788C910B0034C7B12AAC220E688D002E68AE220A7A7
:20152000889F00F2AFC220E688D002E68AE2204C8111C957D023A900EBA788AAC220E688A1
:20154000D002E68AE220A7889F00F2AFC220E688D002E68AE2204C8111C958D02AA900EBB7
:20156000A788C910B0034C7B12AAC220E688D002E68AE220A7889F00F2AFC220E688D00208
:20158000E68AE2204C8111C959D023A900EBA788AAC220E688D002E68AE220A7889F00F324
:2015A000AFC220E688D002E68AE2204C8111C95AD023A900EBA788AAC220E688D002E68AF5
:2015C000E220A7889F00E6AFC220E688D002E68AE2204C8111C95ED023A900EBA788AAC2EB
:2015E00020E688D002E68AE220A7889F00E6AFC220E688D002E68AE2204C8111C95FD0202C
:20160000A900EBA788AAC220E688D002E68AE220A7889F00E7AFC220E688D002E68AE220D1
:201620004C8111A57FC961D020C220A788AA868CE220C220E688D002E68AE220C220E688DB
:20164000D002E68AE2204CA611C962D008A2DF02868C4CA611C963D008A27203868C4CA689
:2016600011C966D00620C8164CA611C967D003204E174CA611A900EBA57F290FAAE8868C34
:201680004CA611A78A8F2AF2AFC220A58A1A858A9005A58C1A858CE220A900EBA57F290F9F
:2016A000AA868C4C81114C8111C220A90000858CA586858A18A03400B784693400658485AA
:2016C000889002E68AE22060C220A90000858C18A01C00B784F023691C008D2001C8C8B7E6
:2016E000848D2201A5848D2401A5868D2601AD28018588AD2A01858A8014A03400B7846926
:20170000340065848588A586858A9002E68AE22060A9448D65018D6D01A9018D66018D6E8D
:2017200001A9008D67018D6F01A9008D61018D62018D63018D69018D6A018D6B01A9018D75
:2017400064018D6C01A90B8D60018D680160A788C220E688D002E68AE220A78848C220E630
:2017600088D002E68AE220C220A7888D2001C220E688D002E68AE220C220E688D002E68AB8
:20178000E220C220A7888D2201C220E688D002E68AE220C220E688D002E68AE220C220A5D7
:2017A000888D2401A58A8D2601AD28018588AD2A01858AE22068F004C9C0D017C220A57D70
:2017C0000A0AAAAD24019D0080AD26019D0280E67DE22060A664E00000F004CA866460A70B
:2017E00060C220E660D002E662E220C950D012A7608F00F1AFC220E660D002E662E2208050
:2018000020C962D007A2DF0286648015C963D007A272038664800AC966D006A57A29FE8546
:201820007A60A66AE00000F004CA866A60A766C220E666D002E668E220C950D012A7668FDC
:2018400000F1AFC220E666D002E668E2208020C962D007A2DF02866A8015C963D007A272D7
:2018600003866A800AC966D006A57A29FD857A60A67BE00000F004CA867B60A76CC220E647
:201880006CD002E66EE220C950D012A76C8F00F1AFC220E66CD002E66EE2208020C962D080
:2018A00007A2DF02867B8015C963D007A27203867B800AC966D006A57A29FB857A60A24FCB
:2018C000468660A9168562A200008664A57A0901857A60A2B7468666A9168568A2000086C3
:2018E0006AA57A0902857A60A24F46866CA916856EA20000867BA57A0904857A60AF80E8D5
:20190000AF29FD09028F80E8AFA900853FA9018F02EAAFA9018F03EAAFAF04EAAF2901C9EC
:2019200001F0F6AF05EAAFF00EA9468F2C21AEA9108F2C41AE8010A901853FA9428F2C21D4
:20194000AEA9108F2C41AEAF80E8AF29FD8F80E8AF6030313233343536373839414243446D
:201960004546000103061047414D45204F5645520053434F52453A004C4556454C3A0042A2
:201980004F4E55533A2020004C494E45533A2020004E4558542050494543453A005265736A
:2019A0007461727420696E200057656C636F6D6520746F20433235362054657472697300EB
:2019C00048617264776172652044657369676E65723A2053746566616E7920416C6C616951
:2019E000726500536F66747761726520446576656C6F7065723A2044616E69656C20547272
:201A0000656D626C61790048492053434F5245533A00454E5445522055534552204E414DB9
:201A2000453A005072657373203C456E7465723E207768656E20646F6E65005072657373DD
:201A4000203C426B73703E20746F2064656C6574650000007465747269732E7363720000B5
:201A600000010000000100000001000000010000010100000101000000000000000000005E
:201A800001000000010000000101000000000000000100000001000001010000000000003E
:201AA00000010000010100000001000000000000000100000101000001000000000000001E
:201AC000010000000101000000010000000000232300000000000000000000232323230030
:201AE0000000000000000000002323232300000000000000000000232323230000000000CE
:201B00000000000000232323230000000000000000000023232323000000000000000000AD
:201B2000002323232300000000000000000000232323230000000000000000000023232324
:201B400023000000000000000000002323232300000000000000000000232323230000004A
:201B600000000000000000232323230000000000000000000023232323000000000000004D
:201B800000000023232323000000000000000000002323232300000000000000000000230A
:201BA0002323230000000000000000000023232323000000000000000000002323232300A4
:201BC0000000000000000000002323232300000000000000000000232323230000000000ED
:201BE00000000000002323232323232323232323232323232344414E2020200086240020B8
:201C0000202020202000000000202020202020000000002020202020200000000020202044
:201C2000202020000000002020202020200000000020202020202000000000202020202024
:201C40002000000000202020202020000000002020202020200000000000000000000000E4
:201C6000000000000000000000000000000000000000000000000000000000000000000064
:201C8000000000000000000000000000000000000000000000000000000000000000000044
:201CA000000000000000000000000000000000000000000000000000000000000000000024
:201CC000000000000000000000000000000000000000000000000000000000000000000004
:201CE0000000000000000000000000000000000000000000000000000000000000000000E4
:201D00000000000000000000000000000000000000000000000000000000000000000000C3
:201D20000000000000000000000000000000000000000000000000000000000000000000A3
:201D4000000000000000000000000000000000000000000000000000000000000000000083
:201D6000000000000000000000000000000000000000000000000000000000000000000063
:201D8000000000000000000000000000000000000000000000000000000000000000000043
:201DA000000000000000000000000000000000000000000000000000000000000000000023
:201DC000000000000000000000000000000000000000000000000000000000000000000003
:151DE000000000000000000000000000000000000000000000EE
:201E130000000000000000000000000000000000030303030303030303030303030303037F
:201E33000052525252525252525252525252520000E6E6E6E6E6E6E6E6E6E6E6E6E6E6007F
:201E530000060606060606060606060606060600008A8A8A8A8A8A8A8A8A8A8A8A8A8A008F
:201E73000001010101010101010101010101010000BEBEBEBEBEBEBEBEBEBEBEBEBEBE00DD
:201E930000666666666666666666666666666600000000000000000000000000000000009B
:201EB30000000000000000000000000000000000000000000000000000000000000000000F
:201ED3000404040404040404040404040404040400000000000000000000000000000000AF
:201EF3000000000000000000000000000000000000000000000000000000000000000000CF
:201F130000000000000000000000000000000000030101010101010101010101010100039B
:201F330052414141414141414141414141414180E6F7F7F7F7F7F7F7F7F7F7F7F7F7F7DFE7
:201F5300060707070707070707070707070707088A4E4E4E4E4E4E4E4E4E4E4E4E4E4E1F11
:201F730001020202020202020202020202020204BECECECECECECECECECECECECECECECF5C
:201F9300664646464646464646464646464646260000000909090909090909090909090959
:201FB300090909090909090909090909090909090909090909090909090909090900000009
:201FD3000404040404040404040404040404040400000000000000000000000000000000AE
:201FF3000000000000000000000000000000000000000000000000000000000000000000CE
:20201300000000000000000000000000000000000301E9E9E9E9E9E9E9E9E9E9E9E90403B6
:2020330052414280428042804280428042804180E6F7E9F9E9F9E9F9E9F9E9F9E9F9F7DFAE
:20205300060717681768176817681768176807088A4E6E2D6E2D6E2D6E2D6E2D6E2D4E1F70
:2020730001020103010301030103010301030204BECEDFBFDFBFDFBFDFBFDFBFDFBFCECF4F
:20209300664617661766176617661766176646260000094B6D6D4B4B6D6D4B4B6D6D4B4B83
:2020B3006D6D4B4B6D6D4B4B6D6D4B4B6D6D4B4B6D6D4B4B6D6D4B4B6D6D4B4B6D09000087
:2020D3000404040404040404040404040404040400000000000000000000000000000000AD
:2020F3000000000000000000000000000000000000000000000000000000000000000000CD
:20211300000000000000000000000000000000000301E9E9E9E9E9E9E9E9E9E9E9E90403B5
:2021330052418042804280428042804280424180E6F7F9E9F9E9F9E9F9E9F9E9F9E9F7DFAD
:20215300060768176817681768176817681707088A4E2D6E2D6E2D6E2D6E2D6E2D6E4E1F6F
:2021730001020301030103010301030103010204BECEBFDFBFDFBFDFBFDFBFDFBFDFCECF4E
:202193006646661766176617661766176617462600094B4B6D6D4B4B6D6D4B4B6D6D4B4B37
:2021B3006D6D4B4B6D6D4B4B6D6D4B4B6D6D4B4B6D6D4B4B6D6D4B4B6D6D4B4B6D6D090019
:2021D3000404040404040404040404040404040400000000000000000000000000000000AC
:2021F3000000000000000000000000000000000000000000000000000000000000000000CC
:20221300000000000000000000000000000000000301E9E9E9E9E9E9E9E9E9E9E9E90403B4
:2022330052414280428042804280428042804180E6F7E9F9E9F9E9F9E9F9E9F9E9F9F7DFAC
:20225300060717681768176817681768176807088A4E6E2D6E2D6E2D6E2D6E2D6E2D4E1F6E
:2022730001020103010301030103010301030204BECEDFBFDFBFDFBFDFBFDFBFDFBFCECF4D
:202293006646176617661766176617661766462600096D6D4B4B26264B4B26264B4B26269C
:2022B3004B4B26264B4B26264B4B26264B4B26264B4B26264B4B26264B4B26264B4B091F1F
:2022D3000404040404040404040404040404040400000000000000000000000000000000AB
:2022F3000000000000000000000000000000000000000000000000000000000000000000CB
:20231300000000000000000000000000000000000301E9E9E9E9E9E9E9E9E9E9E9E90403B3
:2023330052418042804280428042804280424180E6F7F9E9F9E9F9E9F9E9F9E9F9E9F7DFAB
:20235300060768176817681768176817681707088A4E2D6E2D6E2D6E2D6E2D6E2D6E4E1F6D
:2023730001020301030103010301030103010204BECEBFDFBFDFBFDFBFDFBFDFBFDFCECF4C
:202393006646661766176617661766176617462600096D6D4B4B26264B4B26264B4B26269B
:2023B3004B4B26264B4B26264B4B26264B4B26264B4B26264B4B26264B4B26264B4B091F1E
:2023D3000404040404040404040404040404040400000000000000000000000000000000AA
:2023F3000000000000000000000000000000000000000000000000000000000000000000CA
:20241300000000000000000000000000000000000301E9E9E9E9E9E9E9E9E9E9E9E90403B2
:2024330052414280428042804280428042804180E6F7E9F9E9F9E9F9E9F9E9F9E9F9F7DFAA
:20245300060717681768176817681768176807088A4E6E2D6E2D6E2D6E2D6E2D6E2D4E1F6C
:2024730001020103010301030103010301030204BECEDFBFDFBFDFBFDFBFDFBFDFBFCECF4B
:202493006646176617661766176617661766462600094B4B26264B4B26264B4B26264B4BDE
:2024B30026264B4B26264B4B26264B4B26264B4B26264B4B26264B4B26264B4B2626091F67
:2024D3000404040404040404040404040404040400000000000000000000000000000000A9
:2024F3000000000000000000000000000000000000000000000000000000000000000000C9
:20251300000000000000000000000000000000000301E9E9E9E9E9E9E9E9E9E9E9E90403B1
:2025330052418042804280428042804280424180E6F7F9E9F9E9F9E9F9E9F9E9F9E9F7DFA9
:20255300060768176817681768176817681707088A4E2D6E2D6E2D6E2D6E2D6E2D6E4E1F6B
:2025730001020301030103010301030103010204BECEBFDFBFDFBFDFBFDFBFDFBFDFCECF4A
:202593006646661766176617661766176617462600094B4B26264B4B26264B4B26264B4BDD
:2025B30026264B4B26264B4B26264B4B26264B4B26264B4B26264B4B26264B4B2626091F66
:2025D3000404040404040404040404040404040400000000000000000000000000000000A8
:2025F3000000000000000000000000000000000000000000000000000000000000000000C8
:20261300000000000000000000000000000000000301E9E9E9E9E9E9E9E9E9E9E9E90403B0
:2026330052414280428042804280428042804180E6F7E9F9E9F9E9F9E9F9E9F9E9F9F7DFA8
:20265300060717681768176817681768176807088A4E6E2D6E2D6E2D6E2D6E2D6E2D4E1F6A
:2026730001020103010301030103010301030204BECEDFBFDFBFDFBFDFBFDFBFDFBFCECF49
:202693006646176617661766176617661766462600096D6D4B4B26264B4B26264B4B262698
:2026B3004B4B26264B4B26264B4B26264B4B26264B4B26264B4B26264B4B26264B4B091F1B
:2026D3000404040404040404040404040404040400000000000000000000000000000000A7
:2026F3000000000000000000000000000000000000000000000000000000000000000000C7
:20271300000000000000000000000000000000000301E9E9E9E9E9E9E9E9E9E9E9E90403AF
:2027330052418042804280425142514251424180E6F7F9E9F9E9F9E9E7E9E7E9E7E9F7DF6A
:20275300060768176817681736673667361707088A4E2D6E2D6E2D6E4E6E4E6E4E6E4E1FFC
:2027730001020301030103010101010101010204BECEBFDFBFDFBFDFBEDFBEDFBEDFCECF51
:202793006646661766176617051705170517462600096D6D4B4B26264B4B26264B4B2626BA
:2027B3004B4B26264B4B26264B4B26264B4B26264B4B26264B4B26264B4B26264B4B091F1A
:2027D3000404040404040404040404040404040400000000000000000000000000000000A6
:2027F3000000000000000000000000000000000000000000000000000000000000000000C6
:20281300000000000000000000000000000000000301E9E9E9E9E9E9E9E9E9E9E9E90403AE
:2028330052414280428042514251425142804180E6F7E9F9E9F9E9E7E9E7E9E7E9F9F7DF69
:20285300060717681768173667366736676807088A4E6E2D6E2D6E4E6E4E6E4E6E2D4E1FAB
:2028730001020103010301010101010101030204BECEDFBFDFBFDFBEDFBEDFBEDFBFCECF50
:202893006646176617661705170517051766462600094B4B26264B4B26264B4B26264B4BFD
:2028B30026264B4B26264B4B26264B4B26264B4B26264B4B26264B4B26264B4B2626091F63
:2028D3000404040404040404040404040404040400000000000000000000000000000000A5
:2028F3000000000000000000000000000000000000000000000000000000000000000000C5
:20291300000000000000000000000000000000000301E9E9E9E9E9E9E9E9E9E9E9E90403AD
:2029330052418042804280425142514251424180E6F7F9E9F9E9F9E9E7E9E7E9E7E9F7DF68
:20295300060768176817686736673667361707088A4E2D6E2D6E2D6E4E6E4E6E4E6E4E1FAA
:2029730001020301030103010101010101010204BECEBFDFBFDFBFDFBEDFBEDFBEDFCECF4F
:202993006646661766176617051705170517462600094B4B26264B4B26264B4B26264B4BFC
:2029B30026264B4B26264B4B26264B4B26264B4B26264B4B26264B4B26264B4B2626091F62
:2029D3000404040404040404040404040404040400000000000000000000000000000000A4
:2029F3000000000000000000000000000000000000000000000000000000000000000000C4
:202A1300000000000000000000000000000000000301E9E9E9E9E9E9E9E9E9E9E9E90403AC
:202A330052414280428042514251425142804180E6F7E9F9E9F9E9E7E9E7E9E7E9F9F7DF67
:202A5300060717681768173667366736676807088A4E6E2D6E2D6E4E6E4E6E4E6E2D4E1FA9
:202A730001020103010301010101010101030204BECEDFBFDFBFDFBEDFBEDFBEDFBFCECF4E
:202A93006646176617661705170517051766462600096D6D4B4B6D6D4B4B6D6D4B4B6D6D0D
:202AB3004B4B6D6D4B4B6D6D4B4B6D6D4B4B6D6D4B4B6D6D4B4B6D6D4B4B6D6D4B4B091F35
:202AD3000404040404040404040404040404040400000000000000000000000000000000A3
:202AF3000000000000000000000000000000000000000000000000000000000000000000C3
:202B1300000000000000000000000000000000000301E9E9E9E9E9E9E9E9E9E9E9E90403AB
:202B330052418042804280428042804280424180E6F7F9E9F9E9F9E9F9E9F9E9F9E9F7DFA3
:202B5300060768176817681768676817681707088A4E2D6E2D6E2D6E2D6E2D6E2D6E4E1F15
:202B730001020301030103010301030103010204BECEBFDFBFDFBFDFBFDFBFDFBFDFCECF44
:202B9300664666176617661766176617661746260000096D4B4B6D6D4B4B6D6D4B4B6D6D56
:202BB3004B4B6D6D4B4B6D6D4B4B6D6D4B4B6D6D4B4B6D6D4B4B6D6D4B4B6D6D4B091F1F60
:202BD3000404040404040404040404040404040400000000000000000000000000000000A2
:202BF3000000000000000000000000000000000000000000000000000000000000000000C2
:202C1300000000000000000000000000000000000300040404040404040404040404040367
:202C330052414141414141414141414141414180E6F7F7F7F7F7F7F7F7F7F7F7F7F7F7DFDA
:202C5300060707070707070707070707070707088A4E4E4E4E4E4E4E4E4E4E4E4E4E4E1F04
:202C730001020202020202020202020202020204BECECECECECECECECECECECECECECECF4F
:202C930066464646464646464646464646464626000000090909090909090909090909094C
:202CB30009090909090909090909090909090909090909090909090909090909091F1F00BE
:202CD3000404040404040404040404040404040400000000000000000000000000000000A1
:202CF3000000000000000000000000000000000000000000000000000000000000000000C1
:202D1300000000000000000000000000000000000303030303030303030303030303030370
:202D33000080808080808080808080808080800000DFDFDFDFDFDFDFDFDFDFDFDFDFDF004E
:202D530000080808080808080808080808080800001F1F1F1F1F1F1F1F1F1F1F1F1F1F003E
:202D73000004040404040404040404040404040000CFCFCFCFCFCFCFCFCFCFCFCFCFCF00B6
:202D930000262626262626262626262626262600000000001F1F1F1F1F1F1F1F1F1F1F1F98
:202DB3001F1F1F1F1F1F1F1F1F1F1F1F1F1F1F1F1F1F1F1F1F1F1F1F1F1F1F1F1F1F00005E
:202DD3000404040404040404040404040404040400000000000000000000000000000000A0
:202DF3000000000000000000000000000000000000000000000000000000000000000000C0
:202E13001A0A0700090C0900090A10000B0A1700091206001E120300080D1D000A0733003D
:202E33000810170015140700081212000B0E230037120B000B0C2B0005111F000B073E009D
:202E530020131900091C06000C15230014191500321D04001B1B1200161722000D1B180038
:202E73001820080007200E00161A1E00091B1F000A13390008192700051143001F1B1D00EB
:202E9300261F110009260700071E24001B1F1D002A1A39002B271A0022252400292527002A
:202EB300171464002A27230006320B0017282800372B1900121B570011292D0008186D005F
:202ED30037320D002328370017370B0016293C0013244E000A2F33001A341F002C390B0045
:202EF300362B360025215B002C341C000C2162000A352400573219000A2C420022274C006A
:202F13000C3E1000082B5500004116002C3734000C2A800023229400182B7B0010299400B4
:202F33001153150022541000305310003D521000104E2B00853A50003633800020387800FC
:202F53004F5807006A550D004C50260017455B002F512F00664C33003F503100303E700039
:202F7300174C4A0032465900514C3E00464655002241700024388D001838910009427500A7
:202F93004330A000424A4D00434E42003E416E0034504200064A6300354D4E00085F3C0086
:202FB3000B6626003737B200213FAD002345A10068439500634F76000942BC00344AA200A2
:202FD30068741200327917004875220014646700524F9E0081702A000953B0001A5B9600FF
:202FF300327149004B6F4B003C5A94002F54B0006670480015658300595D8B004C5D9000DB
:203013006564750060686A00446B68004F657900606C6100866C5700526C6600726C5E0013
:2030330039677F00386D6D00AD773000395ECF005F61CA00439336004169BE00C289380011
:20305300BC8940009F9333008C9B23002F72C900679743001470D900CC7D840023869B0010
:2030730087925D004B8A88006C7FA5004B859B006E78BE006C8B820085819E006D87920028
:203093007D8C7E00A0868900C89749007E888E00BE974D00A1906C005080B6008F8E790050
:2030B3008D898B0044977300B59757003183BC000E85C1008E7EBC0072997200D4A6580090
:2030D300CDA65A00D9998D00C7A76600C8B35A00ADA79100C0A1A10017A5C300DBB55E0014
:2030F300BCAA8A0043A5BD008B9EC200A8B17E0068A6B400DDB469008BAAA100D6B56F00DA
:20311300D3B37A00A5A2BE009EAD9E00E4A5A6008EA8B500CFB285009FA9B000CCB08E008C
:20313300ADAAAB00A9B09F00CFB781002CA7E600BBB7A100E5C0790058ABE800DCC4750091
:20315300E8B99900DFC28A00DCC094007AB0E300D4C09900DCBE9F00ECC98400D2C2A200E5
:20317300CCD47800E8D47200D7CD9000B6D38900CACC9F00C5C5B700F2CF8C00EBCC98009E
:20319300C9C0C900C0C5BE00EDD19000D3C9B300E7CBA800E7CE9F00E2CDA700EAC8B7007D
:2031B300BCCEB200BDC8C800E0D0B000AAC8DF0069CCE600AFCFCD008ECDE10035D2EB002E
:2031D300E1E28A00EBD4B500EFD8AB00E0D9B700DECFD900F2D3C700F7E29700E9D8BC003A
:2031F300D8D7CB00D2D7CE00E2D9C500ECF0B900ECE7DA00DBE6E600E3E7E30000000000B5
:20321300CCCCCC00999999006666660033333300FFFFFF0000CCFF000099FF000066FF00DC
:203233000033FF0000000000333333006666660099999900CCCCCC00FFFFFF0000CC9900ED
:20325300000000000000000000000000000000000099CC0033CCFF0066CCFF006699FF00C9
:203273003366FF000033CC00000000000000000000000000000000003300CC0000FFCC00DA
:2032930033FFCC0000333300006666000099990000CCCC0000FFFF003399CC003366CC0026
:2032B3000000330000006600000099000000CC000000FF006633FF003300FF0000FF99009C
:2032D30066FFCC0033CC9900336666003399990033CCCC0033FFFF000066990000339900E7
:2032F30033336600333399003333CC003333FF006633CC009966FF006600FF0000FF66002C
:2033130066FF990033CC6600009966006699990066CCCC0066FFFF00336699000033660073
:20333300666699006666CC006666FF00330099009933CC00CC66FF009900FF0000FF330053
:2033530033FF66000099330000CC660033FF990099CCCC0099FFFF006699CC000066CC0034
:203373009999CC009999FF009933FF006600CC0066009900CC33FF00CC00FF0000CC00007A
:2033930000CC3300006633003399660066CC990099FFCC00CCFFFF0099CCFF003399FF0028
:2033B300CCCCFF00CC99FF009966CC0066339900330066009900CC003300330033CC33006C
:2033D30066CC660000FF000033FF330066FF660099FF9900CCFFCC0000000000000000004B
:2033F30000000000CC99CC0099669900993399009900990066336600660066000066000029
:203413003366330000990000339933006699660099CC9900000000000000000000000000D2
:20343300FFCCFF00FF99FF00FF66FF00FF33FF00FF00FF00CC66CC00CC33CC000033000089
:2034530033CC0000336600006699330099CC6600CCFF9900FFFFCC00FF993300FFCC990067
:20347300FFCCCC00FF99CC00CC6699009933660066003300CC009900CC00CC0033FF000079
:2034930066FF33003399000066CC000099FF3300FFFF9900CCCC9900CC660000CC996600F3
:2034B300FF999900CC999900FF339900CC00660099006600FF33CC00FF00CC0066FF0000A0
:2034D30099FF660066CC330066990000FFFF6600CCCC6600999966006633000099663300B2
:2034F300FF666600CC6666009966660099003300CC339900FF66CC00FF00990099FF00002C
:20351300CCFF660099CC3300FFFF3300CCCC330099993300666633009966000099330000A4
:20353300FF333300CC3333009933330066333300CC336600FF669900FF006600CCFF000083
:20355300CCFF3300FFFF0000CCCC0000999900006666000033330000CC993300CC66330063
:20357300FF000000CC000000990000006600000033000000FF336600FF00330099CC00000C
:2035930000000000000000000000000000000000CA990000FFCC3300FFCC6600FF99660088
:2035B300FF663300CC33000000000000000000000000000000000000CC003300FFFFFF0065
:2035D300CCCCCC0099999900666666003333330000000000FFCC0000FF990000FF66000016
:2035F300FF33000000000000333333006666660099999900CCCCCC00FFFFFF00000000008F
:20361300000000000000000000000000000000000000000000000000000000000000000097
:20363300000000000000000000000000000000000000000000000000000000000000000077
:20365300000000000000000000000000000000000000000000000000000000000000000057
:20367300000000000000000000000000000000000000000000000000000000000000000037
:20369300000000000000000000000000000000000000000000000000000000000000000017
:2036B3000000000000000000000000000000000000000000000000000000000000000000F7
:2036D3000000000000000000000404000000010100000505050000000202000000000000BA
:2036F3000000000000000000000000000000000000000000000000000000000000000000B7
:20371300000000000000000004000004000100000100050000000002000000000000000085
:20373300000000000000000000000000000000000000000000000000000000000000000076
:2037530000000000000000000400000000000000010005050500000202020000000000003C
:20377300000000000000000000000000000000000000000000000000000000000000000036
:20379300000000000000000004000000000001010000000000050002000002000000000007
:2037B3000000000000000000000000000000000000000000000000000000000000000000F6
:2037D3000000000000000000040000040001000000000000000500020000020000000000C4
:2037F3000000000000000000000000000000000000000000000000000000000000000000B6
:20381300000000000000000000040400000101010100050505000000020200000000000076
:20383300000000000000000000000000000000000000000000000000000000000000000075
:20385300000000000000000000000000000000000000000000000000000000000000000055
:20387300000000000000000000000000000000000000000000000000000000000000000035
:203893000000000606060600000505000008080808000200000200030303000400000400BE
:2038B3000000000000000000000000000000000000000000000000000000000000000000F5
:2038D3000000000600000000050000050008000000000202000200000300000004040000AC
:2038F3000000000000000000000000000000000000000000000000000000000000000000B5
:2039130000000006060600000500000500080808000002000202000003000000040400004F
:20393300000000000000000000000000000000000000000000000000000000000000000074
:2039530000000006000000000500000500080000000002000202000003000000040400002B
:20397300000000000000000000000000000000000000000000000000000000000000000034
:203993000000000600000000000505000008080808000200000200030303000400000400CF
:2039B3000000000000000000000000000000000000000000000000000000000000000000F4
:2039D3000000000000000000000000000000000000000000000000000000000000000000D4
:2039F3000000000000000000000000000000000000000000000000000000000000000000B4
:203A1300000000050505050002020202000303030300080808000007070700000606000032
:203A3300000000000000000000000000000000000000000000000000000000000000000073
:203A5300000000000505000002000000000003030000080000080000070000060000000024
:203A7300000000000000000000000000000000000000000000000000000000000000000033
:203A93000000000005050000020202000000030300000800000800000700000006060000DA
:203AB3000000000000000000000000000000000000000000000000000000000000000000F3
:203AD30000000000050500000200000000000303000008080800000007000000000006009C
:203AF3000000000000000000000000000000000000000000000000000000000000000000B3
:203B130000000000050500000200000000000303000008000008000007000006000006005D
:203B3300000000000000000000000000000000000000000000000000000000000000000072
:203B5300000000000505000002020202000003030000080000080007070700000606000009
:203B7300000000000000000000000000000000000000000000000000000000000000000032
:203B9300000000000000000000000000000000000000000000000000000000000000000012
:203BB3000000000000000000000000000000000000000000000000000000000000000000F2
:203BD30000000000000000000C0C0C0C0C0C0C0C0C0C0C0C0C0C0C0C0C0C0C0C00000000E2
:203BF3000000000000000000000000000000000000000000000000000000000000000000B2
:203C130000000000000000000C0C0C0C0C0C0C0C0C0C0C0C0C0C0C0C0C0C0C0C00000000A1
:203C3300000000000000000000000000000000000000000000000000000000000000000071
:203C530000000000000000000C0C0C0C0C0C0C0C0C0C0C0C0C0C0C0C0C0C0C0C0000000061
:203C7300000000000000000000000000000000000000000000000000000000000000000031
:203C930000000000000000000C0C0C0C0C0C0C0C0C0C0C0C0C0C0C0C0C0C0C0C0000000021
:203CB3000000000000000000000000000000000000000000000000000000000000000000F1
:203CD3000000000000000000000000000000000000000000000000000000000000000000D1
:203CF3000000000000000000000000000000000000000000000000000000000000000000B1
:203D1300000000000000000000000000000000000000000000000000000000000000000090
:203D3300000000000000000000000000000000000000000000000000000000000000000070
:203D5300000000000000000000000000000000000000000000000000000000000000000050
:203D7300000000000000000000000000000000000000000000000000000000000000000030
:203D9300000000000000000000000000000000000000000000000000000000000000000010
:203DB3000000000000000000000000000000000000000000000000000000000000000000F0
:203DD3000000000000000000000000000000000000000000000000000000000000000000D0
:203DF3000000000000000000000000000000000000000000000000000000000000000000B0
:203E130000000000000000000000000000000000000000000000000000000000000000008F
:203E330000000000000000000000000000000000000000000000000000000000000000006F
:203E5300000000000000140C1400000000000000000000000000000000000000000000001B
:203E730000000000000004143C1000000000000000000000000000000000000000000000CB
:203E930000000000000000000000000000000000000000000000000000000000000000000F
:203EB3000000000000000000000000000000000000000000000000000000000000000000EF
:203ED3000000000000000000000000000000000000000000000000000000000000000000CF
:203EF3000000000000000000000000000000000000000000000000000000000000000000AF
:203F130000000000181818180000180066666600000000006666FF66FF666600183E603CF6
:203F3300067C180062660C18306646003C663C3867663F00060C1800000000000C1830303C
:203F530030180C0030180C0C0C18300000663CFF3C6600000018187E181800000000000025
:203F7300001818300000007E0000000000000000001818000003060C183060003C666E76DD
:203F930066663C001818381818187E003C66060C30607E003C66061C06663C00060E1E6612
:203FB3007F0606007E607C0606663C003C66607C66663C007E660C18181818003C66663C41
:203FD30066663C003C66663E06663C00000018000018000000001800001818300E1830607A
:203FF30030180E0000007E007E00000070180C060C1870003C66060C180018003C666E6ECC
:2040130060623C00183C667E666666007C66667C66667C003C66606060663C00786C666605
:20403300666C78007E60607860607E007E606078606060003C66606E66663C006666667E31
:20405300666666003C18181818183C001E0C0C0C0C6C3800666C7870786C660060606060B5
:2040730060607E0063777F6B6363630066767E7E6E6666003C66666666663C007C66667CB6
:20409300606060003C666666663C0E007C66667C786C66003C66603C06663C007E18181815
:2040B300181818006666666666663C0066666666663C18006363636B7F77630066663C18A6
:2040D3003C6666006666663C181818007E060C1830607E003C30303030303C0000C06030A1
:2040F300180C06003C0C0C0C0C0C3C0000183C6600000000000000000000007E60301800EF
:204113000000000000003C063E663E000060607C66667C0000003C6060603C000006063E02
:2041330066663E0000003C667E603C00000E183E1818180000003E66663E067C0060607CF4
:20415300666666000018003818183C00000600060606063C0060606C786C66000038181826
:2041730018183C000000667F7F6B630000007C666666660000003C6666663C0000007C66EE
:20419300667C606000003E66663E060600007C666060600000003E603C067C0000187E180A
:2041B30018180E000000666666663E0000006666663C18000000636B7F3E36000000663CEF
:2041D300183C660000006666663E0C7800007E0C18307E001C18183018181C0018181800BE
:2041F300181818003818180C181838000000327E4C000000000000000000000000003C3C14
:204213003C3C000000003C24243C00000000183C3C180000000018242418000018242418BB
:2042330000000000003C424266246600001800180C06663C0C12307C3062FC001C207020B3
:2042530070201C00000000000000000000000000000000000000000000000000000000009F
:2042730000000000000000000000000000000000000000000000000000000000000000002B
:2042930000000000000000000000000000000000000000000000000000000000000000000B
:2042B3000000000000000000000000000000000000000000000000000000000000000000EB
:2042D3000000000000000000000000000000000000000000000000000000000000000000CB
:2042F30000000000000000000000000000000000000000000000000000000000FFFFFFFFAF
:20431300FFFFFFFFF0F0F0F0F0F0F0F000000000FFFFFFFFFF000000000000000000000013
:20433300000000FF8080808080808080CCCC3333CCCC333301010101010101010000000067
:20435300CCCC3333FFFEFCF8F0E0C08003030303030303031818181F1F1818180000000065
:204373000F0F0F0F1818181F1F000000000000F8F8181818000000000000FFFF0000001F13
:204393001F181818181818FFFF000000000000FFFF181818181818F8F8181818C0C0C0C097
:2043B300C0C0C0C0E0E0E0E0E0E0E0E00707070707070707FFFF000000000000FFFFFF00B7
:2043D300000000000000000000FFFFFF030303030303FFFF00000000F0F0F0F00F0F0F0FC1
:2043F30000000000181818F8F8000000F0F0F0F000000000F0F0F0F00F0F0F0F000000FFB7
:20441300FF000000081C3E7F7F1C3E001818181818181818000000FFFF0000000000FFFF14
:204433000000000000FFFF000000000000000000FFFF000030303030303030300C0C0C0CBD
:204453000C0C0C0C000000E0F038181818181C0F07000000181838F0E0000000C0C0C0C047
:20447300C0C0FFFFC0E070381C0E070303070E1C3870E0C0FFFFC0C0C0C0C0C0FFFF030331
:2044930003030303003C7E7E7E7E3C000000000000FFFF00367F7F7F3E1C080060606060FA
:2044B30060606060000000070F1C1818C3E77E3C3C7EE7C3003C7E66667E3C001818666603
:2044D30018183C000606060606060606081C3E7F3E1C0800181818FFFF181818C0C030307C
:2044F300C0C0303018181818181818180000033E76363600FF7F3F1F0F07030100000000F0
:20451300000000000000000000000000000000000000000000000000000000000000000088
:20453300000000000000000000000000000000000000000000000000000000000000000068
:2045530000000000CC993366CC9933663399CC663399CC6602060CD8F0E0C0000103070FBA
:204573001F3F7FFF80C0E0F0F8FCFEFFFFFFFFFF000000000F0F0F0F0F0F0F0FF0F0F0F017
:20459300FFFFFFFF0F0F0F0FFFFFFFFFFFFFFFFFF0F0F0F0FFFFFFFF0F0F0F0F0C0C0303C2
:2045B30000000000000000000C0C0303C0C030300000000000000000C0C030300C0C0303EC
:2045D3000C0C0303CCCC33330000000000183C7E181818180010307F7F30100000080CFEEA
:2045F300FE0C0800181818187E3C18000000364936000000000000000000000056676D2065
:204613006300000051010000999E360000000000000000005A4800000000000000000000C3
:20463300000000000600100500000000000000000C000000000000000000000050E550F0CB
:2046530063636350F263636350F463636350F663636350F863636350FA63636350FC6363E1
:204673006350FF6656676D209100000051010000999E36000000000000000000A58400004C
:204693000000000000000000000000000600100500000000000000000C00000000000000E0
:2046B300000000005088500F509063636363509D636363635085500C509063636363509D41
:2046D300636363635085500A509063636363509D63636363508C5007509063636363509D9B
:2046F30063636363508C5009509063636363509462509762509C62509F6656676D20B285C7
:20471300010051010000000000000000000066840100A5D7430073000000A5D74300E8036C
:2047330000000000000000000000000000004C00000000000000000000000000000000001A
:2047530000000000000000000000000000000000000000000000647ADA000000000000008E
:2047730000000000000000000000000000000000000000000000000000005F05015F04005E
:204793005E01205E08005EBD205EC0305E20015E40805E60925E808A5EC0385EE0005E232E
:2047B300E55E433F5E63C15E839E5EE3005EA0575EB0015E430B5EA0985EB02D5EC1305E51
:2047D30021015E41805E61925E818A5EC1385EE1005E24E55E443F5E64C15E849E5EE400A8
:2047F3005EA1575EB1015E440B5EA1225EB12A5EC2105E22015E42805E62925E828A5EC28C
:20481300185EE2005E25E55E453F5E65C15E859E5EE5005EA2685EB2015E450B5EA2945E82
:20483300B22D5EC3205E28015E48805E68925E888A5EC3285EE8005E2BE55E4B3F5E6BC161
:204853005E8B9E5EEB005EA3685EB3015E4B0B5EA31C5EB32A5EC4305E29015E49805E6926
:20487300925E898A5EC4385EE9005E2CE55E4C3F5E6CC15E8C9E5EEC005EA4575EB4015E02
:204893004C145EC5305E2A205E4A0B5E6AF45E8AE15EC5345EEA015E2D205E4D3F5E6DF37F
:2048B3005E8D545EED005EA5575EB5015E4D055EA5225EB52A5EC6305E30005E50075E7076
:2048D300D85E90FF5EC6385EF0005E33005E533F5E73F55E93F05EF3005EA6575EB6015E0F
:2048F30053055EB6095EBD305EC7305E341E5E543F5E74F55E94D75EF4025E54055EBD3801
:204913005EC8305E32045E523F5E72F75E92B55EF2005EC8315E52055EA8665EB8025EA75A
:20493300CB5EB7055EBD3C5EC8115E350E5E553F5E75C95E95045EF5005E550B5EBD3E5E03
:2049530031015E513F5E71985E91065EF1005EC7395E510B5FC0205F20015F40805F609232
:204973005F808A5FC0285FE0005F23E55F433F5F63C15F839E5FE3005FA0575FB0015F43A0
:20499300105FA0985FB02D5FC1105F21015F41805F61925F818A5FC1185FE1005F24E55F55
:2049B300443F5F64C15F849E5FE4005FA1575FB1015F44105FA1225FB12A5FC2305F2201CF
:2049D3005F42805F62925F828A5FC2385FE2005F25E55F453F5F65C15F859E5FE5005FA2B3
:2049F300575FB2015F45145FC3305F28015F48805F68925F888A5FC3385FE8005F2BE55F49
:204A13004B3F5F6BC15F8B9E5FEB005FA3575FB3015F4B145FC4305F29015F49805F699214
:204A33005F898A5FC4385FE9005F2CE55F4C3F5F6CC15F8C9E5FEC005FA4575FB4015F4C7B
:204A5300145FC5305F2AA05F4A045F6AF55F8AC15FC5325FEA015F2DC05F4D3F5F6DF05FAB
:204A73008D045FED005FA5695FB5015F4D055FA51F5FB52A5FC6305F30015F50805F70923D
:204A93005F908A5FC6385FF0005F33E55F533F5F73C15F939E5FF3005FA6575FB6015F53DD
:204AB300145FC7305F31015F51805F71925F918A5FC7385FF1005F34E55F543F5F74C15FD1
:204AD300949E5FF4005FA7575FB7015F54145FC8305F32015F52805F72925F928A5FC838AC
:204AF3005FF2005F35E55F553F5F75C15F959E5FF5005FA8575FB8015F551461D2045EBDDB
:204B13002E5EBD3E5EBD365EBD3E5EBD3A5EBD3E5EBD3C61FF045EBD2C5EBD245EBD2061C6
:204B3300D10E5EB50A5FB50A61D3045EB00D5EB0295EB10A5EB12A5EB20D5EB2295EB30AFB
:204B53005EB32A5EB52A5EBD305E71F85E91CA5EBD315FB00D5FB0295FB10A5FB12A5FB5F7
:204B73002A61FF045EBD215EBD2061D2045EB50A5FB50A61FF045EB0095EB10A5EB2095EA0
:204B9300B30A5FB0095FB10A61D10E5EA0665EB02E5EA1985EB12D5EA25F5EB22E5EA3942E
:204BB3005EB32D5EA5985EB52D5EBD305EBD385EBD3C5E71985E91065EBD3D5FA0665FB0AC
:204BD3002E5FA1985FB12D5FA5965FB52D61D3045EBD355EBD315EBD3061D1095EBD2061EE
:204BF300D2095EB50D5FB50D61FF045EB00E5EA0985EB0295EB10D5EA1225EB12A5EB20EA5
:204C13005EA2945EB2295EB30D5EA31C5EB32A5EA5225EB52A5EBD305E71F85E91CA5EBDF6
:204C3300315FB00E5FA0985FB0295FB10D5FA1225FB12A5FA51F5FB52A61FF045EBD215E6C
:204C5300BD2061D3045EB50A5FB50A61FF045EB0095EB10A5EB2095EB30A5FB0095FB10AF7
:204C730061A40E5EA08A5EB02E5EA1B15EB12D5EA2835EB22E5EA3AC5EB32D5EA5B15EB5EB
:204C93002D5EBD305EBD385EBD3C5E71985E91065EBD3D5FA08A5FB02E5FA1B15FB12D5F18
:204CB300A5AE5FB52D61FF045EBD355EBD315EBD3061D2095EBD2061D1095EB50D5FB50D0F
:204CD30061FF045EB00E5EA0985EB0295EB10D5EA1225EB12A5EB20E5EA2945EB2295EB302
:204CF3000D5EA31C5EB32A5EA5225EB52A5EBD305E71F85E91CA5EBD315FB00E5FA0985FB0
:204D1300B0295FB10D5FA1225FB12A5FA51F5FB52A61D3045EBD215EBD2061FF045EB50A9D
:204D33005FB50A61FF045EB0095EB10A5EB2095EB30A5FB0095FB10A61A40E5EA0225EB007
:204D53002E5EA16C5EB12D5EA21C5EB22E5EA3685EB32D5EA56C5EB52D5EBD305EBD385EBF
:204D7300BD3C5E71985E91065EBD3D5FA0225FB02E5FA16C5FB12D5FA5695FB52D61FF045A
:204D93005EBD355EBD315EBD3061D2095EBD2061D2095EB50D5FB50D61FF045EB00E5EA0A7
:204DB300985EB0295EB10D5EA1225EB12A5EB20E5EA2945EB2295EB30D5EA31C5EB32A5EDC
:204DD300A5225EB52A5EBD305E71F85E91CA5EBD315FB00E5FA0985FB0295FB10D5FA1227A
:204DF3005FB12A5FA51F5FB52A61D2045EBD215EBD2061FF045EB50A5FB50A61D3045EB072
:204E1300095EB10A5EB2095EB30A5FB0095FB10A61D10E5EA0665EB02E5EA1985EB12D5EE6
:204E3300A25F5EB22E5EA3945EB32D5EA5985EB52D5EBD305EBD385EBD3C5E71985E910621
:204E53005EBD3D5FA0665FB02E5FA1985FB12D5FA5965FB52D61D3045EBD355EBD315EBDA6
:204E73003061FD095EBD2061D2095EB50D5FB50D61D3045EB00E5EA0985EB0295EB10D5E35
:204E9300A1225EB12A5EB20E5EA2945EB2295EB30D5EA31C5EB32A5EA5225EB52A5EBD30F5
:204EB3005E71F85E91CA5EBD315FB00E5FA0985FB0295FB10D5FA1225FB12A5FA51F5FB577
:204ED3002A61FF045EBD215EBD2061D3045EB50A5FB50A61FE045EB0095EB10A5EB2095E3D
:204EF300B30A5FB0095FB10A61D10E5EA0E65EB02D5EA18A5EB12A5EA2E15EB22D5EA383ED
:204F13005EB32A5EA58A5EB52A5EBD305EBD385EBD3C5E71985E91065EBD3D5FA0E65FB0DC
:204F33002D5FA18A5FB12A5FA5865FB52A61D3045EBD355EBD315EBD3061D2095EBD2061AE
:204F5300D1095EB50A5FB50A61FF045EB00D5EA0985EB0295EB10A5EA1225EB12A5EB20D4D
:204F73005EA2945EB2295EB30A5EA31C5EB32A5EA5225EB52A5EBD305E71F85E91CA5EBD96
:204F9300315FB00D5FA0985FB0295FB10A5FA1225FB12A5FA51F5FB52A61D3045EBD215E39
:204FB300BD2061FF045EB50A5FB50A61FF045EB0095EB10A5EB2095EB30A5FB0095FB10A68
:204FD30061A40E5EA0225EB02E5EA16C5EB12D5EA21C5EB22E5EA3685EB32D5EA56C5EB525
:204FF3002D5EBD305EBD385EBD3C5E71985E91065EBD3D5FA0225FB02E5FA16C5FB12D5F62
:20501300A5695FB52D61FF045EBD355EBD315EBD3061D2095EBD2061D2095EB50D5FB50DEF
:2050330061FE045EB00E5EA0985EB0295EB10D5EA1225EB12A5EB20E5EA2945EB2295EB39F
:205053000D5EA31C5EB32A5EA5225EB52A5EBD305E71F85E91CA5EBD315FB00E5FA0985F4C
:20507300B0295FB10D5FA1225FB12A5FA51F5FB52A61D3045EBD215EBD2061FF045EB50A3A
:205093005FB50A61D3045EB0095EB10A5EB2095EB30A5FB0095FB10A61D10E5EA0CB5EB0FA
:2050B3002D5EA1665EB12A5EA2C65EB22D5EA35F5EB32A5EA5665EB52A5EBD305EBD385ED2
:2050D300BD3C5E71985E91065EBD3D5FA0CB5FB02D5FA1665FB12A5FA5625FB52A61FE0463
:2050F3005EBD355EBD315EBD3061D2095EBD2061D2095EB50A5FB50A61D3045EB00D5EA077
:20511300985EB0295EB10A5EA1225EB12A5EB20D5EA2945EB2295EB30A5EA31C5EB32A5E7F
:20513300A5225EB52A5EBD305E71F85E91CA5EBD315FB00D5FA0985FB0295FB10A5FA1221A
:205153005FB12A5FA51F5FB52A61FF045EBD215EBD2061D2045EB50A5FB50A61FF045EB0E2
:20517300095EB10A5EB2095EB30A5FB0095FB10A61D10E5EB02D5EB12A5EB22D5EB32A5E0A
:20519300B52A5EBD305EBD385EBD3C5E71985E91065EBD3D5FB02D5FB12A5FB52A61D30488
:2051B3005EBD2D5EBD3D5EBD355EBD3D5EBD395EBD3D5EBD3C61FF045EBD2C5EBD245EBD8C
:2051D3002061D00E5EB50A5FB50A61D3045EB00D5EB0295EB10A5EB12A5EB20D5EB2295E92
:2051F300B30A5EB32A5EB52A5EBD305E71F85E91CA5EBD315FB00D5FB0295FB10A5FB12AA8
:205213005FB52A61FF045EBD215EBD2061D3045EB50A5FB50A61FF045EB0095EB10A5EB24B
:20523300095EB30A5FB0095FB10A61A40E5EA0665EB02E5EA1985EB12D5EA25F5EB22E5E84
:20525300A3945EB32D5EA5985EB52D5EBD305EBD385EBD3C5E71985E91065EBD3D5FA066DD
:205273005FB02E5FA1985FB12D5FA5965FB52D61FF045EBD355EBD315EBD3061D2095EBD8C
:205293002061D1095EB50D5FB50D61FF045EB00E5EA0985EB0295EB10D5EA1225EB12A5E3E
:2052B300B20E5EA2945EB2295EB30D5EA31C5EB32A5EA5225EB52A5EBD305E71F85E91CAAB
:2052D3005EBD315FB00E5FA0985FB0295FB10D5FA1225FB12A5FA51F5FB52A61D3045EBD56
:2052F300215EBD2061FF045EB50A5FB50A61FF045EB0095EB10A5EB2095EB30A5FB0095F61
:20531300B10A61A40E5EA08A5EB02E5EA1B15EB12D5EA2835EB22E5EA3AC5EB32D5EA5B19C
:205333005EB52D5EBD305EBD385EBD3C5E71985E91065EBD3D5FA08A5FB02E5FA1B15FB1EA
:205353002D5FA5AE5FB52D61FF045EBD355EBD315EBD3061D2095EBD2061D2095EB50D5F9D
:20537300B50D61FF045EB00E5EA0985EB0295EB10D5EA1225EB12A5EB20E5EA2945EB229AA
:205393005EB30D5EA31C5EB32A5EA5225EB52A5EBD305E71F85E91CA5EBD315FB00E5FA0EF
:2053B300985FB0295FB10D5FA1225FB12A5FA51F5FB52A61D2045EBD215EBD2061FF045EC0
:2053D300B50A5FB50A61D3045EB0095EB10A5EB2095EB30A5FB0095FB10A61D10E5EA022AF
:2053F3005EB02E5EA16C5EB12D5EA21C5EB22E5EA3685EB32D5EA56C5EB52D5EBD305EBDA1
:20541300385EBD3C5E71985E91065EBD3D5FA0225FB02E5FA16C5FB12D5FA5695FB52D6120
:20543300D2045EBD355EBD315EBD3061FE095EBD2061D2095EB50D5FB50D61D3045EB00E28
:205453005EA0985EB0295EB10D5EA1225EB12A5EB20E5EA2945EB2295EB30D5EA31C5EB3BF
:205473002A5EA5225EB52A5EBD305E71F85E91CA5EBD315FB00E5FA0985FB0295FB10D5F0E
:20549300A1225FB12A5FA51F5FB52A61FF045EBD215EBD2061D2045EB50A5FB50A61FF04EA
:2054B3005EB0095EB10A5EB2095EB30A5FB0095FB10A61D10E5EA0665EB02E5EA1985EB1BD
:2054D3002D5EA25F5EB22E5EA3945EB32D5EA5985EB52D5EBD305EBD385EBD3C5E71985E87
:2054F30091065EBD3D5FA0665FB02E5FA1985FB12D5FA5965FB52D61D3045EBD355EBD3184
:205513005EBD3061D1095EBD2061D2095EB50D5FB50D61FF045EB00E5EA0985EB0295EB1DE
:205533000D5EA1225EB12A5EB20E5EA2945EB2295EB30D5EA31C5EB32A5EA5225EB52A5ED0
:20555300BD305E71F85E91CA5EBD315FB00E5FA0985FB0295FB10D5FA1225FB12A5FA51FF7
:205573005FB52A61FF045EBD215EBD2061D3045EB50A5FB50A61FF045EB0095EB10A5EB2E8
:20559300095EB30A5FB0095FB10A61A40E5EA0E65EB02D5EA18A5EB12A5EA2E15EB22D5E32
:2055B300A3835EB32A5EA58A5EB52A5EBD305EBD385EBD3C5E71985E91065EBD3D5FA0E61F
:2055D3005FB02D5FA18A5FB12A5FA5865FB52A61FF045EBD355EBD315EBD3061D2095EBD4E
:2055F3002061D1095EB50A5FB50A61FF045EB00D5EA0985EB0295EB10A5EA1225EB12A5EE5
:20561300B20D5EA2945EB2295EB30A5EA31C5EB32A5EA5225EB52A5EBD305E71F85E91CA4B
:205633005EBD315FB00D5FA0985FB0295FB10A5FA1225FB12A5FA51F5FB52A61D3045EBDF6
:20565300215EBD2061FF045EB50A5FB50A61D3045EB0095EB10A5EB2095EB30A5FB0095F29
:20567300B10A61D00E5EA0225EB02E5EA16C5EB12D5EA21C5EB22E5EA3685EB32D5EA56CAA
:205693005EB52D5EBD305EBD385EBD3C5E71985E91065EBD3D5FA0225FB02E5FA16C5FB134
:2056B3002D5FA5695FB52D61FF045EBD355EBD315EBD3061D2095EBD2061D2095EB50D5F7F
:2056D300B50D61D3045EB00E5EA0985EB0295EB10D5EA1225EB12A5EB20E5EA2945EB22973
:2056F3005EB30D5EA31C5EB32A5EA5225EB52A5EBD305E71F85E91CA5EBD315FB00E5FA08C
:20571300985FB0295FB10D5FA1225FB12A5FA51F5FB52A61FE045EBD215EBD2061FF045E30
:20573300B50A5FB50A61D3045EB0095EB10A5EB2095EB30A5FB0095FB10A61D10E5EA0CBA2
:205753005EB02D5EA1665EB12A5EA2C65EB22D5EA35F5EB32A5EA5665EB52A5EBD305EBDB3
:20577300385EBD3C5E71985E91065EBD3D5FA0CB5FB02D5FA1665FB12A5FA5625FB52A6128
:20579300D3045EBD355EBD315EBD3061FD095EBD2061D2095EB50A5FB50A61D3045EB00DCC
:2057B3005EA0985EB0295EB10A5EA1225EB12A5EB20D5EA2945EB2295EB30A5EA31C5EB363
:2057D3002A5EA5225EB52A5EBD305E71F85E91CA5EBD315FB00D5FA0985FB0295FB10A5FAF
:2057F300A1225FB12A5FA51F5FB52A61FF045EBD215EBD2061D3045EB50A5FB50A61FE0487
:205813005EB0095EB10A5EB2095EB30A5FB0095FB10A61D10E5EB02D5EB12A5EB22D5EB3DD
:205833002A5EB52A5EBD305EBD385EBD3C5E71985E91065EBD3D5FB02D5FB12A5FB52A6130
:20585300D3045EBD2D5EBD3D5EBD355EBD3D5EBD395EBD3D5EBD3C61FF045EBD2C5EBD2429
:205873005EBD2061A40E5EB50A5FB50A61FF045EB00D5EB0295EB10A5EB12A5EB20D5EB257
:20589300295EB30A5EB32A5EB52A5EBD305E71F85E91CA5EBD315FB00D5FB0295FB10A5F55
:2058B300B12A5FB52A61D3045EBD215EBD2061FF045EB50A5FB50A61FF045EB0095EB10ADA
:2058D3005EB2095EB30A5FB0095FB10A61A40E5EA0665EB02E5EA1985EB12D5EA25F5EB25A
:2058F3002E5EA3945EB32D5EA5985EB52D5EBD305EBD385EBD3C5E71985E91065EBD3D5FB1
:20591300A0665FB02E5FA1985FB12D5FA5965FB52D61FF045EBD355EBD315EBD3061D209FA
:205933005EBD2061D2095EB50D5FB50D61FE045EB00E5EA0985EB0295EB10D5EA1225EB104
:205953002A5EB20E5EA2945EB2295EB30D5EA31C5EB32A5EA5225EB52A5EBD305E71F85ED7
:2059730091CA5EBD315FB00E5FA0985FB0295FB10D5FA1225FB12A5FA51F5FB52A61D3046F
:205993005EBD215EBD2061FF045EB50A5FB50A61D3045EB0095EB10A5EB2095EB30A5FB033
:2059B300095FB10A61D10E5EA08A5EB02E5EA1B15EB12D5EA2835EB22E5EA3AC5EB32D5EB7
:2059D300A5B15EB52D5EBD305EBD385EBD3C5E71985E91065EBD3D5FA08A5FB02E5FA1B1FE
:2059F3005FB12D5FA5AE5FB52D61FE045EBD355EBD315EBD3061D2095EBD2061D2095EB554
:205A13000D5FB50D61D3045EB00E5EA0985EB0295EB10D5EA1225EB12A5EB20E5EA2945E9E
:205A3300B2295EB30D5EA31C5EB32A5EA5225EB52A5EBD305E71F85E91CA5EBD315FB00E6C
:205A53005FA0985FB0295FB10D5FA1225FB12A5FA51F5FB52A61FF045EBD215EBD2061D27C
:205A7300045EB50A5FB50A61FF045EB0095EB10A5EB2095EB30A5FB0095FB10A61D10E5E3C
:205A9300A0225EB02E5EA16C5EB12D5EA21C5EB22E5EA3685EB32D5EA56C5EB52D5EBD3053
:205AB3005EBD385EBD3C5E71985E91065EBD3D5FA0225FB02E5FA16C5FB12D5FA5695FB5ED
:205AD3002D61D3045EBD355EBD315EBD3061D1095EBD2061FE095EB50D5FB50D61D3045EB2
:205AF300B00E5EA0985EB0295EB10D5EA1225EB12A5EB20E5EA2945EB2295EB30D5EA31C6C
:205B13005EB32A5EA5225EB52A5EBD305E71F85E91CA5EBD315FB00E5FA0985FB0295FB1C2
:205B33000D5FA1225FB12A5FA51F5FB52A61FF045EBD215EBD2061D3045EB50A5FB50A61D9
:205B5300FF045EB0095EB10A5EB2095EB30A5FB0095FB10A61A40E5EA0665EB02E5EA1984F
:205B73005EB12D5EA25F5EB22E5EA3945EB32D5EA5985EB52D5EBD305EBD385EBD3C5E71C7
:205B9300985E91065EBD3D5FA0665FB02E5FA1985FB12D5FA5965FB52D61FF045EBD355EA9
:205BB300BD315EBD3061D2095EBD2061D1095EB50D5FB50D61FF045EB00E5EA0985EB02959
:205BD3005EB10D5EA1225EB12A5EB20E5EA2945EB2295EB30D5EA31C5EB32A5EA5225EB5A3
:205BF3002A5EBD305E71F85E91CA5EBD315FB00E5FA0985FB0295FB10D5FA1225FB12A5F8D
:205C1300A51F5FB52A61D3045EBD215EBD2061FF045EB50A5FB50A61FF045EB0095EB10A8D
:205C33005EB2095EB30A5FB0095FB10A61A40E5EA0E65EB02D5EA18A5EB12A5EA2E15EB206
:205C53002D5EA3835EB32A5EA58A5EB52A5EBD305EBD385EBD3C5E71985E91065EBD3D5F73
:205C7300A0E65FB02D5FA18A5FB12A5FA5865FB52A61FF045EBD355EBD315EBD3061D2093C
:205C93005EBD2061D2095EB50A5FB50A61FF045EB00D5EA0985EB0295EB10A5EA1225EB1AA
:205CB3002A5EB20D5EA2945EB2295EB30A5EA31C5EB32A5EA5225EB52A5EBD305E71F85E78
:205CD30091CA5EBD315FB00D5FA0985FB0295FB10A5FA1225FB12A5FA51F5FB52A61D20411
:205CF3005EBD215EBD2061FF045EB50A5FB50A61D3045EB0095EB10A5EB2095EB30A5FB0D0
:205D1300095FB10A61D10E5EA0225EB02E5EA16C5EB12D5EA21C5EB22E5EA3685EB32D5EAB
:205D3300A56C5EB52D5EBD305EBD385EBD3C5E71985E91065EBD3D5FA0225FB02E5FA16C8C
:205D53005FB12D5FA5695FB52D61D2045EBD355EBD315EBD3061FE095EBD2061D2095EB535
:205D73000D5FB50D61D3045EB00E5EA0985EB0295EB10D5EA1225EB12A5EB20E5EA2945E3B
:205D9300B2295EB30D5EA31C5EB32A5EA5225EB52A5EBD305E71F85E91CA5EBD315FB00E09
:205DB3005FA0985FB0295FB10D5FA1225FB12A5FA51F5FB52A61FF045EBD215EBD2061D219
:205DD300045EB50A5FB50A61FF045EB0095EB10A5EB2095EB30A5FB0095FB10A61D10E5ED9
:205DF300A0CB5EB02D5EA1665EB12A5EA2C65EB22D5EA35F5EB32A5EA5665EB52A5EBD30BD
:205E13005EBD385EBD3C5E71985E91065EBD3D5FA0CB5FB02D5FA1665FB12A5FA5625FB5F1
:205E33002A61D3045EBD355EBD315EBD3061D1095EBD2061D2095EB10A5EB30A5EB50A5FA4
:205E5300B10A5FB50A61FF045EB00D5EA0985EB0295EA1225EB12A5EB20D5EA2945EB229C6
:205E73005EA31C5EB32A5EA5225EB52A5EBD305E71F85E91CA5EBD315FB00D5FA0985FB07C
:205E9300295FA1225FB12A5FA51F5FB52A61FF045EBD215EBD2061D3045EB50A5FB50A615A
:205EB300FF045EB0095EB10A5EB2095EB30A5FB0095FB10A61A40E5EB02D5EB12A5EB22D72
:205ED3005EB32A5EB52A5EBD305EBD385EBD3C5E71985E91065EBD3D5FB02D5FB12A5FB504
:205EF3002A61FF045EBD355EBD3D5EBD395EBD3D5EBD3C61D3045EBD345EBD3061FF045EC2
:205F1300BD2061D1095EB50A5FB50A61FF045EB00D5EB0295EB10A5EB12A5EB20D5EB229BD
:205F33005EB30A5EB32A5EB52A5EBD305E71F85E91CA5EBD315FB00D5FB0295FB10A5FB126
:205F53002A5FB52A61D3045EBD215EBD2061FF045EB50A5FB50A61D3045EB0095EB10A5EB2
:205F7300B2095EB30A5FB0095FB10A61D00E5EA0665EB02E5EA1985EB12D5EA25F5EB22EB7
:205F93005EA3945EB32D5EA5985EB52D5EBD305EBD385EBD3C5E71985E91065EBD3D5FA098
:205FB300665FB02E5FA1985FB12D5FA5965FB52D61FF045EBD355EBD315EBD3061D2095E96
:205FD300BD2061D2095EB50D5FB50D61D3045EB00E5EA0985EB0295EB10D5EA1225EB12ABD
:205FF3005EB20E5EA2945EB2295EB30D5EA31C5EB32A5EA5225EB52A5EBD305E71F85E91CA
:20601300CA5EBD315FB00E5FA0985FB0295FB10D5FA1225FB12A5FA51F5FB52A61FE045ED0
:20603300BD215EBD2061FF045EB50A5FB50A61D3045EB0095EB10A5EB2095EB30A5FB009E1
:206053005FB10A61D10E5EA08A5EB02E5EA1B15EB12D5EA2835EB22E5EA3AC5EB32D5EA574
:20607300B15EB52D5EBD305EBD385EBD3C5E71985E91065EBD3D5FA08A5FB02E5FA1B15F9D
:20609300B12D5FA5AE5FB52D61D3045EBD355EBD315EBD3061FD095EBD2061D2095EB50DFF
:2060B3005FB50D61D3045EB00E5EA0985EB0295EB10D5EA1225EB12A5EB20E5EA2945EB253
:2060D300295EB30D5EA31C5EB32A5EA5225EB52A5EBD305E71F85E91CA5EBD315FB00E5F19
:2060F300A0985FB0295FB10D5FA1225FB12A5FA51F5FB52A61FF045EBD215EBD2061D30430
:206113005EB50A5FB50A61FE045EB0095EB10A5EB2095EB30A5FB0095FB10A61D10E5EA0FA
:20613300225EB02E5EA16C5EB12D5EA21C5EB22E5EA3685EB32D5EA56C5EB52D5EBD305EEE
:20615300BD385EBD3C5E71985E91065EBD3D5FA0225FB02E5FA16C5FB12D5FA5695FB52D77
:2061730061D3045EBD355EBD315EBD3061D2095EBD2061D1095EB50D5FB50D61FF045EB088
:206193000E5EA0985EB0295EB10D5EA1225EB12A5EB20E5EA2945EB2295EB30D5EA31C5E17
:2061B300B32A5EA5225EB52A5EBD305E71F85E91CA5EBD315FB00E5FA0985FB0295FB10D6D
:2061D3005FA1225FB12A5FA51F5FB52A61D3045EBD215EBD2061FF045EB50A5FB50A61FF41
:2061F300045EB0095EB10A5EB2095EB30A5FB0095FB10A61A40E5EA0225EB02E5EA1985E8E
:20621300B12D5EA21C5EB22E5EA3945EB32D5EB52A5EBD305EBD385EBD3C5EC8215EBD3E8E
:206233005FA0225FB02E5FA1985FB12D5FB52A61FF045EBD2E5EBD3E5EBD365EBD3E5EBD0F
:206253003A5EBD3E5EBD3C61D3045EBD345EBD3061FE095EBD2061D3045EB50A5FB50A61F8
:20627300FE045EB00E5EB10D5EB20E5EB30D5EBD305EBD315FB00E5FB10D61D3045EBD2150
:206293005EBD2061A3185EBD305EBD3161FE045EBD215EBD206177185EB02E5EB12D5EB2AB
:2062B3002E5EB32D5EB52A5EBD305EBD385EBD3C5EC8115EBD3E5FB02E5FB12D5FB52A6184
:2062D300FF045EBD365EBD325EBD3061D1095EBD2061D10E5EC6285E30325E50445E70F845
:2062F3005EC62E5E33115E937F5EB60D5EBD305E34325E54495E74F85E94FF5EF4005EBDD4
:20631300385EBD3C5E71985E91065EBD3D61D3045EBD3C61D1095EBD3461D10E5EB20E5E52
:20633300C2385E62815E827A5EE2025E25C35E857E5EA21F5EB2325E29215E49145E6971D0
:206353005E89AE5EC43A5E2C315E6CF05E8CFC5EEC015E4C0B5EA4225EB4325EBD245EC613
:206373003E5EA6435EB60A5EBD345EBD3C5EBD385EBD3C5FC2185FA25B5F450D5FA2295F48
:20639300B2325FA3655F4B0D5FA3195FB32E61FF045EA2225EA4255FA22C5FA31C61D3045D
:2063B3005EA2255EA4295FA22F5FA31F61FF045EA2225EA4255EBD345FA22C5FA31C61D2AF
:2063D300045EA21F5EA4225FA2295FA31961FF045EA2225EA4255FA22C5FA31C61D3045E90
:2063F300B2125EA2255EA2695EB2325EB30D5EC3385E68815E887A5EE8025E2BC35E8B7EDD
:206413005E4B105EA31C5EB3325EB4125EA4295EA46D5EB4325EBD245EC61E5EA6B15EB604
:20643300095EBD345EBD3C5EBD385EBD3C5FB2125FA22F5FA2745FB2325FB30E5FA31F5F45
:20645300A3625FB32E61FF045EA2665EA31F5EA4695FA2705FA35F61FF045EA2625EA322D4
:206473005EA4665FA26D5FA35B61D3045EA2665EA31F5EA4695EBD345FA2705FA35F61FF2C
:20649300045EA2695EA31C5EA46D5FA2745FA36261D2045EA2665EA31F5EA4695FA2705F1F
:2064B300A35F61FF045EB2125EA2625EA2865EB2325EB3125EA3225EA3665EB3325EB41203
:2064D3005EA4665EA48A5EB4325EBD245EC63E5E30005E50075E70D85EC6385E33005E9309
:2064F300F05EA6575EBD345EBD305FB2125FA26D5FA2925FB2325FB30E5FA35B5FA37F5FE0
:20651300B32E61D3045EA28A5EA3625EA48D5EBD205FA2955FA38361FF045EA28D5EA35F2C
:206533005EA4925FA29A5FA38661FF045EA28A5EA3625EA48D5FA2955FA38361D3045EA25E
:20655300865EA3665EA48A5FA2925FA37F61FF045EA28A5EA3625EA48D5EB50A5FA2955FA9
:20657300A3835FB50A61D2045EB00E5EB02E5EB10D5EB12D5EB2125EA28D5EA2255EB232C7
:206593005EB3125EA35F5EA3835EB3325EB4125EA4925EA4295EB4325EB52A5EBD305EC8C9
:2065B300215EBD325FB00E5FB02E5FB10D5FB12D5FB2125FA29A5FA22F5FB2325FB30E5FF6
:2065D300A3865FA31F5FB32E5FB52A61FF045EA2225EA3865EA4255EBD225EBD205FA22C07
:2065F3005FA31C61D3045EA21F5EA38A5EA4225FA2295FA31961FF045EA2225EA3865EA410
:20661300255FA22C5FA31C61D3045EA2255EA3835EA4295FA22F5FA31F61FF045EA2225EB6
:20663300A3865EA4255EB50A5FA22C5FA31C5FB50A61FF045EB00E5EB02A5EB10D5EB12965
:206653005EA21F5EB3125EA38A5EA3225EB3325EA4225EB52A5E71F85E91CA5EBD215FB0C8
:206673000E5FB02A5FB10D5FB1295FA2295FA3195FB52A61D2045EA2225EA31F5EA4255EE9
:20669300BD205FA22C5FA31C61FF045EA2255EA31C5EA4295FA22F5FA31F61D3045EB00A4D
:2066B3005EB1095EA2225EA31F5EA4255FB00A5FB1095FA22C5FA31C61FF045EA21F5EA345
:2066D300225EA4225FA2295FA31961D3045EA2225EA31F5EA4255EB50A5FA22C5FA31C5FB4
:2066F300B50A61FF045EB02A5EB1295EA2255EA31C5EA4295EB52A5EBD305E341E5E540598
:206713005E74F55E94D75EF4025EBD385EBD3C5EBD3D5FB02A5FB1295FA22F5FA31F5FB5A9
:206733002A61D2045EA2225EA31F5EA4255EBD355EBD315EBD305FA22C5FA31C61FF045E88
:20675300A21F5EA3225EA4225FA2295FA31961FF045EB00A5EB1095EA2225EA31F5EA425DC
:206773005EBD205FB00A5FB1095FA22C5FA31C61D3045EA2255EA31C5EA4295FA22F5FA377
:206793001F61FF045EA2225EA31F5EA4255EB50A5FA22C5FA31C5FB50A61D3045EB02E5EA2
:2067B300B12D5EB2125EA21F5EA2625EB2325EA3225EB4125EA4225EA4665EB4325EB52AAF
:2067D3005EBD305EBD315FB02E5FB12D5FB2125FA2295FA26D5FB2325FB30E5FA3195FA35A
:2067F3005B5FB32E5FB52A61FF045EA2665EA31F5EA4695EBD215EBD205FA2705FA35F61AE
:20681300D2045EA2695EA31C5EA46D5FA2745FA36261FF045EA2665EA31F5EA4695FA270FB
:206833005FA35F61FF045EA2625EA3225EA4665FA26D5FA35B61D3045EA2665EA31F5EA408
:20685300695EB50A5FA2705FA35F5FB50A61FF045EB00E5EB02A5EB10D5EB1295EA2695EDC
:20687300B3125EA31C5EA35F5EB3325EA46D5EB52A5EBD215FB00E5FB02A5FB10D5FB129EC
:206893005FA2745FA3625FB52A61D3045EA2665EA3625EA4695EBD205FA2705FA35F61FFF5
:2068B300045EA2625EA3665EA4665FA26D5FA35B61D2045EB00A5EB1095EA2665EA3625E37
:2068D300A4695FB00A5FB1095FA2705FA35F61FF045EA2695EA35F5EA46D5FA2745FA3621F
:2068F30061D3045EA2665EA3625EA4695EB50A5FA2705FA35F5FB50A61FF045EB02A5EB161
:20691300295EA2625EA3665EA4665EB52A5EBD305EBD315FB02A5FB1295FA26D5FA35B5F9A
:20693300B52A61FF045EA2665EA3625EA4695EBD215EBD205FA2705FA35F61D3045EA269E3
:206953005EA35F5EA46D5FA2745FA36261FF045EB00A5EB1095EA2665EA3625EA4695FB0A5
:206973000A5FB1095FA2705FA35F61D2045EA2625EA3665EA4665FA26D5FA35B61FF045E1A
:20699300A2665EA3625EA4695EB50A5FA2705FA35F5FB50A61D3045EB02E5EB12D5EB2122F
:2069B3005EA2695EA28D5EB2325EA35F5EB4125EA46D5EA4925EB4325EB52A5EBD305EBD1E
:2069D300385EBD3C5EBD3D5FB02E5FB12D5FB2125FA2745FA29A5FB2325FB30E5FA3625FEA
:2069F300A3865FB32E5FB52A61FF045EA28A5EA3625EA48D5EBD355EBD315EBD305FA29580
:206A13005FA38361D3045EA2865EA3665EA48A5FA2925FA37F61FF045EA28A5EA3625EA4C6
:206A33008D5EBD205FA2955FA38361FF045EA28D5EA35F5EA4925FA29A5FA38661D2045EC3
:206A5300A28A5EA3625EA48D5EB50A5FA2955FA3835FB50A61FF045EB00E5EB02A5EB10DDB
:206A73005EB1295EA2865EB3125EA3665EA38A5EB3325EA48A5EB52A5EBD215FB00E5FB0BC
:206A93002A5FB10D5FB1295FA2925FA37F5FB52A61D3045EA28A5EA3865EA48D5EBD205F9F
:206AB300A2955FA38361FF045EA28D5EA3835EA4925FA29A5FA38661D3045EB00A5EB10973
:206AD3005EA28A5EA3865EA48D5FB00A5FB1095FA2955FA38361FF045EA2865EA38A5EA43F
:206AF3008A5FA2925FA37F61FF045EA28A5EA3865EA48D5EB50A5FA2955FA3835FB50A612A
:206B1300D2045EB02A5EB1295EA2835EA3835EA4865EB52A5EBD305EBD315FB02A5FB12947
:206B33005FA28D5FA37C5FB52A61FF045EA28A5EA3865EA48D5EBD215EBD205FA2955FA3E5
:206B53008361D3045EA2925EA38A5EA4955FA29D5FA38A61FF045EB00A5EB1095EA28A5E0D
:206B7300A3865EA48D5FB00A5FB1095FA2955FA38361D3045EA2835EA3835EA4865FA28DA8
:206B93005FA37C61FF045EA28A5EA3865EA48D5EB50A5FA2955FA3835FB50A61D3045EB0C4
:206BB3002E5EB12D5EA2925EA37F5EA4955EB52A5EBD305EBD315FB02E5FB12D5FA29D5F64
:206BD300A38A5FB52A61FE045EA28A5EA3865EA48D5EBD215EBD205FA2955FA38361FF043E
:206BF3005EA2835EA38D5EA4865FA28D5FA37C61D3045EA28A5EA3865EA48D5FA2955FA36D
:206C13008361FF045EA2925EA37F5EA4955FA29D5FA38A61D3045EA28A5EA3865EA48D5E71
:206C3300B50A5FA2955FA3835FB50A61FF045EB00E5EB02A5EB10D5EB1295EA27F5EA38D30
:206C53005EA4835EB52A5EBD305EBD385EBD3C5EBD3D5FB00E5FB02A5FB10D5FB1295FA265
:206C73008A5FA3775FB52A61D3045EA28A5EA3865EA48D5EBD355EBD315EBD305FA2955F0C
:206C9300A38361FE045EA2955EA37F5EA49A5FA2A25FA38D61FF045EB00A5EB1095EA28A57
:206CB3005EA3865EA48D5EBD205FB00A5FB1095FA2955FA38361D3045EA27F5EA38D5EA4DC
:206CD300835FA28A5FA37761FF045EA28A5EA3865EA48D5EB50A5FA2955FA3835FB50A615F
:206CF300D3045EB02A5EB1295EA2955EA37C5EA49A5EB52A5EBD305EBD315FB02A5FB12946
:206D13005FA2A25FA38D5FB52A61FF045EA28A5EA3865EA48D5EBD215EBD205FA2955FA3DD
:206D33008361D3045EA27F5EA3925EA4835FA28A5FA37761FE045EB00A5EB1095EA28A5E6F
:206D5300A3865EA48D5FB00A5FB1095FA2955FA38361D3045EA2955EA37C5EA49A5FA2A292
:206D73005FA38D61FF045EA28A5EA3865EA48D5EB50A5FA2955FA3835FB50A61FF045EB0A5
:206D93002E5EB12D5EA27C5EA3925EA47F5EA5985EB52D5EBD215FB02E5FB12D5FA2865F6F
:206DB300A3745FA5965FB52D61D3045EA28A5EA3865EA48D5EBD205FA2955FA38361FF043C
:206DD3005EA29A5EA37C5EA49D5FA2A55FA39261D3045EA28A5EA3865EA48D5FA2955FA340
:206DF3008361FE045EA27C5EA3925EA47F5FA2865FA37461D3045EA28A5EA3865EA48D5ED7
:206E1300B50D5FA2955FA3835FB50D61FF045EB00E5EB02A5EB10D5EB1295EA29A5EA37743
:206E33005EA49D5EA5225EB52A5EBD305EBD315FB00E5FB02A5FB10D5FB1295FA2A55FA353
:206E5300925FA51F5FB52A61D3045EA28A5EA3865EA48D5EBD215EBD205FA2955FA3836161
:206E7300FF045EA27C5EA3955EA47F5FA2865FA37461FF045EB00A5EB1095EA28A5EA386C7
:206E93005EA48D5FB00A5FB1095FA2955FA38361D3045EA29A5EA3775EA49D5FA2A55FA372
:206EB3009261FE045EA28A5EA3865EA48D5EB50A5FA2955FA3835FB50A61D3045EA0E65E5A
:206ED300B02D5EA16C5EB12D5EB2125EA28D5EA2695EB2325EA3955EB4125EA4925EA46D04
:206EF3005EB4325EA58A5EB52A5EBD305EBD385EBD3C5EBD3D5FA0E65FB02D5FA16C5FB187
:206F13002D5FB2125FA29A5FA2745FB2325FB30E5FA3865FA3625FB32E5FA5865FB52A6146
:206F3300FF045EA2665EA3865EA4695EBD355EBD315EBD305FA2705FA35F61D3045EA26290
:206F53005EA3775EA4665FA26D5FA35B61FF045EA2665EA3865EA4695EBD205FA2705FA309
:206F73005F61FF045EA2695EA3955EA46D5FA2745FA36261D3045EA2665EA3865EA4695E06
:206F9300B50A5FA2705FA35F5FB50A61FE045EB00D5EA0225EB02E5EB10D5EA1985EB12D66
:206FB3005EB2125EA2625EA2865EB2325EB3125EA38A5EA3665EB3325EB4125EA4665EA48C
:206FD3008A5EB4325EA5225EB52A5EBD305E71985E91065EBD315FB00D5FA0225FB02E5FA2
:206FF300B10D5FA1985FB12D5FB2125FA26D5FA2925FB2325FB30E5FA35B5FA37F5FB32E46
:207013005FA51F5FB52A61D3045EA28A5EA3625EA48D5EBD215EBD205FA2955FA38361FF56
:20703300045EA28D5EA35F5EA4925FA29A5FA38661D3045EA28A5EA3625EA48D5FA2955FEC
:20705300A38361FF045EA2865EA3665EA48A5FA2925FA37F61D3045EA28A5EA3625EA48D52
:207073005EB50A5FA2955FA3835FB50A61FF045EB00E5EA0E65EB02D5EB10D5EA16C5EB172
:207093002D5EB2125EA28D5EA2695EB2325EB3125EA35F5EA3835EB3325EB4125EA4925EF6
:2070B300A46D5EB4325EA5E65EB5295EBD305FB00E5FA0E65FB02D5FB10D5FA16C5FB12DF4
:2070D3005FB2125FA29A5FA2745FB2325FB30E5FA3865FA3625FB32E5FA5E35FB52961FE58
:2070F300045EA2665EA3865EA4695EBD205FA2705FA35F61D3045EA2625EA38A5EA4665F28
:20711300A26D5FA35B61FF045EA2665EA3865EA4695FA2705FA35F61D3045EA2695EA3833D
:207133005EA46D5FA2745FA36261FF045EA2665EA3865EA4695EB5095FA2705FA35F5FB536
:207153000961D3045EB00D5EB0295EB10D5EB1295EA2625EB3125EA38A5EA3665EB3325E1D
:20717300A4665EB5295E71F85E91CA5EBD215FB00D5FB0295FB10D5FB1295FA26D5FA35B85
:207193005FB52961FF045EA2665EA3625EA4695EBD205FA2705FA35F61D2045EA2695EA359
:2071B3005F5EA46D5FA2745FA36261FF045EB0095EB1095EA2665EA3625EA4695FB0095FD7
:2071D300B1095FA2705FA35F61FF045EA2625EA3665EA4665FA26D5FA35B61D3045EA26612
:2071F3005EA3625EA4695EB5095FA2705FA35F5FB50961FF045EB0295EB1295EA2695EA366
:207213005F5EA46D5EB5295EBD305EBD385EBD3C5EBD3D5FB0295FB1295FA2745FA3625F5B
:20723300B52961D3045EA2665EA3625EA4695EBD355EBD315EBD305FA2705FA35F61FF04D4
:207253005EA2625EA3665EA4665FA26D5FA35B61D2045EB0095EB1095EA2665EA3625EA4EE
:20727300695EBD205FB0095FB1095FA2705FA35F61FF045EA2695EA35F5EA46D5FA2745FE4
:20729300A36261FF045EA2665EA3625EA4695EB5095FA2705FA35F5FB50961D3045EB02DC0
:2072B3005EB12D5EB2125EA2625EA21F5EB2325EA3665EB4125EA4665EA4225EB4325EB52C
:2072D300295EBD305EBD315FB02D5FB12D5FB2125FA26D5FA2295FB2325FB30E5FA35B5F88
:2072F300A3195FB32E5FB52961FF045EA2225EA3625EA4255EBD215EBD205FA22C5FA31C70
:2073130061D3045EA2255EA35F5EA4295FA22F5FA31F61FF045EA2225EA3625EA4255FA210
:207333002C5FA31C61D2045EA21F5EA3665EA4225FA2295FA31961FF045EA2225EA3625E83
:20735300A4255EB5095FA22C5FA31C5FB50961D3045EB00D5EB0295EB10D5EB1295EA225CA
:207373005EB3125EA35F5EA31C5EB3325EA4295EB5295EBD215FB00D5FB0295FB10D5FB1F3
:20739300295FA22F5FA31F5FB52961FF045EA2225EA31F5EA4255EBD205FA22C5FA31C616F
:2073B300FF045EA21F5EA3225EA4225FA2295FA31961D3045EB0095EB1095EA2225EA31F63
:2073D3005EA4255FB0095FB1095FA22C5FA31C61FF045EA2255EA31C5EA4295FA22F5FA3F4
:2073F3001F61D2045EA2225EA31F5EA4255EB5095FA22C5FA31C5FB50961FF045EB0295E3E
:20741300B1295EA21F5EA3225EA4225EB5295EBD305EBD315FB0295FB1295FA2295FA31990
:207433005FB52961D3045EA2225EA31F5EA4255EBD215EBD205FA22C5FA31C61FF045EA235
:20745300255EA31C5EA4295FA22F5FA31F61FF045EB0095EB1095EA2225EA31F5EA4255F00
:20747300B0095FB1095FA22C5FA31C61D3045EA21F5EA3225EA4225FA2295FA31961FF0495
:207493005EA2225EA31F5EA4255EB5095FA22C5FA31C5FB50961D2045EB02D5EB12D5EB22E
:2074B300125EA2255EA2E95EB2315EA31C5EB4125EA4295EA4EC5EB4315EB5295EBD305ED6
:2074D300BD385EBD3C5EBD3D5FB02D5FB12D5FB2125FA22F5FA2F25FB2315FB30E5FA31FB3
:2074F3005FA3E35FB32D5FB52961FF045EA2E65EA31F5EA4E95EBD355EBD315EBD305FA2DB
:20751300EF5FA3E161D3045EA2E35EA3225EA4E65FA2EC5FA3DE61FF045EA2E65EA31F5ECB
:20753300A4E95EBD205FA2EF5FA3E161D3045EA2E95EA31C5EA4EC5FA2F25FA3E361FF0435
:207553005EA2E65EA31F5EA4E95EB5095FA2EF5FA3E15FB50961FF045EB00D5EB0295EB156
:207573000D5EB1295EA2E35EB3125EA3225EA3E65EB3315EA4E65EB5295EBD215FB00D5F86
:20759300B0295FB10D5FB1295FA2EC5FA3DE5FB52961D2045EA2E65EA3E35EA4E95EBD2078
:2075B3005FA2EF5FA3E161FF045EA2E95EA3E15EA4EC5FA2F25FA3E361D3045EB0095EB192
:2075D300095EA2E65EA3E35EA4E95FB0095FB1095FA2EF5FA3E161FF045EA2E35EA3E65E4A
:2075F300A4E65FA2EC5FA3DE61D3045EA2E65EA3E35EA4E95EB5095FA2EF5FA3E15FB50928
:2076130061FF045EB0295EB1295EA2E15EA3E15EA4E35EB5295EBD305EBD315FB0295FB1C1
:20763300295FA2E95FA3DB5FB52961D2045EA2E65EA3E35EA4E95EBD215EBD205FA2EF5F58
:20765300A3E161FF045EA2EC5EA3E65EA4EF5FA2F45FA3E661FF045EB0095EB1095EA2E615
:207673005EA3E35EA4E95FB0095FB1095FA2EF5FA3E161D3045EA2E15EA3E15EA4E35FA243
:20769300E95FA3DB61FF045EA2E65EA3E35EA4E95EB5095FA2EF5FA3E15FB50961D3045E56
:2076B300B02D5EB12D5EA2EC5EA3DE5EA4EF5EB5295EBD305EBD315FB02D5FB12D5FA2F4A1
:2076D3005FA3E65FB52961FF045EA2E65EA3E35EA4E95EBD215EBD205FA2EF5FA3E161D2DC
:2076F300045EA2E15EA3E95EA4E35FA2E95FA3DB61FF045EA2E65EA3E35EA4E95FA2EF5F94
:20771300A3E161FF045EA2EC5EA3DE5EA4EF5FA2F45FA3E661D3045EA2E65EA3E35EA4E9E8
:207733005EB5095FA2EF5FA3E15FB50961FF045EB00D5EB0295EB10D5EB1295EA2DE5EA341
:20775300E95EA4E15EB5295EBD305EBD385EBD3C5EBD3D5FB00D5FB0295FB10D5FB1295FB8
:20777300A2E65FA3D85FB52961D3045EA2E65EA3E35EA4E95EBD355EBD315EBD305FA2EF93
:207793005FA3E161FF045EA2EF5EA3DE5EA4F25FA2F85FA3E961D2045EB0095EB1095EA283
:2077B300E65EA3E35EA4E95EBD205FB0095FB1095FA2EF5FA3E161FF045EA2DE5EA3E95E38
:2077D300A4E15FA2E65FA3D861D3045EA2E65EA3E35EA4E95EB5095FA2EF5FA3E15FB50957
:2077F30061FF045EB0295EB1295EA2EF5EA3DB5EA4F25EB5295EBD305EBD315FB0295FB1C9
:20781300295FA2F85FA3E95FB52961FF045EA2E65EA3E35EA4E95EBD215EBD205FA2EF5F2C
:20783300A3E161D3045EA2DE5EA3EC5EA4E15FA2E65FA3D861FF045EB0095EB1095EA2E691
:207853005EA3E35EA4E95FB0095FB1095FA2EF5FA3E161D2045EA2EF5EA3DB5EA4F25FA24B
:20787300F85FA3E961FF045EA2E65EA3E35EA4E95EB5095FA2EF5FA3E15FB50961D3045E57
:20789300B02D5EB12D5EB2115EA2E95EA3EC5EB4115EA4EC5EA56C5EB52D5EBD215FB02D8D
:2078B3005FB12D5FB2115FA2F25FB30D5FA3E35FA5695FB52D61FF045EA2E65EA3E35EA481
:2078D300E95EBD205FA2EF5FA3E161D3045EA2E35EA3DB5EA4E65FA2EC5FA3DE61FF045E30
:2078F300A2E65EA3E35EA4E95FA2EF5FA3E161FF045EA2E95EA3EC5EA4EC5FA2F25FA3E34B
:2079130061D2045EA2E65EA3E35EA4E95EB50D5FA2EF5FA3E15FB50D61FF045EB00D5EB0C7
:20793300295EB10D5EB1295EA2E35EB2315EB3115EA3E65EA4E65EB4315EA5E65EB5295EDC
:20795300BD305EBD315FB00D5FB0295FB10D5FB1295FA2EC5FB2315FA3DE5FB32D5FA5E3FC
:207973005FB52961D3045EA2E65EA3E35EA4E95EBD215EBD205FA2EF5FA3E161FF045EA21C
:20799300E95EA3E15EA4EC5FA2F25FA3E361D3045EB0095EB1095EA2E65EA3E35EA4E95FC8
:2079B300B0095FB1095FA2EF5FA3E161FF045EA2E35EA3E65EA4E65FA2EC5FA3DE61FF04C8
:2079D3005EA2E65EA3E35EA4E95EB5095FA2EF5FA3E15FB50961D2045EA0B15EB02D5EA1B3
:2079F3008A5EB12A5EB2115EA2E95EA2255EB2325EA3E15EB3315EB4115EA4EC5EA4295E82
:207A1300B4325EA5225EB52A5EBD305EBD385EBD3C5EBD3D5FA0B15FB02D5FA18A5FB12A0E
:207A33005FB2115FA2F25FA22F5FB2325FB30D5FA3E35FA31F5FB32E5FA51F5FB52A61FF85
:207A5300045EA2225EA3E35EA4255EBD355EBD315EBD305FA22C5FA31C61D3045EA21F5EFB
:207A7300A3E65EA4225FA2295FA31961FF045EA2225EA3E35EA4255EBD205FA22C5FA31CEA
:207A930061D3045EA2255EA3E15EA4295FA22F5FA31F61FF045EA2225EA3E35EA4255EB574
:207AB3000A5FA22C5FA31C5FB50A61D3045EB00D5EA0E65EB02D5EB10A5EA16C5EB12D5EB0
:207AD300B2125EA21F5EA2625EB2325EB3115EA3E65EA3225EB3325EB4125EA4225EA466ED
:207AF3005EB4325EA5E65EB5295E71985E91065EBD215FB00D5FA0E65FB02D5FB10A5FA11B
:207B13006C5FB12D5FB2125FA2295FA26D5FB2325FB30E5FA3195FA35B5FB32E5FA5E35F8D
:207B3300B52961FE045EA2665EA31F5EA4695EBD205FA2705FA35F61FF045EA2695EA31C09
:207B53005EA46D5FA2745FA36261D3045EA2665EA31F5EA4695FA2705FA35F61FF045EA26B
:207B7300625EA3225EA4665FA26D5FA35B61D3045EA2665EA31F5EA4695EB5095FA2705F25
:207B9300A35F5FB50961FF045EB00D5EA0B15EB02D5EB10D5EA18A5EB12A5EB2125EA269E1
:207BB3005EA28D5EB2325EB3125EA31C5EA35F5EB3325EB4125EA46D5EA4925EB4325EA592
:207BD300B15EB5295EBD305FB00D5FA0B15FB02D5FB10D5FA18A5FB12A5FB2125FA2745F7A
:207BF300A29A5FB2325FB30E5FA3625FA3865FB32E5FA5AE5FB52961D3045EA28A5EA36293
:207C13005EA48D5EBD205FA2955FA38361FE045EA2865EA3665EA48A5FA2925FA37F61FF1C
:207C3300045EA28A5EA3625EA48D5FA2955FA38361D3045EA28D5EA35F5EA4925FA29A5FE3
:207C5300A38661FF045EA28A5EA3625EA48D5EB5095FA2955FA3835FB50961D3045EB00D61
:207C73005EB0295EB10A5EB1265EA2865EB3125EA3665EA38A5EB3325EA48A5EB5295E71F7
:207C9300F85E91CA5EBD215FB00D5FB0295FB10A5FB1265FA2925FA37F5FB52961FF045E2D
:207CB300A28A5EA3865EA48D5EBD205FA2955FA38361D3045EA28D5EA3835EA4925FA29AA1
:207CD3005FA38661FE045EB0095EB1065EA28A5EA3865EA48D5FB0095FB1065FA2955FA314
:207CF3008361D3045EA2865EA38A5EA48A5FA2925FA37F61FF045EA28A5EA3865EA48D5EA3
:207D1300B5095FA2955FA3835FB50961FF045EB0295EB1265EA28D5EA3835EA4925EB529A9
:207D33005EBD305EBD385EBD3C5EBD3D5FB0295FB1265FA29A5FA3865FB52961D3045EA2DD
:207D53008A5EA3865EA48D5EBD355EBD315EBD305FA2955FA38361FF045EA2865EA38A5E9B
:207D7300A48A5FA2925FA37F61D3045EB0095EB1065EA28A5EA3865EA48D5EBD205FB00957
:207D93005FB1065FA2955FA38361FE045EA28D5EA3835EA4925FA29A5FA38661D3045EA23C
:207DB3008A5EA3865EA48D5EB5095FA2955FA3835FB50961FF045EB02D5EB12A5EB2125E64
:207DD300A2865EA2695EB2355EA38A5EB4125EA48A5EA46C5EB4355EB5295EBD305EBD31F7
:207DF3005FB02D5FB12A5FB2125FA2925FA2705FB2355FB30E5FA37F5FA3655FB3315FB52E
:207E13002961D3045EA26C5EA3865EA46D5EBD215EBD205FA2725FA36861FF045EA26D5E09
:207E3300A3835EA4705FA2745FA36961FF045EA26C5EA3865EA46D5FA2725FA36861D304DC
:207E53005EA2695EA38A5EA46C5FA2705FA36561FE045EA26C5EA3865EA46D5EB5095FA2F3
:207E7300725FA3685FB50961D3045EB00D5EB0295EB10A5EB1265EA26D5EB3125EA3835EAC
:207E9300A3685EB3355EA4705EB5295EBD215FB00D5FB0295FB10A5FB1265FA2745FA36910
:207EB3005FB52961FF045EA26C5EA3695EA46D5EBD205FA2725FA36861D3045EA2695EA30F
:207ED3006C5EA46C5FA2705FA36561FF045EB0095EB1065EA26C5EA3695EA46D5FB0095F91
:207EF300B1065FA2725FA36861FF045EA26D5EA3685EA4705FA2745FA36961D3045EA26CAB
:207F13005EA3695EA46D5EB5095FA2725FA3685FB50961FE045EB0295EB1265EA2695EA326
:207F33006C5EA46C5EB5295EBD305EBD315FB0295FB1265FA2705FA3655FB52961D3045E68
:207F5300A26C5EA3695EA46D5EBD215EBD205FA2725FA36861FF045EA26D5EA3685EA47027
:207F73005FA2745FA36961D3045EB0095EB1065EA26C5EA3695EA46D5FB0095FB1065FA236
:207F9300725FA36861FF045EA2695EA36C5EA46C5FA2705FA36561D3045EA26C5EA3695E06
:207FB300A46D5EB5095FA2725FA3685FB50961FF045EB02D5EB12A5EB2155EA26D5EA2839A
:207FD3005EB2355EA3685EB4155EA4705EA4865EB4355EB5295EBD305EBD385EBD3C5EBD2C
:207FF3003D5FB02D5FB12A5FB2155FA2745FA28B5FB2355FB3115FA3695FA37F5FB3315F9D
:20801300B52961FE045EA2815EA3695EA4835EBD355EBD315EBD305FA2885FA37D61D30475
:208033005EA27F5EA36C5EA4815FA2865FA37B61FF045EA2815EA3695EA4835EBD205FA2AA
:20805300885FA37D61D3045EA2835EA3685EA4865FA28B5FA37F61FF045EA2815EA3695EA0
:20807300A4835EB5095FA2885FA37D5FB50961D3045EB00D5EB0295EB10A5EB1265EA27F2E
:208093005EB3155EA36C5EA3815EB3355EA4815EB5295EBD215FB00D5FB0295FB10A5FB1F9
:2080B300265FA2865FA37B5FB52961FF045EA2815EA37F5EA4835EBD205FA2885FA37D61B8
:2080D300D2045EA2835EA37D5EA4865FA28B5FA37F61FF045EB0095EB1065EA2815EA37F90
:2080F3005EA4835FB0095FB1065FA2885FA37D61FF045EA27F5EA3815EA4815FA2865FA341
:208113007B61D3045EA2815EA37F5EA4835EB5095FA2885FA37D5FB50961FF045EB0295ED9
:20813300B1265EB2155EA2835EA29A5EB2355EA37D5EB4155EA4865EA49D5EB4355EB5297F
:208153005EBD305EBD315FB0295FB1265FB2155FA28B5FA2A25FB2355FB3115FA37F5FA3C6
:20817300965FB3315FB52961D3045EA2985EA37F5EA49A5EBD215EBD205FA29F5FA39461DC
:20819300FF045EA2965EA3815EA4985FA29D5FA39161D2045EB0095EB1065EA2985EA37F6B
:2081B3005EA49A5FB0095FB1065FA29F5FA39461FF045EA29A5EA37D5EA49D5FA2A25FA3EC
:2081D3009661FF045EA2985EA37F5EA49A5EB5095FA29F5FA3945FB50961D3045EB02D5E9E
:2081F300B12A5EA2965EB3155EA3815EA3985EB3355EA4985EB5295EBD305EBD315FB02DCB
:208213005FB12A5FA29D5FA3915FB52961FF045EA2985EA3965EA49A5EBD215EBD205FA2FC
:208233009F5FA39461D3045EA29A5EA3945EA49D5FA2A25FA39661FF045EA2985EA3965EC4
:20825300A49A5FA29F5FA39461D2045EA2965EA3985EA4985FA29D5FA39161FF045EA2986A
:208273005EA3965EA49A5EB5095FA29F5FA3945FB50961D3045EB00D5EB0295EB10A5EB197
:20829300265EA29A5EA3945EA49D5EB5295EBD305EBD385EBD3C5EBD3D5FB00D5FB0295F9B
:2082B300B10A5FB1265FA2A25FA3965FB52961FF045EA2985EA3965EA49A5EBD355EBD3177
:2082D3005EBD305FA29F5FA39461FF045EA2965EA3985EA4985FA29D5FA39161D3045EB066
:2082F300095EB1065EA2985EA3965EA49A5EBD205FB0095FB1065FA29F5FA39461FF045E21
:20831300A29A5EA3945EA49D5FA2A25FA39661D2045EA2985EA3965EA49A5EB5095FA29FE1
:208333005FA3945FB50961FF045EB0295EB1265EB2155EA2965EA2695EB2355EA3985EB493
:20835300155EA4985EA46C5EB4355EB5295EBD305EBD315FB0295FB1265FB2155FA29D5F42
:20837300A2705FB2355FB3115FA3915FA3655FB3315FB52961D3045EA26C5EA3965EA46D4B
:208393005EBD215EBD205FA2725FA36861FF045EA26D5EA3945EA4705FA2745FA36961FF5E
:2083B300045EB0095EB1065EA26C5EA3965EA46D5FB0095FB1065FA2725FA36861D3045E67
:2083D300A2695EA3985EA46C5FA2705FA36561FF045EA26C5EA3965EA46D5EB5095FA2723B
:2083F3005FA3685FB50961D2045EB02D5EB12A5EA26D5EB3155EA3945EA3685EB3355EA45F
:20841300705EA58A5EB52A5EBD305EBD315FB02D5FB12A5FA2745FA3695FA5865FB52A61F9
:20843300FF045EA26C5EA3695EA46D5EBD215EBD205FA2725FA36861D3045EA2695EA36C7F
:208453005EA46C5FA2705FA36561FF045EA26C5EA3695EA46D5FA2725FA36861D3045EA205
:208473006D5EA3685EA4705FA2745FA36961FF045EA26C5EA3695EA46D5EB50A5FA2725F29
:20849300A3685FB50A61FF045EB00D5EB0295EB10A5EB1265EA2695EA36C5EA46C5EA5B1A4
:2084B3005EB5295EBD305EBD315FB00D5FB0295FB10A5FB1265FA2705FA3655FA5AE5FB594
:2084D3002961D2045EA26C5EA3695EA46D5EBD215EBD205FA2725FA36861FF045EA26D5E61
:2084F300A3685EA4705FA2745FA36961D3045EB0095EB1065EA26C5EA3695EA46D5FB0094B
:208513005FB1065FA2725FA36861FF045EA2695EA36C5EA46C5FA2705FA36561D3045EA29D
:208533006C5EA3695EA46D5EB5095FA2725FA3685FB50961FF045EA0985EB02D5EA1665ED5
:20855300B12A5EB2155EA26D5EA28D5EB2325EA3685EB4155EA4705EA4925EB4325EA56689
:208573005EB52A5EBD305EBD385EBD3C5EBD3D5FA0985FB02D5FA1665FB12A5FB2155FA2C4
:20859300745FA29A5FB2325FB3115FA3695FA3865FB32E5FA5625FB52A61D2045EA28A5E5D
:2085B300A3695EA48D5EBD355EBD315EBD305FA2955FA38361FF045EA2865EA36C5EA48A28
:2085D3005FA2925FA37F61FF045EA28A5EA3695EA48D5EBD205FA2955FA38361D3045EA2FF
:2085F3008D5EA3685EA4925FA29A5FA38661FF045EA28A5EA3695EA48D5EB50A5FA2955FC2
:20861300A3835FB50A61D3045EB00D5EA0B15EB02D5EB10A5EA18A5EB12A5EA2865EB3153F
:208633005EA36C5EA38A5EB3325EA48A5EA5B15EB5295EBD305E71985E91065EBD315FB06E
:208653000D5FA0B15FB02D5FB10A5FA18A5FB12A5FA2925FA37F5FA5AE5FB52961FF045E6B
:20867300A28A5EA3865EA48D5EBD215EBD205FA2955FA38361D2045EA28D5EA3835EA49237
:208693005FA29A5FA38661FF045EA28A5EA3865EA48D5FA2955FA38361FF045EA2865EA39A
:2086B3008A5EA48A5FA2925FA37F61D3045EA28A5EA3865EA48D5EB5095FA2955FA3835F0F
:2086D300B50961FF045EB00D5EA0CB5EB02D5EB10A5EA1665EB12A5EB2125EA28D5EA26977
:2086F3005EB2325EA3835EB4125EA4925EA46D5EB4325EA5665EB52A5EBD305EBD385EBDD7
:208713003C5EBD3D5FB00D5FA0CB5FB02D5FB10A5FA1665FB12A5FB2125FA29A5FA2745F44
:20873300B2325FB30E5FA3865FA3625FB32E5FA5625FB52A61D3045EA2665EA3865EA469C2
:208753005EBD2D5EBD3D5EBD355EBD3D5EBD395EBD3D5EBD3C5FA2705FA35F61FF045EA285
:20877300625EA38A5EA4665EBD345EBD305FA26D5FA35B61D2045EA2665EA3865EA4695F3E
:20879300A2705FA35F61FF045EA2695EA3835EA46D5EBD205FA2745FA36261D3045EA266E1
:2087B3005EA3865EA4695EB50A5FA2705FA35F5FB50A61FF045EB00D5EA0225EB0265EB1C5
:2087D3000A5EA1985EB1295EA2625EB3125EA38A5EA3665EB3325EA4665EA5225EB52A5ECB
:2087F300BD305E71F85E91CA5EBD315FB00D5FA0225FB0265FB10A5FA1985FB1295FA26DE2
:208813005FA35B5FA51F5FB52A61FF045EA2665EA3625EA4695EBD215EBD205FA2705FA305
:208833005F61D3045EA2695EA35F5EA46D5FA2745FA36261FF045EB0065EB1095EA2665E29
:20885300A3625EA4695FB0065FB1095FA2705FA35F61D2045EA2625EA3665EA4665FA26DBF
:208873005FA35B61FF045EA2665EA3625EA4695EB50A5FA2705FA35F5FB50A61D3045EA0AD
:20889300665EB02E5EB12D5EA25F5EA35F5EA4625EA5985EB52D5EBD305EBD385EBD3C5E96
:2088B30071985E91065EBD3D5FA0665FB02E5FB12D5FA2695FA3585FA5965FB52D61FF046D
:2088D3005EA2665EA3625EA4695EBD355EBD315EBD305FA2705FA35F61D3045EA26D5EA3F2
:2088F300665EA4705FA2775FA36661FF045EA2665EA3625EA4695EBD205FA2705FA35F61A7
:20891300FF045EA25F5EA35F5EA4625FA2695FA35861D2045EA2665EA3625EA4695EB50DCF
:208933005FA2705FA35F5FB50D61FF045EB00E5EA0225EB0265EB10D5EB1295EA26D5EA39B
:208953005B5EA4705EA5225EB52A5EBD305E71F85E91CA5EBD315FB00E5FA0225FB0265FEC
:20897300B10D5FB1295FA2775FA3665FA51F5FB52A61D3045EA2665EA3625EA4695EBD2104
:208993005EBD205FA2705FA35F61FF045EA25F5EA3695EA4625FA2695FA35861D3045EB01C
:2089B300065EB1095EA2665EA3625EA4695FB0065FB1095FA2705FA35F61FF045EA26D5E23
:2089D300A35B5EA4705FA2775FA36661FF045EA2665EA3625EA4695EB50A5FA2705FA35FAD
:2089F3005FB50A61D2045EA08A5EB02E5EA1B15EB12D5EA25B5EA3695EA45F5EA5B15EB572
:208A13002D5EBD305EBD385EBD3C5E71985E91065EBD3D5FA08A5FB02E5FA1B15FB12D5F5A
:208A3300A2665FA3545FA5AE5FB52D61FF045EA2665EA3625EA4695EBD355EBD315EBD3053
:208A53005FA2705FA35F61D3045EA2705EA35B5EA4745FA27C5FA36961FF045EA2665EA304
:208A7300625EA4695EBD205FA2705FA35F61D3045EA25B5EA3695EA45F5FA2665FA354618D
:208A9300FF045EA2665EA3625EA4695EB50D5FA2705FA35F5FB50D61D3045EB00E5EA02205
:208AB3005EB0265EB10D5EA1985EB1295EA2705EA3585EA4745EA5225EB52A5EBD305E71C9
:208AD300F85E91CA5EBD315FB00E5FA0225FB0265FB10D5FA1985FB1295FA27C5FA3695FDE
:208AF300A51F5FB52A61FE045EA2665EA3625EA4695EBD215EBD205FA2705FA35F61FF041D
:208B13005EA25B5EA36D5EA45F5FA2665FA35461D3045EB0065EB1095EA2665EA3625EA42C
:208B3300695FB0065FB1095FA2705FA35F61FF045EA2705EA3585EA4745FA27C5FA36961CD
:208B5300D3045EA2665EA3625EA4695EB50A5FA2705FA35F5FB50A61FF045EB02E5EA16CDF
:208B73005EB12D5EB2125EA2695EA2255EB2325EA36D5EB4125EA46D5EA4295EB4325EA541
:208B93006C5EB52D5EBD305EBD385EBD3C5E71985E91065EBD3D5FB02E5FA16C5FB12D5F28
:208BB300B2125FA2745FA22F5FB2325FB30E5FA3625FA31F5FB32E5FA5695FB52D61D3042B
:208BD3005EA2225EA3625EA4255EBD355EBD315EBD305FA22C5FA31C61FE045EA21F5EA321
:208BF300585EA4225FA2295FA31961FF045EA2225EA3625EA4255EBD205FA22C5FA31C61AA
:208C1300D3045EA2255EA36D5EA4295FA22F5FA31F61FF045EA2225EA3625EA4255EB50D2B
:208C33005FA22C5FA31C5FB50D61D3045EB00E5EB0265EB10D5EA1985EB1295EA21F5EB312
:208C5300125EA3665EA3225EB3325EA4225EA5225EB52A5EBD305E71F85E91CA5EBD315F26
:208C7300B00E5FB0265FB10D5FA1985FB1295FA2295FA3195FA51F5FB52A61FF045EA222D4
:208C93005EA31F5EA4255EBD215EBD205FA22C5FA31C61D3045EA2255EA31C5EA4295FA212
:208CB3002F5FA31F61FE045EB0065EB1095EA2225EA31F5EA4255FB0065FB1095FA22C5F9F
:208CD300A31C61D3045EA21F5EA3225EA4225FA2295FA31961FF045EA2225EA31F5EA42512
:208CF3005EB50A5FA22C5FA31C5FB50A61FF045EA0665EB02E5EB12D5EB2125EA2255EA254
:208D1300065EB2325EA31C5EB4125EA4295EA40A5EB4325EA5985EB52D5EBD305EBD385E65
:208D3300BD3C5E71985E91065EBD3D5FA0665FB02E5FB12D5FB2125FA22F5FA2105FB232ED
:208D53005FB30E5FA31F5FA3005FB32E5FA5965FB52D61D3045EA2035EA31F5EA4065EBD24
:208D7300355EBD315EBD305FA20C5FA3FE5FB32D61FF045EA2005EA3225EA4035FA20A5FD2
:208D9300A3FA61D3045EA2035EA31F5EA4065EBD205FA20C5FA3FE61FE045EA2065EA31CF2
:208DB3005EA40A5FA2105FA3005FB32E61D3045EA2035EA31F5EA4065EB50D5FA20C5FA3AF
:208DD300FE5FB32D5FB50D61FF045EB00E5EA0225EB0265EB10D5EB1295EA2005EB3125E79
:208DF300A3225EA3035EB3325EA4035EA5225EB52A5EBD305E71F85E91CA5EBD315FB00EB9
:208E13005FA0225FB0265FB10D5FB1295FA20A5FA3FA5FA51F5FB52A61D3045EA2035EA3EF
:208E3300005EA4065EBD215EBD205FA20C5FA3FE61FF045EA2065EA3FE5EB3315EA40A5F7D
:208E5300A2105FA3005FB32E61FF045EB0065EB1095EA2035EA3005EB3325EA4065FB00617
:208E73005FB1095FA20C5FA3FE5FB32D61D3045EA2005EA3035EA4035FA20A5FA3FA61FED3
:208E9300045EA2035EA3005EA4065EB50A5FA20C5FA3FE5FB50A61D3045EA0E65EB02D5EB2
:208EB300A18A5EB12A5EA2FE5EB2315EA3FE5EB3315EA4005EA58A5EB52A5EBD305EBD3851
:208ED3005EBD3C5E71985E91065EBD3D5FA0E65FB02D5FA18A5FB12A5FA2065FA3F85FA58A
:208EF300865FB52A61FF045EA2035EB2325EA3005EB3325EA4065EBD355EBD315EBD305F60
:208F1300A20C5FA3FE61D3045EA20A5EA3035EA40C5FA2125FA3035FB32E61FF045EA2037D
:208F33005EA3005EA4065EBD205FA20C5FA3FE5FB32D61FF045EA2FE5EB2315EA3FE5EB3DB
:208F5300315EA4005FA2065FA3F861D3045EA2035EB2325EA3005EB3325EA4065EB50A5F85
:208F7300A20C5FA3FE5FB50A61FE045EB00D5EA0225EB0265EB10A5EA1985EB1295EA20A4E
:208F93005EA3FA5EB3315EA40C5EA5225EB52A5EBD305E71F85E91CA5EBD315FB00D5FA0DF
:208FB300225FB0265FB10A5FA1985FB1295FA2125FA3035FB32E5FA51F5FB52A61D3045E0D
:208FD300A2035EA3005EB3325EA4065EBD215EBD205FA20C5FA3FE5FB32D61FF045EA2FE68
:208FF3005EB2315EA3065EA4005FA2065FA3F861D3045EB0065EB1095EA2035EB2325EA369
:20901300005EA4065FB0065FB1095FA20C5FA3FE61FF045EA20A5EA3FA5EB3315EA40C5FE2
:20903300A2125FA3035FB32E61D3045EA2035EA3005EB3325EA4065EB50A5FA20C5FA3FE73
:209053005FB32D5FB50A61FF045EB02E5EA16C5EB12D5EA2FA5EB2315EA3065EA4FE5EB405
:20907300315EA56C5EB52D5EBD305EBD385EBD3C5E71985E91065EBD3D5FB02E5FA16C5F4C
:20909300B12D5FA2035FA3F45FA5695FB52D61FE045EA2035EB2325EA3005EA4065EB43242
:2090B3005EBD355EBD315EBD305FA20C5FA3FE61D3045EA20C5EA3FA5EB3315EA4105FA215
:2090D300165FA3065FB32E61FF045EA2035EA3005EB3325EA4065EBD205FA20C5FA3FE5FC5
:2090F300B32D61D3045EA2FA5EB2315EA3065EA4FE5EB4315FA2035FA3F461FF045EA2035F
:209113005EB2325EA3005EA4065EB4325EB50D5FA20C5FA3FE5FB50D61D3045EB00E5EB0FD
:20913300265EB10D5EA1985EB1295EA20C5EA3F85EB3315EA4105EA5225EB52A5EBD305EA7
:2091530071F85E91CA5EBD315FB00E5FB0265FB10D5FA1985FB1295FA2165FA3065FB32EEF
:209173005FA51F5FB52A61FF045EA2035EA3005EB3325EA4065EBD215EBD205FA20C5FA342
:20919300FE5FB32D61D2045EA2FA5EB2315EA30A5EA4FE5EB4315FA2035FA3F461FF045E03
:2091B300B0065EB1095EA2035EB2325EA3005EA4065EB4325FB0065FB1095FA20C5FA3FE01
:2091D30061FF045EA20C5EA3F85EB3315EA4105FA2165FA3065FB32E61D3045EA2035EA324
:2091F300005EB3325EA4065EB50A5FA20C5FA3FE5FB32D5FB50A61FF045EA0CB5EB02D5EC4
:20921300A1665EB12A5EA2F85EB2315EA30A5EA4FA5EB4315EA5665EB52A5EC6185E3032D6
:209233005E50445E70F85EC61E5E33115E937F5EB60D5EBD305E34325E54495E74F85E9428
:20925300FF5EF4005EBD385EBD3C5FA0CB5FB02D5FA1665FB12A5FA2005FA3F25FA5625FA0
:20927300B52A61D3045EA2035EB2325EA3005EA4065EB4325FA20C5FA3FE61FF045EA210B1
:209293005EA3F85EB3315EA4125FA2195FA30A5FB32E61D2045EA2035EA3005EB3325EA486
:2092B300065EBD2C5EC63E5EA6035EB60A5EBD3C5EBD345EBD3C5EBD385EBD3C5FA20C5FB4
:2092D300A3FE5FB32D61FF045EA2F85EB2315EA30A5EA4FA5EB4315FA2005FA3F261FF045B
:2092F3005EA2035EB2325EA3005EA4065EB4325EB50A5FA20C5FA3FE5FB50A61D3045EB03B
:209313000D5EA0225EB0265EB10A5EA1985EB1295EA2105EA3F45EB3315EA4125EA5225E13
:20933300B52A5EBD2C5EC62E5EA6815EB6095EBD3C5EBD345EBD3C5EBD385EBD3C5FB00D3D
:209353005FA0225FB0265FB10A5FA1985FB1295FA2195FA30A5FB32E5FA51F5FB52A61FF92
:20937300045EA2035EA3005EB3325EA4065FA20C5FA3FE5FB32D61D3045EA2F85EB2315E6C
:20939300A30C5EA4FA5EB4315FA2005FA3F261FF045EB0065EB1095EA2035EB2325EA30001
:2093B3005EA4065EB4325EBD2C5EBD245EBD205FB0065FB1095FA20C5FA3FE61D2045EA21B
:2093D300105EA3F45EB3315EA4125FA2195FA30A5FB32E61FF045EA2035EA3005EB3325EB0
:2093F300A4065EB50A5FA20C5FA3FE5FB32D5FB50A61D3045EB02E5EB12D5EB2125EA20651
:209413005EA2255EB2325EA30C5EB4125E29F15E49C05E69005E89EE5EC43C5EE9025E2CF5
:20943300F15E8CD95EEC005E4C095EA49A5EB4315EB52A5EC63E5E30005E50075E70D85EA3
:20945300C6385E33005E93F05EA6575EBD305E341E5E54055E74F55E94D75EF4025EC81161
:209473005EBD325FB02E5FB12D5FB2125FA2105FA22F5FB2325FB30D5FA3005FB30E5FA328
:209493001F5FB32E5FC4185F29B15F49AF5F69005F89F15FC4165F2CA25F6C705F8C155FEE
:2094B300EC015FA45D5F4C0D5FA49F5FB42D5FB52A61FF045EA2225EA3005EA4985EBD2216
:2094D3005EBD205FA22C5FA31C5FA49D61FF045EA21F5EA3F45EB3315EA4965FA2295FA3D5
:2094F300195FA49A61D3045EA2225EA3005EB3325EA4985FA22C5FA31C5FA49D61FF045EBE
:20951300A2255EA30C5EA49A5FA22F5FA31F5FA49F61D2045EA2225EA3005EA4985EB50AC4
:209533005FA22C5FA31C5FA49D5FB50A61FF045EB00E5EB02A5EB10D5EB1295EA21F5EB3D3
:20955300125EA3035EA3225EB3325EA4965EB52A5EBD215FB00E5FB02A5FB10D5FB1295F60
:20957300A2295FA3195FA49A5FB52A61D3045EA2225EA31F5EA4985EBD205FA22C5FA31C7D
:209593005FA49D61FF045EA2255EA31C5EA49A5FA22F5FA31F5FA49F61FF045EB00A5EB158
:2095B300095EA2225EA31F5EA4985FB00A5FB1095FA22C5FA31C5FA49D61D3045EA21F5EE1
:2095D300A3225EA4965FA2295FA3195FA49A61FF045EA2225EA31F5EA4985EB50A5FA22CAF
:2095F3005FA31C5FA49D5FB50A61D2045EB02A5EB1295EA2255EA31C5EA49A5EB52A5EBD9F
:20961300305EBD385EBD3C5EBD3D5FB02A5FB1295FA22F5FA31F5FA49F5FB52A61FF045EA0
:20963300A2225EA31F5EA4985EBD355EBD315EBD305FA22C5FA31C5FA49D61D3045EA21F70
:209653005EA3225EA4965FA2295FA3195FA49A61FF045EB00A5EB1095EA2225EA31F5EA482
:20967300985EBD205FB00A5FB1095FA22C5FA31C5FA49D61D3045EA2255EA31C5EA49A5F72
:20969300A22F5FA31F5FA49F61FF045EA2225EA31F5EA4985EB50A5FA22C5FA31C5FA49DDB
:2096B3005FB50A61FF045EB02E5EB12D5EB2125EA21F5EA2625EB2325EA3225EB4115EA470
:2096D300965EA4E35EB4315EB52A5EBD305EBD315FB02E5FB12D5FB2125FA2295FA26D5F51
:2096F300B2325FB30E5FA3195FA35B5FB32E5FB40D5FA49A5FA4E95FB42D5FB52A61D2043D
:209713005EA2665EA31F5EA4E65EBD215EBD205FA2705FA35F5FA4EC61FF045EA2695EA3C2
:209733001C5EA4E95FA2745FA3625FA4EF61D3045EA2665EA31F5EA4E65FA2705FA35F5F6D
:20975300A4EC61FF045EA2625EA3225EA4E35FA26D5FA35B5FA4E961D3045EA2665EA31F23
:209773005EA4E65EB50A5FA2705FA35F5FA4EC5FB50A61FF045EB00E5EB02A5EB10D5EB10F
:20979300295EA2695EB3125EA31C5EA35F5EB3325EA4E95EB52A5EBD215FB00E5FB02A5F28
:2097B300B10D5FB1295FA2745FA3625FA4EF5FB52A61D2045EA2665EA3625EA4E65EBD2073
:2097D3005FA2705FA35F5FA4EC61FF045EA2625EA3665EA4E35FA26D5FA35B5FA4E961FF8C
:2097F300045EB00A5EB1095EA2665EA3625EA4E65FB00A5FB1095FA2705FA35F5FA4EC611D
:20981300D3045EA2695EA35F5EA4E95FA2745FA3625FA4EF61FF045EA2665EA3625EA4E6CA
:209833005EB50A5FA2705FA35F5FA4EC5FB50A61D3045EB02A5EB1295EA2625EA3665EA4A6
:20985300E35EB52A5EBD305EBD315FB02A5FB1295FA26D5FA35B5FA4E95FB52A61FF045E15
:20987300A2665EA3625EA4E65EBD215EBD205FA2705FA35F5FA4EC61D2045EA2695EA35F4A
:209893005EA4E95FA2745FA3625FA4EF61FF045EB00A5EB1095EA2665EA3625EA4E65FB0AB
:2098B3000A5FB1095FA2705FA35F5FA4EC61FF045EA2625EA3665EA4E35FA26D5FA35B5F75
:2098D300A4E961D3045EA2665EA3625EA4E65EB50A5FA2705FA35F5FA4EC5FB50A61FF049F
:2098F3005EB02E5EB12D5EB2125EA2695EA28D5EB2325EA35F5EB4115EA4E95EA4255EB4DC
:20991300325EB52A5EBD305EBD385EBD3C5EBD3D5FB02E5FB12D5FB2125FA2745FA29A5F6C
:20993300B2325FB30E5FA3625FA3865FB32E5FB40D5FA4EF5FA42C5FB42E5FB52A61D304EC
:209953005EA28A5EA3625EA4225EBD355EBD315EBD305FA2955FA3835FA42961FF045EA251
:20997300865EA3665EA41F5FA2925FA37F5FA42561D2045EA28A5EA3625EA4225EBD205FA8
:20999300A2955FA3835FA42961FF045EA28D5EA35F5EA4255FA29A5FA3865FA42C61D304CA
:2099B3005EA28A5EA3625EA4225EB50A5FA2955FA3835FA4295FB50A61FF045EB00E5EB073
:2099D3002A5EB10D5EB1295EA2865EB3125EA3665EA38A5EB3325EA41F5EB52A5EBD215F1F
:2099F300B00E5FB02A5FB10D5FB1295FA2925FA37F5FA4255FB52A61FF045EA28A5EA38618
:209A13005EA4225EBD205FA2955FA3835FA42961D3045EA28D5EA3835EA4255FA29A5FA380
:209A3300865FA42C61FF045EB00A5EB1095EA28A5EA3865EA4225FB00A5FB1095FA2955F6E
:209A5300A3835FA42961D2045EA2865EA38A5EA41F5FA2925FA37F5FA42561FF045EA28A0E
:209A73005EA3865EA4225EB50A5FA2955FA3835FA4295FB50A61D3045EB02A5EB1295EA2FE
:209A9300835EA3835EA41C5EB52A5EBD305EBD315FB02A5FB1295FA28D5FA37C5FA4225FB8
:209AB300B52A61FF045EA28A5EA3865EA4225EBD215EBD205FA2955FA3835FA42961D30425
:209AD3005EA2925EA38A5EA4295FA29D5FA38A5FA42F61FF045EB00A5EB1095EA28A5EA3B0
:209AF300865EA4225FB00A5FB1095FA2955FA3835FA42961FF045EA2835EA3835EA41C5F48
:209B1300A28D5FA37C5FA42261D2045EA28A5EA3865EA4225EB50A5FA2955FA3835FA42990
:209B33005FB50A61FF045EB02E5EB12D5EA2925EA37F5EA4295EB52A5EBD305EBD315FB0F8
:209B53002E5FB12D5FA29D5FA38A5FA42F5FB52A61D3045EA28A5EA3865EA4225EBD215EE6
:209B7300BD205FA2955FA3835FA42961FF045EA2835EA38D5EA41C5FA28D5FA37C5FA422EA
:209B930061D3045EA28A5EA3865EA4225FA2955FA3835FA42961FF045EA2925EA37F5EA486
:209BB300295FA29D5FA38A5FA42F61FF045EA28A5EA3865EA4225EB50A5FA2955FA3835FDD
:209BD300A4295FB50A61D2045EB00E5EB02A5EB10D5EB1295EA27F5EA38D5EA4195EB52A43
:209BF3005EBD305EBD385EBD3C5EBD3D5FB00E5FB02A5FB10D5FB1295FA28A5FA3775FA452
:209C13001F5FB52A61FF045EA28A5EA3865EA4225EBD355EBD315EBD305FA2955FA3835FDA
:209C3300A42961D3045EA2955EA37F5EA42C5FA2A25FA38D5FA43261FF045EB00A5EB109CE
:209C53005EA28A5EA3865EA4225EBD205FB00A5FB1095FA2955FA3835FA42961D3045EA2D0
:209C73007F5EA38D5EA4195FA28A5FA3775FA41F61FF045EA28A5EA3865EA4225EB50A5F6E
:209C9300A2955FA3835FA4295FB50A61D3045EB02A5EB1295EA2955EA37C5EA42C5EB52A86
:209CB3005EBD305EBD315FB02A5FB1295FA2A25FA38D5FA4325FB52A61FE045EA28A5EA3F5
:209CD300865EA4225EBD215EBD205FA2955FA3835FA42961FF045EA27F5EA3925EA4195F19
:209CF300A28A5FA3775FA41F61D3045EB00A5EB1095EA28A5EA3865EA4225FB00A5FB109BB
:209D13005FA2955FA3835FA42961FF045EA2955EA37C5EA42C5FA2A25FA38D5FA43261D3AA
:209D3300045EA28A5EA3865EA4225EB50A5FA2955FA3835FA4295FB50A61FF045EB02E5E57
:209D5300B12D5EA27C5EA3925EA4165EA5985EB52D5EBD215FB02E5FB12D5FA2865FA3745D
:209D73005FA41C5FA5965FB52D61D3045EA28A5EA3865EA4225EBD205FA2955FA3835FA410
:209D93002961FE045EA29A5EA37C5EA42F5FA2A55FA3925FA43661FF045EA28A5EA3865E96
:209DB300A4225FA2955FA3835FA42961D3045EA27C5EA3925EA4165FA2865FA3745FA41C08
:209DD30061FF045EA28A5EA3865EA4225EB50D5FA2955FA3835FA4295FB50D61D3045EB009
:209DF3000E5EB02A5EB10D5EB1295EA29A5EA3775EA42F5EA5225EB52A5EBD305EBD315F1B
:209E1300B00E5FB02A5FB10D5FB1295FA2A55FA3925FA4365FA51F5FB52A61FF045EA28A20
:209E33005EA3865EA4225EBD215EBD205FA2955FA3835FA42961D3045EA27C5EA3955EA45A
:209E5300165FA2865FA3745FA41C61FE045EB00A5EB1095EA28A5EA3865EA4225FB00A5F7D
:209E7300B1095FA2955FA3835FA42961D3045EA29A5EA3775EA42F5FA2A55FA3925FA436E0
:209E930061FF045EA28A5EA3865EA4225EB50A5FA2955FA3835FA4295FB50A61FF045EA032
:209EB300E65EB02D5EA16C5EB12D5EB2125EA28D5EA2695EB2325EA3955EB4125EA4255E2E
:209ED300A4E95EB4315EA58A5EB52A5EBD305EBD385EBD3C5EBD3D5FA0E65FB02D5FA16CFB
:209EF3005FB12D5FB2125FA29A5FA2745FB2325FB30E5FA3865FA3625FB32E5FB40E5FA42C
:209F13002C5FA4EF5FB42D5FA5865FB52A61D3045EA2665EA3865EA4E65EBD355EBD315E01
:209F3300BD305FA2705FA35F5FA4EC61FF045EA2625EA3775EA4E35FA26D5FA35B5FA4E986
:209F530061D3045EA2665EA3865EA4E65EBD205FA2705FA35F5FA4EC61FE045EA2695EA318
:209F7300955EA4E95FA2745FA3625FA4EF61D3045EA2665EA3865EA4E65EB50A5FA2705F89
:209F9300A35F5FA4EC5FB50A61FF045EB00D5EA0225EB02E5EB10D5EA1985EB12D5EB212B3
:209FB3005EA2625EA2865EB2325EB3125EA38A5EA3665EB3325EB4115EA4E35EA41F5EB4D1
:209FD300325EA5225EB52A5EBD305E71985E91065EBD315FB00D5FA0225FB02E5FB10D5FF1
:209FF300A1985FB12D5FB2125FA26D5FA2925FB2325FB30E5FA35B5FA37F5FB32E5FB40D13
:20A013005FA4E95FA4255FB42E5FA51F5FB52A61D3045EA28A5EA3625EA4225EBD215EBDD7
:20A03300205FA2955FA3835FA42961FF045EA28D5EA35F5EA4255FA29A5FA3865FA42C617B
:20A05300FF045EA28A5EA3625EA4225FA2955FA3835FA42961D3045EA2865EA3665EA41F4C
:20A073005FA2925FA37F5FA42561FE045EA28A5EA3625EA4225EB50A5FA2955FA3835FA4E2
:20A09300295FB50A61D3045EB00E5EA0E65EB02D5EB10D5EA16C5EB12D5EB2125EA28D5E23
:20A0B300A2695EB2325EB3125EA35F5EA3835EB3325EB4125EA4255EA4E95EB4315EA5E694
:20A0D3005EB5295EBD305FB00E5FA0E65FB02D5FB10D5FA16C5FB12D5FB2125FA29A5FA223
:20A0F300745FB2325FB30E5FA3865FA3625FB32E5FB40E5FA42C5FA4EF5FB42D5FA5E35F82
:20A11300B52961FF045EA2665EA3865EA4E65EBD205FA2705FA35F5FA4EC61D3045EA2627F
:20A133005EA38A5EA4E35FA26D5FA35B5FA4E961FF045EA2665EA3865EA4E65FA2705FA339
:20A153005F5FA4EC61FF045EA2695EA3835EA4E95FA2745FA3625FA4EF61D3045EA2665E9B
:20A17300A3865EA4E65EB5095FA2705FA35F5FA4EC5FB50961FE045EB00D5EB0295EB10DF0
:20A193005EB1295EA2625EB3125EA38A5EA3665EB3325EA4E35EB5295E71F85E91CA5EBDFE
:20A1B300215FB00D5FB0295FB10D5FB1295FA26D5FA35B5FA4E95FB52961D3045EA2665ED1
:20A1D300A3625EA4E65EBD205FA2705FA35F5FA4EC61FF045EA2695EA35F5EA4E95FA274F6
:20A1F3005FA3625FA4EF61D3045EB0095EB1095EA2665EA3625EA4E65FB0095FB1095FA2AC
:20A21300705FA35F5FA4EC61FF045EA2625EA3665EA4E35FA26D5FA35B5FA4E961D3045E0C
:20A23300A2665EA3625EA4E65EB5095FA2705FA35F5FA4EC5FB50961FF045EB0295EB129EB
:20A253005EA2695EA35F5EA4E95EB5295EBD305EBD385EBD3C5EBD3D5FB0295FB1295FA23C
:20A27300745FA3625FA4EF5FB52961FE045EA2665EA3625EA4E65EBD355EBD315EBD305F6A
:20A29300A2705FA35F5FA4EC61D3045EA2625EA3665EA4E35FA26D5FA35B5FA4E961FF0448
:20A2B3005EB0095EB1095EA2665EA3625EA4E65EBD205FB0095FB1095FA2705FA35F5FA46A
:20A2D300EC61D3045EA2695EA35F5EA4E95FA2745FA3625FA4EF61FF045EA2665EA3625E3D
:20A2F300A4E65EB5095FA2705FA35F5FA4EC5FB50961D3045EB02D5EB12D5EB2125EA26294
:20A313005EA2865EB2325EA3665EB4115EA4E35EA41F5EB4325EB5295EBD305EBD315FB0AC
:20A333002D5FB12D5FB2125FA26D5FA2925FB2325FB30E5FA35B5FA37F5FB32E5FB40D5F7C
:20A35300A4E95FA4255FB42E5FB52961FF045EA28A5EA3625EA4225EBD215EBD205FA29535
:20A373005FA3835FA42961D2045EA28D5EA35F5EA4255FA29A5FA3865FA42C61FF045EA218
:20A393008A5EA3625EA4225FA2955FA3835FA42961FF045EA2865EA3665EA41F5FA2925FEE
:20A3B300A37F5FA42561D3045EA28A5EA3625EA4225EB5095FA2955FA3835FA4295FB50977
:20A3D30061FF045EB00D5EB0295EB10D5EB1295EA28D5EB3125EA35F5EA3835EB3325EA487
:20A3F300255EB5295EBD215FB00D5FB0295FB10D5FB1295FA29A5FA3865FA42C5FB5296113
:20A41300D3045EA28A5EA3865EA4225EBD205FA2955FA3835FA42961FF045EA2865EA38A26
:20A433005EA41F5FA2925FA37F5FA42561D2045EB0095EB1095EA28A5EA3865EA4225FB002
:20A45300095FB1095FA2955FA3835FA42961FF045EA28D5EA3835EA4255FA29A5FA3865F62
:20A47300A42C61FF045EA28A5EA3865EA4225EB5095FA2955FA3835FA4295FB50961D304A8
:20A493005EB0295EB1295EA2865EA38A5EA41F5EB5295EBD305EBD315FB0295FB1295FA2C3
:20A4B300925FA37F5FA4255FB52961FF045EA28A5EA3865EA4225EBD215EBD205FA2955F0C
:20A4D300A3835FA42961D3045EA28D5EA3835EA4255FA29A5FA3865FA42C61FF045EB009DA
:20A4F3005EB1095EA28A5EA3865EA4225FB0095FB1095FA2955FA3835FA42961D2045EA24D
:20A51300865EA38A5EA41F5FA2925FA37F5FA42561FF045EA28A5EA3865EA4225EB5095FA6
:20A53300A2955FA3835FA4295FB50961D3045EB02D5EB12D5EB2125EA28D5EA2595EB23507
:20A553005EA3835EB4125EA4255EA4465EB4325EB5295EBD305EBD385EBD3C5EBD3D5FB0F5
:20A573002D5FB12D5FB2125FA29A5FA25F5FB2355FB30E5FA3865FA3AD5FB32E5FB40E5FE3
:20A59300A42C5FA44D5FB42E5FB52961FF045EA2575EA3865EA4435EBD355EBD315EBD309C
:20A5B3005FA25D5FA3AA5FA44A61FF045EA2AD5EB2325EA38A5EA43F5FA25B5FA3A55FA40C
:20A5D3004661D3045EA2575EB2355EA3865EA4435EBD205FA25D5FA3AA5FA44A61FF045E2E
:20A5F300A2595EA3835EA4465FA25F5FA3AD5FA44D61D2045EA2575EA3865EA4435EB509AC
:20A613005FA25D5FA3AA5FA44A5FB50961FF045EB00D5EB0295EB10D5EB1295EA2AD5EB2EC
:20A63300325EB3125EA38A5EA3575EB3355EA43F5EB5295EBD215FB00D5FB0295FB10D5F00
:20A65300B1295FA25B5FA3A55FA4465FB52961D3045EA2575EB2355EA3AD5EB3325EA4437A
:20A673005EBD205FA25D5FA3AA5FA44A61FF045EA2595EA3AA5EA4465FA25F5FA3AD5FA473
:20A693004D61FF045EB0095EB1095EA2575EA3AD5EA4435FB0095FB1095FA25D5FA3AA5FE3
:20A6B300A44A61D3045EA2AD5EB2325EA3575EB3355EA43F5FA25B5FA3A55FA44661FF04E3
:20A6D3005EA2575EB2355EA3AD5EB3325EA4435EB5095FA25D5FA3AA5FA44A5FB50961D2D2
:20A6F300045EB0295EB1295EB2155EA2595EA26D5EB2355EA3AA5EB4125EA4465EA4695EC4
:20A71300B4325EB5295EBD305EBD315FB0295FB1295FB2155FA25F5FA2745FB2355FB30E9B
:20A733005FA3AD5FA3695FB3315FB40E5FA44D5FA4705FB42E5FB52961FF045EA26C5EA376
:20A75300AD5EA4665EBD215EBD205FA2725FA3685FA46D61D3045EA2695EA3575EB3355E70
:20A77300A4625FA2705FA3655FA46961FF045EB0095EB1095EA26C5EA3AD5EB3325EA46624
:20A793005FB0095FB1095FA2725FA3685FA46D61D3045EA26D5EA3AA5EA4695FA2745FA3F6
:20A7B300695FA47061FF045EA26C5EA3AD5EA4665EB5095FA2725FA3685FA46D5FB50961DD
:20A7D300FF045EB02D5EB12D5EA2695EB3125EA3575EB3155EA36C5EB3355EA4625EB5298F
:20A7F3005EBD305EBD315FB02D5FB12D5FA2705FA3655FA4695FB52961D2045EA26C5EA311
:20A81300695EA4665EBD215EBD205FA2725FA3685FA46D61FF045EA26D5EA3685EA4695F8C
:20A83300A2745FA3695FA47061D3045EA26C5EA3695EA4665FA2725FA3685FA46D61FF04EA
:20A853005EA2695EA36C5EA4625FA2705FA3655FA46961D3045EA26C5EA3695EA4665EB5DE
:20A87300095FA2725FA3685FA46D5FB50961FF045EB00D5EB0295EB10D5EB1295EA2685E82
:20A89300A3685EA45F5EB5295EBD305EBD385EBD3C5EBD3D5FB00D5FB0295FB10D5FB12906
:20A8B3005FA26D5FA3645FA4665FB52961D2045EA26C5EA3695EA4665EBD355EBD315EBDDF
:20A8D300305FA2725FA3685FA46D61FF045EA2705EA36C5EA46D5FA2765FA36C5FA474617B
:20A8F300FF045EB0095EB1095EA26C5EA3695EA4665EBD205FB0095FB1095FA2725FA3688C
:20A913005FA46D61D3045EA2685EA3685EA45F5FA26D5FA3645FA46661FF045EA26C5EA33C
:20A93300695EA4665EB5095FA2725FA3685FA46D5FB50961D3045EB0295EB1295EA2705E38
:20A95300A3655EA46D5EB5295EBD305EBD315FB0295FB1295FA2765FA36C5FA4745FB52990
:20A9730061FF045EA26C5EA3695EA4665EBD215EBD205FA2725FA3685FA46D61D2045EA227
:20A99300685EA36D5EA45F5FA26D5FA3645FA46661FF045EB0095EB1095EA26C5EA3695E69
:20A9B300A4665FB0095FB1095FA2725FA3685FA46D61FF045EA2705EA3655EA46D5FA276DC
:20A9D3005FA36C5FA47461D3045EA26C5EA3695EA4665EB5095FA2725FA3685FA46D5FB58C
:20A9F3000961FF045EB02D5EB12D5EA2655EA36D5EA45B5EA56C5EB52D5EBD215FB02D5FAA
:20AA1300B12D5FA26C5FA3615FA4625FA5695FB52D61D3045EA26C5EA3695EA4665EBD20B1
:20AA33005FA2725FA3685FA46D61FF045EA2725EA3655EA4705FA2795FA36D5FA47761D272
:20AA5300045EA26C5EA3695EA4665FA2725FA3685FA46D61FF045EA2655EA36D5EA45B5F61
:20AA7300A26C5FA3615FA46261D3045EA26C5EA3695EA4665EB50D5FA2725FA3685FA46D0A
:20AA93005FB50D61FF045EB00D5EB0295EB10D5EB1295EA2725EA3645EA4705EA5E65EB533
:20AAB300295EBD305E71985E91065EBD315FB00D5FB0295FB10D5FB1295FA2795FA36D5F75
:20AAD300A4775FA5E35FB52961FF045EA26C5EA3695EA4665EBD215EBD205FA2725FA3682E
:20AAF3005FA46D61D3045EA2655EA3705EA45B5FA26C5FA3615FA46261FF045EB0095EB1A9
:20AB1300095EA26C5EA3695EA4665FB0095FB1095FA2725FA3685FA46D61D2045EA2725E56
:20AB3300A3645EA4705FA2795FA36D5FA47761FF045EA26C5EA3695EA4665EB5095FA272F5
:20AB53005FA3685FA46D5FB50961D3045EA0B15EB02D5EA18A5EB12A5EB2155EA26D5EA275
:20AB73008D5EB2325EA3705EB4125EA4695EA4255EB4325EA5225EB52A5EBD305EBD385E2A
:20AB9300BD3C5E71F85E91CA5EBD3D5FA0B15FB02D5FA18A5FB12A5FB2155FA2745FA29AEB
:20ABB3005FB2325FB3115FA3695FA3865FB32E5FB40E5FA4705FA42C5FB42E5FA51F5FB5AE
:20ABD3002A61FF045EA28A5EA3695EA4225EBD355EBD315EBD305FA2955FA3835FA429612D
:20ABF300D3045EA2865EA3645EA41F5FA2925FA37F5FA42561FF045EA28A5EA3695EA422A7
:20AC13005EBD205FA2955FA3835FA42961FF045EA28D5EA3705EA4255FA29A5FA3865FA4F0
:20AC33002C61D2045EA28A5EA3695EA4225EB50A5FA2955FA3835FA4295FB50A61FF045E42
:20AC5300B00D5EA0E65EB02D5EB10A5EA16C5EB12D5EB2125EA2865EA2695EB2355EB315C9
:20AC73005EA36C5EA38A5EB3325EB4125EA41F5EA4625EB4325EA5E65EB5295E71985E911E
:20AC9300065EBD215FB00D5FA0E65FB02D5FB10A5FA16C5FB12D5FB2125FA2925FA2705FD9
:20ACB300B2355FB30E5FA37F5FA3655FB3315FB40E5FA4255FA4695FB42E5FA5E35FB52935
:20ACD30061D3045EA26C5EA3865EA4665EBD205FA2725FA3685FA46D61FF045EA26D5EA374
:20ACF300835EA4695FA2745FA3695FA47061D3045EA26C5EA3865EA4665FA2725FA3685F31
:20AD1300A46D61FF045EA2695EA38A5EA4625FA2705FA3655FA46961FF045EA26C5EA386B8
:20AD33005EA4665EB5095FA2725FA3685FA46D5FB50961D2045EB00D5EA0B15EB02D5EB1C7
:20AD53000D5EA18A5EB12A5EB2155EA26D5EA28D5EB2325EB3125EA3835EA3685EB3355EFC
:20AD7300B4125EA4695EA4255EB4325EA5B15EB5295EBD305FB00D5FA0B15FB02D5FB10DC4
:20AD93005FA18A5FB12A5FB2155FA2745FA29A5FB2325FB3115FA3695FA3865FB32E5FB4FA
:20ADB3000E5FA4705FA42C5FB42E5FA5AE5FB52961FF045EA28A5EA3695EA4225EBD205F8A
:20ADD300A2955FA3835FA42961D3045EA2865EA36C5EA41F5FA2925FA37F5FA42561FF048C
:20ADF3005EA28A5EA3695EA4225FA2955FA3835FA42961D3045EA28D5EA3685EA4255FA28B
:20AE13009A5FA3865FA42C61FF045EA28A5EA3695EA4225EB5095FA2955FA3835FA4295F90
:20AE3300B50961D3045EB00D5EB0295EB10A5EB1265EA2865EB3155EA36C5EA38A5EB33282
:20AE53005EA41F5EB5295E71F85E91CA5EBD215FB00D5FB0295FB10A5FB1265FA2925FA38D
:20AE73007F5FA4255FB52961FE045EA28A5EA3865EA4225EBD205FA2955FA3835FA4296160
:20AE9300FF045EA28D5EA3835EA4255FA29A5FA3865FA42C61D3045EB0095EB1065EA28A24
:20AEB3005EA3865EA4225FB0095FB1065FA2955FA3835FA42961FF045EA2865EA38A5EA4E8
:20AED3001F5FA2925FA37F5FA42561D3045EA28A5EA3865EA4225EB5095FA2955FA3835F01
:20AEF300A4295FB50961FF045EB0295EB1265EA28D5EA3835EA4255EB5295EBD305EBD3873
:20AF13005EBD3C5EBD3D5FB0295FB1265FA29A5FA3865FA42C5FB52961D3045EA28A5EA3AF
:20AF3300865EA4225EBD355EBD315EBD305FA2955FA3835FA42961FE045EA2865EA38A5E54
:20AF5300A41F5FA2925FA37F5FA42561FF045EB0095EB1065EA28A5EA3865EA4225EBD20DF
:20AF73005FB0095FB1065FA2955FA3835FA42961D3045EA28D5EA3835EA4255FA29A5FA33C
:20AF9300865FA42C61FF045EA28A5EA3865EA4225EB5095FA2955FA3835FA4295FB509616F
:20AFB300D3045EB02D5EB12A5EB2125EA2865EA2695EB2355EA38A5EB4125EA41F5EA462A9
:20AFD3005EB4325EB5295EBD305EBD315FB02D5FB12A5FB2125FA2925FA2705FB2355FB352
:20AFF3000E5FA37F5FA3655FB3315FB40E5FA4255FA4695FB42E5FB52961FF045EA26C5EA4
:20B01300A3865EA4665EBD215EBD205FA2725FA3685FA46D61D3045EA26D5EA3835EA46934
:20B033005FA2745FA3695FA47061FE045EA26C5EA3865EA4665FA2725FA3685FA46D61D36B
:20B05300045EA2695EA38A5EA4625FA2705FA3655FA46961FF045EA26C5EA3865EA4665E20
:20B07300B5095FA2725FA3685FA46D5FB50961FF045EB00D5EB0295EB10A5EB1265EA26D24
:20B093005EB3125EA3835EA3685EB3355EA4695EB5295EBD215FB00D5FB0295FB10A5FB1E6
:20B0B300265FA2745FA3695FA4705FB52961D3045EA26C5EA3695EA4665EBD205FA2725F44
:20B0D300A3685FA46D61FF045EA2695EA36C5EA4625FA2705FA3655FA46961D3045EB009B1
:20B0F3005EB1065EA26C5EA3695EA4665FB0095FB1065FA2725FA3685FA46D61FE045EA20C
:20B113006D5EA3685EA4695FA2745FA3695FA47061D3045EA26C5EA3695EA4665EB5095F97
:20B13300A2725FA3685FA46D5FB50961FF045EB0295EB1265EA2695EA36C5EA4625EB529AB
:20B153005EBD305EBD315FB0295FB1265FA2705FA3655FA4695FB52961D3045EA26C5EA3B1
:20B17300695EA4665EBD215EBD205FA2725FA3685FA46D61FF045EA26D5EA3685EA4695F23
:20B19300A2745FA3695FA47061FF045EB0095EB1065EA26C5EA3695EA4665FB0095FB106AC
:20B1B3005FA2725FA3685FA46D61D3045EA2695EA36C5EA4625FA2705FA3655FA46961FE1A
:20B1D300045EA26C5EA3695EA4665EB5095FA2725FA3685FA46D5FB50961D3045EB02D5EC3
:20B1F300B12A5EB2155EA26D5EA2835EB2355EA3685EB4125EA4695EA48D5EB4325EB52900
:20B213005EBD305EBD385EBD3C5EBD3D5FB02D5FB12A5FB2155FA2745FA28B5FB2355FB3D9
:20B23300115FA3695FA37F5FB3315FB40E5FA4705FA4955FB42E5FB52961FF045EA2815ECE
:20B25300A3695EA48A5EBD355EBD315EBD305FA2885FA37D5FA49261D3045EA27F5EA36C9B
:20B273005EA4865FA2865FA37B5FA48D61FF045EA2815EA3695EA48A5EBD205FA2885FA3FE
:20B293007D5FA49261FF045EA2835EA3685EA48D5FA28B5FA37F5FA49561D3045EA2815EEE
:20B2B300A3695EA48A5EB5095FA2885FA37D5FA4925FB50961FE045EB00D5EB0295EB10A3F
:20B2D3005EB1265EA27F5EB3155EA36C5EA3815EB3355EA4865EB5295EBD215FB00D5FB021
:20B2F300295FB10A5FB1265FA2865FA37B5FA48D5FB52961D3045EA2815EA37F5EA48A5ECE
:20B31300BD205FA2885FA37D5FA49261FF045EA2835EA37D5EA48D5FA28B5FA37F5FA49507
:20B3330061D3045EB0095EB1065EA2815EA37F5EA48A5FB0095FB1065FA2885FA37D5FA4D0
:20B353009261FF045EA27F5EA3815EA4865FA2865FA37B5FA48D61D3045EA2815EA37F5E30
:20B37300A48A5EB5095FA2885FA37D5FA4925FB50961FF045EB0295EB1265EB2155EA2833E
:20B393005EA29A5EB2355EA37D5EB4125EA48D5EB4325EB5295EBD305EBD315FB0295FB12B
:20B3B300265FB2155FA28B5FA2A25FB2355FB3115FA37F5FA3965FB3315FB40E5FA4955F22
:20B3D300B42E5FB52961FE045EA2985EA37F5EA48A5EBD215EBD205FA29F5FA3945FA492F2
:20B3F30061D3045EA2965EA3815EA4865FA29D5FA3915FA48D61FF045EB0095EB1065EA211
:20B41300985EA37F5EA48A5FB0095FB1065FA29F5FA3945FA49261D3045EA29A5EA37D5ECE
:20B43300A48D5FA2A25FA3965FA49561FF045EA2985EA37F5EA48A5EB5095FA29F5FA3949B
:20B453005FA4925FB50961D3045EB02D5EB12A5EA2965EB3155EA3815EA3985EB3355EA45C
:20B47300865EB5295EBD305EBD315FB02D5FB12A5FA29D5FA3915FA48D5FB52961FF045E2A
:20B49300A2985EA3965EA48A5EBD215EBD205FA29F5FA3945FA49261D2045EA29A5EA39494
:20B4B3005EA48D5FA2A25FA3965FA49561FF045EA2985EA3965EA48A5FA29F5FA3945FA4BF
:20B4D3009261FF045EA2965EA3985EA4865FA29D5FA3915FA48D61D3045EA2985EA3965E26
:20B4F300A48A5EB5095FA29F5FA3945FA4925FB50961FF045EB00D5EB0295EB10A5EB12603
:20B513005EA29A5EA3945EA48D5EB5295EBD305EBD385EBD3C5EBD3D5FB00D5FB0295FB16D
:20B533000A5FB1265FA2A25FA3965FA4955FB52961D3045EA2985EA3965EA48A5EBD355E07
:20B55300BD315EBD305FA29F5FA3945FA49261FF045EA2965EA3985EA4865FA29D5FA39188
:20B573005FA48D61D2045EB0095EB1065EA2985EA3965EA48A5EBD205FB0095FB1065FA2A0
:20B593009F5FA3945FA49261FF045EA29A5EA3945EA48D5FA2A25FA3965FA49561FF045E17
:20B5B300A2985EA3965EA48A5EB5095FA29F5FA3945FA4925FB50961D3045EB0295EB12673
:20B5D3005EB2155EA2965EA2AE5EB2355EA3985EB4125EA4865EB4325EB5295EBD305E71CB
:20B5F300985E91065EBD315FB0295FB1265FB2155FA29D5FA2B65FB2355FB3115FA3915F1B
:20B61300A3A95FB3315FB40E5FA48D5FB42E5FB52961FF045EA2B15EA3965EA48A5EBD21E5
:20B633005EBD205FA2B85FA3AC5FA49261D3045EA2B35EA3945EA48D5FA2BB5FA3AE5FA442
:20B653009561FF045EB0095EB1065EA2B15EA3965EA48A5FB0095FB1065FA2B85FA3AC5FEA
:20B67300A49261D2045EA2AE5EA3985EA4865FA2B65FA3A95FA48D61FF045EA2B15EA396DD
:20B693005EA48A5EB5095FA2B85FA3AC5FA4925FB50961D3045EB02D5EB12A5EA2B35EB366
:20B6B300155EA3945EA3AC5EB3355EA48D5EA58A5EB52A5EBD305E71F85E91CA5EBD315F0B
:20B6D300B02D5FB12A5FA2BB5FA3AE5FA4955FA5865FB52A61FF045EA2B15EA3AE5EA48A24
:20B6F3005EBD215EBD205FA2B85FA3AC5FA49261FF045EA2AE5EA3B15EA4865FA2B65FA3BF
:20B71300A95FA48D61D3045EA2B15EA3AE5EA48A5FA2B85FA3AC5FA49261FF045EA2B35E48
:20B73300A3AC5EA48D5FA2BB5FA3AE5FA49561D2045EA2B15EA3AE5EA48A5EB50A5FA2B81B
:20B753005FA3AC5FA4925FB50A61FF045EB00D5EB0295EB10A5EB1265EA2AE5EA3B15EA40F
:20B77300865EA5B15EB5295EBD305E71985E91065EBD315FB00D5FB0295FB10A5FB1265F4A
:20B79300A2B65FA3A95FA48D5FA5AE5FB52961D3045EA2B15EA3AE5EA48A5EBD215EBD2079
:20B7B3005FA2B85FA3AC5FA49261FF045EA2B35EA3AC5EA48D5FA2BB5FA3AE5FA49561FFC3
:20B7D300045EB0095EB1065EA2B15EA3AE5EA48A5FB0095FB1065FA2B85FA3AC5FA49261AF
:20B7F300D3045EA2AE5EA3B15EA4865FA2B65FA3A95FA48D61FF045EA2B15EA3AE5EA48A35
:20B813005EB5095FA2B85FA3AC5FA4925FB50961D2045EA0985EB02D5EA1665EB12A5EB22A
:20B83300155EA2B35EA2835EB2355EA3AC5EB4125EA48D5EB4325EA5665EB52A5EBD305E72
:20B85300BD385EBD3C5E71F85E91CA5EBD3D5FA0985FB02D5FA1665FB12A5FB2155FA2BB5C
:20B873005FA28B5FB2355FB3115FA3AE5FA37F5FB3315FB40E5FA4955FB42E5FA5625FB5D8
:20B893002A61FF045EA2815EA3AE5EA48A5EBD355EBD315EBD305FA2885FA37D5FA4926166
:20B8B300D3045EA27F5EA3B15EA4865FA2865FA37B5FA48D61FF045EA2815EA3AE5EA48A31
:20B8D3005EBD205FA2885FA37D5FA49261D3045EA2835EA3AC5EA48D5FA28B5FA37F5FA476
:20B8F3009561FF045EA2815EA3AE5EA48A5EB50A5FA2885FA37D5FA4925FB50A61FF045EE6
:20B91300B00D5EA0B15EB02D5EB10A5EA18A5EB12A5EA27F5EB3155EA3B15EA3815EB33573
:20B933005EA4865EA5B15EB5295EBD305E71985E91065EBD315FB00D5FA0B15FB02D5FB171
:20B953000A5FA18A5FB12A5FA2865FA37B5FA48D5FA5AE5FB52961D2045EA2815EA37F5EED
:20B97300A48A5EBD215EBD205FA2885FA37D5FA49261FF045EA2835EA37D5EA48D5FA28BF2
:20B993005FA37F5FA49561D3045EA2815EA37F5EA48A5FA2885FA37D5FA49261FF045EA2B5
:20B9B3007F5EA3815EA4865FA2865FA37B5FA48D61D3045EA2815EA37F5EA48A5EB5095F17
:20B9D300A2885FA37D5FA4925FB50961FF045EB00D5EA0985EB02D5EB10A5EA1665EB12AF2
:20B9F3005EB2155EA2835EA29A5EB2355EA37D5EB4125EA48D5EA4695EB4325EA5985EB51F
:20BA1300295EBD305FB00D5FA0985FB02D5FB10A5FA1665FB12A5FB2155FA28B5FA2A25F42
:20BA3300B2355FB3115FA37F5FA3965FB3315FB40E5FA4955FA4705FB42E5FA5965FB52949
:20BA530061D2045EA2985EA37F5EA4665EBD205FA29F5FA3945FA46D61FF045EA2965EA340
:20BA7300815EA4625FA29D5FA3915FA46961FF045EA2985EA37F5EA4665FA29F5FA3945FB8
:20BA9300A46D61D3045EA29A5EA37D5EA4695FA2A25FA3965FA47061FF045EA2985EA37F9D
:20BAB3005EA4665EB5095FA29F5FA3945FA46D5FB50961D3045EB00D5EB0295EB10A5EB17A
:20BAD300265EA2965EB3155EA3815EA3985EB3355EA4625EB5295E71F85E91CA5EBD215F55
:20BAF300B00D5FB0295FB10A5FB1265FA29D5FA3915FA4695FB52961FF045EA2985EA39681
:20BB13005EA4665EBD205FA29F5FA3945FA46D61D2045EA29A5EA3945EA4695FA2A25FA353
:20BB3300965FA47061FF045EB0095EB1065EA2985EA3965EA4665FB0095FB1065FA29F5F95
:20BB5300A3945FA46D61FF045EA2965EA3985EA4625FA29D5FA3915FA46961D3045EA298C7
:20BB73005EA3965EA4665EB5095FA29F5FA3945FA46D5FB50961FF045EB0295EB1265EA204
:20BB9300945EA3945EA45F5EB5295EBD305EBD385EBD3C5EBD3D5FB0295FB1265FA29A5F17
:20BBB300A38F5FA4665FB52961D3045EA2985EA3965EA4665EBD355EBD315EBD305FA29F44
:20BBD3005FA3945FA46D61FF045EA29D5EA3985EA46D5FA2A45FA3985FA47461D2045EB048
:20BBF300095EB1065EA2985EA3965EA4665EBD205FB0095FB1065FA29F5FA3945FA46D610D
:20BC1300FF045EA2945EA3945EA45F5FA29A5FA38F5FA46661D3045EA2985EA3965EA46620
:20BC33005EB5095FA29F5FA3945FA46D5FB50961FF045EA0665EB02A5EA1985EB1295EA243
:20BC53009D5EA3915EA46D5EB5295EBD215FA0665FB02A5FA1985FB1295FA2A45FA3985FAE
:20BC7300A4745FB52961FF045EA2985EA3965EA4665EBD205FA29F5FA3945FA46D61D30448
:20BC93005EA2945EA39A5EA45F5FA29A5FA38F5FA46661FF045EA2985EA3965EA4665FA270
:20BCB3009F5FA3945FA46D61D2045EA29D5EA3915EA46D5FA2A45FA3985FA47461FF045E7F
:20BCD300A2985EA3965EA4665EB5095FA29F5FA3945FA46D5FB50961D3045EB00A5EA09853
:20BCF3005EB0295EB1095EA1665EB12A5EA2915EA39A5EA45B5EB5295EBD305EBD315FB0D9
:20BD13000A5FA0985FB0295FB1095FA1665FB12A5FA2985FA38D5FA4625FB52961FF045EF2
:20BD3300A2985EA3965EA4665EBD215EBD205FA29F5FA3945FA46D61D3045EA29F5EA39131
:20BD53005EA4705FA2A75FA39A5FA47761FF045EA2985EA3965EA4665FA29F5FA3945FA46C
:20BD73006D61FF045EA2915EA39A5EA45B5FA2985FA38D5FA46261D2045EA2985EA3965E05
:20BD9300A4665EB5095FA29F5FA3945FA46D5FB50961FF045EB0095EA0035EB02A5EB10ADA
:20BDB3005EA1815EB12D5EA29F5EA38F5EA4705EA5035EB52A5EBD305EBD315FB0095FA022
:20BDD300035FB02A5FB10A5FA1815FB12D5FA2A75FA39A5FA4775FA5005FB52A61D3045EA6
:20BDF300A2985EA3965EA4665EBD215EBD205FA29F5FA3945FA46D61FF045EA2915EA39D47
:20BE13005EA45B5FA2985FA38D5FA46261D3045EA2985EA3965EA4665FA29F5FA3945FA41D
:20BE33006D61FF045EA29F5EA38F5EA4705FA2A75FA39A5FA47761FF045EA2985EA3965ECE
:20BE5300A4665EB50A5FA29F5FA3945FA46D5FB50A61D2045EB00A5EA0665EB02A5EB10DDD
:20BE73005EA1CB5EB12D5EA28F5EA39D5EA4585EA5665EB52A5EBD305EBD385EBD3C5EBD6C
:20BE93003D5FB00A5FA0665FB02A5FB10D5FA1CB5FB12D5FA2965FA38B5FA45F5FA5625F2B
:20BEB300B52A61FF045EA2985EA3965EA4665EBD355EBD315EBD305FA29F5FA3945FA46D08
:20BED30061D3045EA2A25EA38F5EA4745FA2A95FA39D5FA47C61FF045EA2985EA3965EA412
:20BEF300665EBD205FA29F5FA3945FA46D61D3045EA28F5EA39D5EA4585FA2965FA38B5FA6
:20BF1300A45F61FF045EA2985EA3965EA4665EB50A5FA29F5FA3945FA46D5FB50A61D304F7
:20BF33005EB00A5EA06C5EB02D5EB10D5EA1225EB12E5EA2A25EA38D5EA4745EA56C5EB58F
:20BF53002D5E71985E91065EBD215FB00A5FA06C5FB02D5FB10D5FA1225FB12E5FA2A95FC3
:20BF7300A39D5FA47C5FA5695FB52D61FE045EA2985EA3965EA4665EBD205FA29F5FA394D6
:20BF93005FA46D61FF045EA28F5EA39F5EA4585FA2965FA38B5FA45F61D3045EA2985EA3DA
:20BFB300965EA4665FA29F5FA3945FA46D61FF045EA2A25EA38D5EA4745FA2A95FA39D5F18
:20BFD300A47C61D3045EA2985EA3965EA4665EB50D5FA29F5FA3945FA46D5FB50D61FF0414
:20BFF3005EB00D5EA0985EB02D5EB10E5EA1665EB12A5EB2155EA29A5EA2255EB2365EA35C
:20C013009F5EB4125EA4695EA48D5EB4325EA5985EB5295EBD305EBD385EBD3C5FB00D5FC5
:20C03300A0985FB02D5FB10E5FA1665FB12A5FB2155FA2A25FA22F5FB2365FB3115FA396C0
:20C053005FA31F5FB3325FB40E5FA4705FA4955FB42E5FA5965FB52961D3045EA2225EA3C9
:20C07300965EA48A5EBD345EBD305FA22C5FA31C5FA49261FE045EA21F5EA38D5EA4865F1A
:20C09300A2295FA3195FA48D61FF045EA2225EA3965EA48A5EBD205FA22C5FA31C5FA49253
:20C0B30061D3045EA2255EA39F5EA48D5FA22F5FA31F5FA49561FF045EA2225EA3965EA4D9
:20C0D3008A5FA22C5FA31C5FA49261D3045EA21F5EB3155EA3985EA3225EB3365EA4865E7D
:20C0F300BD305E71F85E91CA5EBD315FA2295FA3195FA48D61FF045EA2225EA31F5EA48A6D
:20C113005EBD215EBD205FA22C5FA31C5FA49261D3045EA2255EA31C5EA48D5FA22F5FA37A
:20C133001F5FA49561FE045EA2225EA31F5EA48A5FA22C5FA31C5FA49261D3045EA21F5E6F
:20C15300A3225EA4865FA2295FA3195FA48D61FF045EA2225EA31F5EA48A5EB5095FA22C2F
:20C173005FA31C5FA4925FB50961FF045EB00D5EA0CB5EB02D5EB10A5EA1575EB12D5EB29E
:20C19300165EA2255EA2065EB2365EA31C5EB4125EA48D5EA4695EB4325EA5CB5EB5295E1E
:20C1B300BD305EBD385EBD3C5EBD3D5FB00D5FA0CB5FB02D5FB10A5FA1575FB12D5FB21686
:20C1D3005FA22F5FA2105FB2365FB3125FA31F5FA3005FB3325FB40E5FA4955FA4705FB4FA
:20C1F3002E5FA5C85FB52961D3045EA2035EA31F5EA4665EBD355EBD315EBD305FA20C5FDF
:20C21300A3FE5FB3315FA46D61FF045EA2005EA3225EA4625FA20A5FA3FA5FA46961D30421
:20C233005EA2035EA31F5EA4665EBD205FA20C5FA3FE5FA46D61FE045EA2065EA31C5EA420
:20C25300695FA2105FA3005FB3325FA47061D3045EA2035EA31F5EA4665FA20C5FA3FE5F69
:20C27300B3315FA46D61FF045EA2005EB3165EA3225EA3035EB3365EA4625EBD305EBD3163
:20C293005FA20A5FA3FA5FA46961D3045EA2035EA3005EA4665EBD215EBD205FA20C5FA3EE
:20C2B300FE5FA46D61FF045EA2065EA3FE5EB3355EA4695FA2105FA3005FB3325FA47061B8
:20C2D300FF045EA2035EA3005EB3365EA4665FA20C5FA3FE5FB3315FA46D61D3045EA2009D
:20C2F3005EA3035EA4625FA20A5FA3FA5FA46961FE045EA2035EA3005EA4665EB5095FA264
:20C313000C5FA3FE5FA46D5FB50961D3045EB00D5EA0035EB02E5EB10D5EA1815EB12D5EAB
:20C33300B2165EA2065EA2255EB2365EA3FE5EB3355EB4125EA4695EA4255EB4325EA5036C
:20C353005EB52A5EBD305EBD315FB00D5FA0035FB02E5FB10D5FA1815FB12D5FB2165FA298
:20C37300105FA22F5FB2365FB3115FA3005FB3125FA31F5FB3325FB40E5FA4705FA42C5F53
:20C39300B42E5FA5005FB52A61FF045EA2225EA3005EB3365EA4225EBD215EBD205FA22CD0
:20C3B3005FA31C5FA42961D3045EA21F5EA3035EA41F5FA2295FA3195FA42561FF045EA2D3
:20C3D300225EA3005EA4225FA22C5FA31C5FA42961FF045EA2255EA3FE5EB3355EA4255F38
:20C3F300A22F5FA31F5FA42C61D3045EA2225EA3005EB3365EA4225FA22C5FA31C5FA429CC
:20C4130061FE045EA21F5EB3165EA3035EA3225EB3365EA41F5EBD305EBD385EBD3C5EBDC1
:20C433003D5FA2295FA3195FA42561D3045EA2225EA31F5EA4225EBD355EBD315EBD305F5B
:20C45300A22C5FA31C5FA42961FF045EA2255EA31C5EA4255FA22F5FA31F5FA42C61D3042C
:20C473005EA2225EA31F5EA4225EBD205FA22C5FA31C5FA42961FF045EA21F5EA3225EA4E9
:20C493001F5FA2295FA3195FA42561D3045EA2225EA31F5EA4225EB50A5FA22C5FA31C5F98
:20C4B300A4295FB50A61FF045EB00E5EA0665EB02E5EB10D5EA1CB5EB12D5EB2165EA225F1
:20C4D3005EA2695EB2365EA31C5EB4125EA4255EA4065EB4325EA5665EB52A5EBD305EBDDA
:20C4F300385EBD3C5EBD3D5FB00E5FA0665FB02E5FB10D5FA1CB5FB12D5FB2165FA22F5FA8
:20C51300A2745FB2365FB3125FA31F5FA3625FB3325FB40E5FA42C5FA40C5FB42E5FA562B8
:20C533005FB52A61FE045EA2665EA31F5EA4035EBD355EBD315EBD305FA2705FA35F5FA400
:20C553000A61D3045EA2625EA3225EA4005FA26D5FA35B5FA40661FF045EA2665EA31F5EE3
:20C57300A4035EBD205EBD305EBD385EBD3C5FA2705FA35F5FA40A61D3045EA2695EA31C34
:20C593005EA4065EBD345EBD305FA2745FA3625FA40C61FF045EA2665EA31F5EA4035FA20E
:20C5B300705FA35F5FA40A61D3045EA2625EB3165EA3225EA3665EB3365EA4005EBD205E5D
:20C5D300BD305EBD385EBD3C5E71985E91065EBD3D5FA26D5FA35B5FA40661FF045EA2665F
:20C5F3005EA3625EA4035EBD355EBD315EBD305FA2705FA35F5FA40A61D2045EA2695EA359
:20C613005F5EA4065FA2745FA3625FA40C61FF045EA2665EA3625EA4035EBD205FA2705F7B
:20C63300A35F5FA40A61FF045EA2625EA3665EA4005FA26D5FA35B5FA40661D3045EA26637
:20C653005EA3625EA4035EB50A5FA2705FA35F5FA40A5FB50A61FF045EB00E5EA0225EB097
:20C673002E5EB10D5EA1985EB12D5EB2165EC2285EA2695EA2255EB2365EA35F5EB4125E66
:20C6930029C15E490E5E69715E89EF5EE9035E2C515E6C905E8CCB5EA40C5E4C0D5EA42CB3
:20C6B3005EB4365EA5225EB52A5EBD305EBD385EBD3C5EC8215EBD3E5FB00E5FA0225FB0DB
:20C6D3002E5FB10D5FA1985FB12D5FB2165FA2745FA22F5FB2365FB3125FA3625FA31F5F0C
:20C6F300B3325FB40E5FA51F5FB52A61D3045EA2225EA3625EA4295EBD365EBD325EBD30EF
:20C713005FA22C5FA31C61FF045EA21F5EA3665EA4255FA2295FA31961D2045EC2385EA2D6
:20C73300225EA3625EA4295EBD205FA22C5FA31C61FF045EA2255EA35F5EA42C5FA22F5F0A
:20C75300A31F61FF045EA2225EA3625EA4295EB50A5FA22C5FA31C5FB50A61D3045EB00E16
:20C773005EB02A5EB10D5EB1295EB2165EC2185EA21F5EA2965EB2355EB3165EA3665EA333
:20C79300225EB3365EB4165EA4255EA49A5EB4355EA5985EB5295EBD305E71F85E91CA5EEB
:20C7B300BD315FB00E5FB02A5FB10D5FB1295FB2165FA2295FA29D5FB2355FB3125FA31958
:20C7D3005FA3915FB3315FA5965FB52961FF045EA2985EA31F5EA49D5EBD215EBD205FA266
:20C7F3009F5FA39461D3045EA29A5EA31C5EA49F5EB5095FA2A25FA3965FB50961FF045E2B
:20C81300B00A5EB1095EC2385EA2985EA31F5EA49D5FB00A5FB1095FA29F5FA39461D204E5
:20C833005EA2965EA3225EA49A5FA29D5FA39161FF045EA2985EA31F5EA49D5FA29F5FA302
:20C853009461D3045EB02A5EB1295EB2155EC2285EA29A5EA28D5EB2325EB3165EA31C5E11
:20C87300A3945EB3355EB4155EA49F5EA4955EB4325EB5295EBD305EBD315FB02A5FB12940
:20C893005FB2155FA2A25FA29A5FB2325FB3115FA3965FA3865FB32E5FB52961FF045EA2BA
:20C8B3008A5EA3965EA4925EBD215EBD205FA2955FA38361FF045EA2865EA3985EA48D5EAE
:20C8D300B5095FA2925FA37F5FB50961D3045EB00A5EB1095EC2385EA28A5EA3965EA492E1
:20C8F3005FB00A5FB1095FA2955FA38361FF045EA28D5EA3945EA4955FA29A5FA38661D265
:20C91300045EA28A5EA3965EA4925FA2955FA38361FF045EB02E5EB12D5EB2125EC2185E9C
:20C93300A2865EA21F5EB2365EB3155EA3985EA38A5EB3325EB4125EA48D5EA4255EB436A8
:20C953005EA5225EB52A5EBD305EBD385EBD3C5EC8115EBD3E5FB02E5FB12D5FB2125FA23F
:20C97300925FA2295FB2365FB30E5FA37F5FA3195FB3325FA51F5FB52A61D3045EA2225E88
:20C99300A3865EA4295EBD365EBD325EBD305FA22C5FA31C61FF045EA2255EA3835EA42CC1
:20C9B3005FA22F5FA31F61FF045EC2385EA2225EA3865EA4295EBD205FA22C5FA31C61D3C9
:20C9D300045EA21F5EA38A5EA4255FA2295FA31961FF045EA2225EA3865EA4295FA22C5F66
:20C9F300A31C61D2045EB2165EC2285EA2255EA29A5EB2355EB3125EA3835EA31C5EB336B1
:20CA13005EB4165EA42C5EA49F5EB4355EBD305EBD315FB2165FA22F5FA2A25FB2355FB3DC
:20CA3300125FA31F5FA3965FB33161FF045EA2985EA31F5EA49D5EBD215EBD205FA29F5FA4
:20CA5300A39461D3045EA2965EA3225EA49A5FA29D5FA39161FF045EC2385EA2985EA31F5A
:20CA73005EA49D5FA29F5FA39461D3045EA29A5EA31C5EA49F5FA2A25FA39661FF045EA29F
:20CA9300985EA31F5EA49D5EB50A5FA29F5FA3945FB50A61FF045EB2155EC2185EA2965E06
:20CAB300A2865EB2325EB3165EA3225EA3985EB3355EB4155EA49A5EA48D5EB4325EB52EF9
:20CAD3005EBD305EBD315FB2155FA29D5FA2925FB2325FB3115FA3915FA37F5FB32E5FB587
:20CAF3002E61D2045EA28A5EA3965EA4925EBD215EBD205FA2955FA38361FF045EA28D5E28
:20CB1300A3945EA4955FA29A5FA38661D3045EC2385EA28A5EA3965EA4925FA2955FA383B1
:20CB330061FF045EA2865EA3985EA48D5FA2925FA37F61D3045EA28A5EA3965EA4925EB5BC
:20CB53000E5FA2955FA3835FB50E61FF045EB2125EC2285EA28D5EA29A5EB2355EB3155EB9
:20CB7300A3945EA3835EB3325EB4125EA4955EA49F5EB4355EA5E65EB5295EC6185E3032E0
:20CB93005E50445E70F85EC61E5E33115E937F5EB60D5EBD305EBD385EBD3C5EBD3D5FB2F7
:20CBB300125FA29A5FA2A25FB2355FB30E5FA3865FA3965FB3315FA5E35FB52961D2045E90
:20CBD300A2985EA3865EA49D5EBD355EBD315EBD305FA29F5FA39461FF045EA2965EA38A40
:20CBF3005EA49A5FA29D5FA39161FF045EC2385EA2985EA3865EA49D5EBD205FA29F5FA3FE
:20CC13009461D3045EA29A5EA3835EA49F5FA2A25FA39661FF045EA2985EA3865EA49D5EBB
:20CC3300B5095FA29F5FA3945FB50961D3045EB2155EC2185EA2965EA21F5EB2365EB3121D
:20CC53005EA38A5EA3985EB3355EB4155EA49A5EA4255EB4365EA5225EB52A5EC62E5EA66D
:20CC7300035EB60A5EBD305EBD385EBD3C5EBD3D5FB2155FA29D5FA2295FB2365FB3115F7C
:20CC9300A3915FA3195FB3325FA51F5FB52A61FF045EA2225EA3965EA4295EBD355EBD31A9
:20CCB3005EBD305FA22C5FA31C61D2045EA2255EA3945EA42C5FA22F5FA31F61FF045EC2D7
:20CCD300385EA2225EA3965EA4295EBD205FA22C5FA31C61FF045EA21F5EA3985EA4255FFD
:20CCF300A2295FA31961D3045EA2225EA3965EA4295EB50A5FA22C5FA31C5FB50A61FF0435
:20CD13005EB00E5EA0E65EB02D5EB10D5EA16C5EB12D5EB2165EC2285EA2255EA2E95EB276
:20CD3300355EB3155EA3945EA31C5EB3365EB4165EA42C5EA4EF5EB4355EA5E65EB5295E7B
:20CD5300C63E5E30005E50075E70D85EC6385E33005E93F05EA6575EB6095EBD305EBD38EF
:20CD73005EBD3C5EBD3E5FB00E5FA0E65FB02D5FB10D5FA16C5FB12D5FB2165FA22F5FA294
:20CD9300F25FB2355FB3125FA31F5FA3E35FB3315FA5E35FB52961D3045EA2E65EA31F5E1B
:20CDB300A4EC5EBD365EBD325EBD305FA2EF5FA3E161FF045EA2E35EA3225EA4E95FA2ECD2
:20CDD3005FA3DE61D2045EC2385EA2E65EA31F5EA4EC5EBD205FA2EF5FA3E161FF045EA26B
:20CDF300E95EA31C5EA4EF5FA2F25FA3E361D3045EA2E65EA31F5EA4EC5EB5095FA2EF5FBA
:20CE1300A3E15FB50961FF045EB00D5EB0295EB10D5EB1295EB2155EC2185EA2E35EA269AB
:20CE33005EB2355EB3165EA3225EA3E65EB3355EB4155EA4E95EA46D5EB4355EA56C5EB5D9
:20CE5300295EBD305EBD315FB00D5FB0295FB10D5FB1295FB2155FA2EC5FA2705FB2355F2C
:20CE7300B3115FA3DE5FA3655FB3315FA5695FB52961FF045EA26C5EA3E35EA4705EBD2145
:20CE93005EBD205FA2725FA36861D3045EA26D5EA3E15EA4725EB5095FA2745FA3695FB55C
:20CEB3000961FF045EB0095EB1095EC2385EA26C5EA3E35EA4705FB0095FB1095FA2725FA6
:20CED300A36861D2045EA2695EA3E65EA46D5FA2705FA36561FF045EA26C5EA3E35EA47040
:20CEF3005FA2725FA36861D3045EB0295EB1295EB2155EC2285EA26D5EA2695EB2325EB305
:20CF1300155EA3E15EA3685EB3355EB4155EA4725EA4705EB4325EB5295EBD305EBD315FD5
:20CF3300B0295FB1295FB2155FA2745FB2325FB3115FA3695FA3625FB32E5FB52961FF041B
:20CF53005EA2665EA3695EA46D5EBD215EBD205FA2705FA35F61D3045EA2625EA36C5EA42D
:20CF7300695EB5095FA26D5FA35B5FB50961FF045EB0095EB1095EC2385EA2665EA3695E18
:20CF9300A46D5FB0095FB1095FA2705FA35F61FF045EA2695EA3685EA4705FA2745FA362E9
:20CFB30061D2045EA2665EA3695EA46D5FA2705FA35F61FF045EB02D5EB12D5EB2125EC2F9
:20CFD300185EA2625EA2E35EB2355EB3155EA36C5EA3665EB3325EB4125EA4695EA4E95E87
:20CFF300B4355EA5E65EB5295EBD305EBD385EBD3C5EC8215EBD3E5FB02D5FB12D5FB212DF
:20D013005FA26D5FA2EC5FB2355FB30E5FA35B5FA3DE5FB3315FA5E35FB52961D3045EA260
:20D03300E65EA3625EA4EC5EBD365EBD325EBD305FA2EF5FA3E161FF045EA2E95EA35F5EDF
:20D05300A4EF5FA2F25FA3E361D3045EC2385EA2E65EA3625EA4EC5EBD205FA2EF5FA3E17D
:20D0730061FF045EA2E35EA3665EA4E95FA2EC5FA3DE61FF045EA2E65EA3625EA4EC5FA29B
:20D09300EF5FA3E161D2045EB2155EC2285EA2E95EA26D5EB2355EB3125EA35F5EA3E15EA9
:20D0B300B3355EB4155EA4EF5EA4725EB4355EBD305EBD315FB2155FA2F25FA2745FB23537
:20D0D3005FB3115FA3E35FA3695FB33161FF045EA26C5EA3E35EA4705EBD215EBD205FA2E9
:20D0F300725FA36861D3045EA2695EA3E65EA46D5FA2705FA36561FF045EC2385EA26C5EEC
:20D11300A3E35EA4705FA2725FA36861D3045EA26D5EA3E15EA4725FA2745FA36961FF04E8
:20D133005EA26C5EA3E35EA4705EB5095FA2725FA3685FB50961D2045EB2155EC2185EA270
:20D15300695EA2625EB2325EB3155EA3E65EA36C5EB3355EB4155EA46D5EA4695EB4325E4C
:20D17300B52D5EBD305E71985E91065EBD315FB2155FA2705FA26D5FB2325FB3115FA365F5
:20D193005FA35B5FB32E5FB52D61FF045EA2665EA3695EA46D5EBD215EBD205FA2705FA311
:20D1B3005F61FF045EA2695EA3685EA4705FA2745FA36261D3045EC2385EA2665EA3695EBE
:20D1D300A46D5FA2705FA35F61FF045EA2625EA36C5EA4695FA26D5FA35B61D3045EA26652
:20D1F3005EA3695EA46D5EB50D5FA2705FA35F5FB50D61FF045EB2125EC2285EA2695EA2F9
:20D213006D5EB2355EB3155EA3685EA35F5EB3325EB4125EA4705EA4725EB4355EA5B15EB4
:20D23300B5295EBD305EBD385EBD3C5E71F85E91CA5EBD3D5FB2125FA2745FB2355FB30E32
:20D253005FA3625FA3695FB3315FA5AE5FB52961D2045EA26C5EA3625EA4705EBD355EBDD7
:20D27300315EBD305FA2725FA36861FF045EA2695EA3665EA46D5FA2705FA36561FF045E05
:20D29300C2385EA26C5EA3625EA4705EBD205FA2725FA36861D3045EA26D5EA35F5EA472AF
:20D2B3005FA2745FA36961FF045EA26C5EA3625EA4705EB5095FA2725FA3685FB50961D38C
:20D2D300045EB2155EC2185EA2695EA2E35EB2355EB3125EA3665EA36C5EB3355EB4155E87
:20D2F300A46D5EA4E95EB4355EA5E65EB5295EBD305E71985E91065EBD315FB2155FA27029
:20D313005FA2EC5FB2355FB3115FA3655FA3DE5FB3315FA5E35FB52961FF045EA2E65EA3AB
:20D33300695EA4EC5EBD215EBD205FA2EF5FA3E161D2045EA2E95EA3685EA4EF5FA2F25F6D
:20D35300A3E361FF045EC2385EA2E65EA3695EA4EC5FA2EF5FA3E161D3045EA2E35EA36CDF
:20D373005EA4E95FA2EC5FA3DE61FF045EA2E65EA3695EA4EC5EB5095FA2EF5FA3E15FB53D
:20D393000961FF045EB00D5EA0B15EB02D5EB10D5EA18A5EB12A5EB2155EC2285EA2E95E76
:20D3B300A2B35EB2355EB3155EA3685EA3E15EB3355EB4155EA4EF5EA4B85EB4355EA5B13C
:20D3D3005EB5295EBD305EBD385EBD3C5EBD3E5FB00D5FA0B15FB02D5FB10D5FA18A5FB1F1
:20D3F3002A5FB2155FA2F25FA2BB5FB2355FB3115FA3E35FA3AE5FB3315FA5AE5FB529618A
:20D41300D3045EA2B15EA3E35EA4B65EBD365EBD325EBD305FA2B85FA3AC61FF045EA2AE73
:20D433005EA3E65EA4B35FA2B65FA3A961D2045EC2385EA2B15EA3E35EA4B65EBD205FA2C3
:20D45300B85FA3AC61FF045EA2B35EA3E15EA4B85FA2BB5FA3AE61D3045EA2B15EA3E35E09
:20D47300A4B65EB5095FA2B85FA3AC5FB50961FF045EB00D5EB0295EB10A5EB1265EB21576
:20D493005EC2185EA2AE5EA2865EB2325EB3155EA3E65EA3B15EB3355EB4155EA4B35EA4E8
:20D4B3008D5EB4325EA58A5EB5265EBD305E71F85E91CA5EBD315FB00D5FB0295FB10A5FDE
:20D4D300B1265FB2155FA2B65FA2925FB2325FB3115FA3A95FA37F5FB32E5FA5865FB5265C
:20D4F30061D3045EA28A5EA3AE5EA4925EBD215EBD205FA2955FA38361FF045EA28D5EA390
:20D51300AC5EA4955EB5065FA29A5FA3865FB50661FF045EB0095EB1065EC2385EA28A5E8F
:20D53300A3AE5EA4925FB0095FB1065FA2955FA38361D2045EA2865EA3B15EA48D5FA29219
:20D553005FA37F61FF045EA28A5EA3AE5EA4925FA2955FA38361D3045EB0295EB1265EB237
:20D57300125EC2285EA28D5EA2255EB2325EB3155EA3AC5EA3835EB3325EB4125EA4955E97
:20D59300A42C5EB4325EB5265EBD305EBD315FB0295FB1265FB2125FA29A5FA22F5FB232F5
:20D5B3005FB30E5FA3865FA31F5FB32E5FB52661FF045EA2225EA3865EA4295EBD215EBD86
:20D5D300205FA22C5FA31C61D3045EA21F5EA38A5EA4255EB5065FA2295FA3195FB50661EB
:20D5F300FF045EB0095EB1065EC2385EA2225EA3865EA4295FB0095FB1065FA22C5FA31C44
:20D6130061FF045EA2255EA3835EA42C5FA22F5FA31F61D2045EA2225EA3865EA4295FA25F
:20D633002C5FA31C61FF045EB02D5EB12A5EB2125EC2185EA21F5EA2AE5EB2355EB3125EC8
:20D65300A38A5EA3225EB3325EB4125EA4255EA4B35EB4355EA5B15EB5295EBD305EBD384F
:20D673005EBD3C5EC8115EBD3E5FB02D5FB12A5FB2125FA2295FA2B65FB2355FB30E5FA3CE
:20D69300195FA3A95FB3315FA5AE5FB52961D3045EA2B15EA31F5EA4B65EBD365EBD325EC4
:20D6B300BD305FA2B85FA3AC61FF045EA2B35EA31C5EA4B85FA2BB5FA3AE61D3045EC23819
:20D6D3005EA2B15EA31F5EA4B65EBD205FA2B85FA3AC61FF045EA2AE5EA3225EA4B35FA221
:20D6F300B65FA3A961D3045EA2B15EA31F5EA4B65FA2B85FA3AC61FE045EB2155EC2285E60
:20D71300A2B35EA28D5EB2325EB3125EA31C5EA3AC5EB3355EB4155EA4B85EA4955EB432E3
:20D733005EBD305EBD315FB2155FA2BB5FA29A5FB2325FB3115FA3AE5FA3865FB32E61FF84
:20D75300045EA28A5EA3AE5EA4925EBD215EBD205FA2955FA38361D3045EA2865EA3B15E85
:20D77300A48D5FA2925FA37F61FF045EC2385EA28A5EA3AE5EA4925FA2955FA38361D30475
:20D793005EA28D5EA3AC5EA4955FA29A5FA38661FF045EA28A5EA3AE5EA4925EB5095FA234
:20D7B300955FA3835FB50961D3045EB2125EC2185EA2865EA21F5EB2325EB3155EA3B15E70
:20D7D300A38A5EB3325EB4125EA48D5EA4255EB4325EB52D5EBD305EBD315FB2125FA2921B
:20D7F3005FA2295FB2325FB30E5FA37F5FA3195FB32E5FB52D61FE045EA2225EA3865EA45E
:20D81300295EBD215EBD205FA22C5FA31C61D3045EA2255EA3835EA42C5FA22F5FA31F6149
:20D83300FF045EC2385EA2225EA3865EA4295FA22C5FA31C61FF045EA21F5EA38A5EA42526
:20D853005FA2295FA31961D3045EA2225EA3865EA4295EB50D5FA22C5FA31C5FB50D61FF78
:20D87300045EB2125EC2285EA2255EA28D5EB2325EB3125EA3835EA31C5EB3325EB4125EAA
:20D89300A42C5EA4955EB4325EA5985EB5295EC6185E30325E50445E70F85EC61E5E33115B
:20D8B3005E937F5EB60D5EBD305EBD385EBD3C5EBD3D5FB2125FA22F5FA29A5FB2325FB334
:20D8D3000E5FA31F5FA3865FB32E5FA5965FB52961D3045EA28A5EA31F5EA4925EBD355E43
:20D8F300BD315EBD305FA2955FA38361FE045EA2865EA3225EA48D5FA2925FA37F61D304DA
:20D913005EC2385EA28A5EA31F5EA4925EBD205FA2955FA38361FF045EA28D5EA31C5EA4F8
:20D93300955FA29A5FA38661FF045EA28A5EA31F5EA4925EB5095FA2955FA3835FB50961C5
:20D95300D3045EB2125EC2185EA2865EA2AE5EB2355EB3125EA3225EA38A5EB3325EB412D2
:20D973005EA48D5EA4B35EB4355EA5B15EB5295EC62E5EA6035EB60A5EBD305EBD385EBDE9
:20D993003C5EBD3D5FB2125FA2925FA2B65FB2355FB30E5FA37F5FA3A95FB3315FA5AE5F8D
:20D9B300B52961FF045EA2B15EA3865EA4B65EBD355EBD315EBD305FA2B85FA3AC61D3049C
:20D9D3005EA2B35EA3835EA4B85FA2BB5FA3AE61FE045EC2385EA2B15EA3865EA4B65EBD11
:20D9F300205FA2B85FA3AC61D3045EA2AE5EA38A5EA4B35FA2B65FA3A961FF045EA2B15E92
:20DA1300A3865EA4B65EB5095FA2B85FA3AC5FB50961D3045EB00D5EA0E65EB02D5EB10AE7
:20DA33005EA16C5EB12D5EB2155EC2285EA2B35EA2E95EB2355EB3125EA3835EA3AC5EB379
:20DA5300355EB4155EA4B85EA4EF5EB4355EA5E65EB5295EC63E5E30005E50075E70D85E97
:20DA7300C6385E33005E93F05EA6575EB6095EBD305EBD385EBD3C5EBD3E5FB00D5FA0E65C
:20DA93005FB02D5FB10A5FA16C5FB12D5FB2155FA2BB5FA2F25FB2355FB3115FA3AE5FA384
:20DAB300E35FB3315FA5E35FB52961FF045EA2E65EA3AE5EA4EC5EBD365EBD325EBD305FDA
:20DAD300A2EF5FA3E161FF045EA2E35EA3B15EA4E95FA2EC5FA3DE61D3045EC2385EA2E698
:20DAF3005EA3AE5EA4EC5EBD205FA2EF5FA3E161FE045EA2E95EA3AC5EA4EF5FA2F25FA389
:20DB1300E361D3045EA2E65EA3AE5EA4EC5EB5095FA2EF5FA3E15FB50961FF045EB00D5E6B
:20DB3300B0295EB10D5EB1295EB2155EC2185EA2E35EA2695EB2355EB3155EA3B15EA3E6F8
:20DB53005EB3355EB4155EA4E95EA46D5EB4355EA56C5EB5295EBD305EBD315FB00D5FB037
:20DB7300295FB10D5FB1295FB2155FA2EC5FA2705FB2355FB3115FA3DE5FA3655FB3315F3D
:20DB9300A5695FB52961D3045EA26C5EA3E35EA4705EBD215EBD205FA2725FA36861FF0475
:20DBB3005EA26D5EA3E15EA4725EB5095FA2745FA3695FB50961FF045EB0095EB1095EC2C3
:20DBD300385EA26C5EA3E35EA4705FB0095FB1095FA2725FA36861D3045EA2695EA3E65E44
:20DBF300A46D5FA2705FA36561FE045EA26C5EA3E35EA4705FA2725FA36861D3045EB029B8
:20DC13005EB1295EB2155EC2285EA26D5EA2695EB2325EB3155EA3E15EA3685EB3355EB46B
:20DC3300155EA4725EA4705EB4325EB5295EBD305EBD315FB0295FB1295FB2155FA2745F54
:20DC5300B2325FB3115FA3695FA3625FB32E5FB52961FF045EA2665EA3695EA46D5EBD217F
:20DC73005EBD205FA2705FA35F61D3045EA2625EA36C5EA4695EB5095FA26D5FA35B5FB517
:20DC93000961FF045EB0095EB1095EC2385EA2665EA3695EA46D5FB0095FB1095FA2705F3D
:20DCB300A35F61D3045EA2695EA3685EA4705FA2745FA36261FF045EA2665EA3695EA46D57
:20DCD3005FA2705FA35F61FE045EB02D5EB12D5EB2125EC2185EA2625EA2E35EB2355EB390
:20DCF300155EA36C5EA3665EB3325EB4125EA4695EA4E95EB4355EA5E65EB5295EBD305E56
:20DD1300BD385EBD3C5EC8215EBD3E5FB02D5FB12D5FB2125FA26D5FA2EC5FB2355FB30EA7
:20DD33005FA35B5FA3DE5FB3315FA5E35FB52961D3045EA2E65EA3625EA4EC5EBD365EBD51
:20DD5300325EBD305FA2EF5FA3E161FF045EA2E95EA35F5EA4EF5FA2F25FA3E361D3045E54
:20DD7300C2385EA2E65EA3625EA4EC5EBD205FA2EF5FA3E161FF045EA2E35EA3665EA4E9B8
:20DD93005FA2EC5FA3DE61D3045EA2E65EA3625EA4EC5FA2EF5FA3E161FF045EB2155EC2B8
:20DDB300285EA2E95EA26D5EB2355EB3125EA35F5EA3E15EB3355EB4155EA4EF5EA4725EF8
:20DDD300B4355EBD305EBD315FB2155FA2F25FA2745FB2355FB3115FA3E35FA3695FB33126
:20DDF30061D2045EA26C5EA3E35EA4705EBD215EBD205FA2725FA36861FF045EA2695EA3F5
:20DE1300E65EA46D5FA2705FA36561FF045EC2385EA26C5EA3E35EA4705FA2725FA3686106
:20DE3300D3045EA26D5EA3E15EA4725FA2745FA36961FF045EA26C5EA3E35EA4705EB50913
:20DE53005FA2725FA3685FB50961D3045EB2155EC2185EA2695EA2625EB2325EB3155EA3EC
:20DE7300E65EA36C5EB3355EB4155EA46D5EA4695EB4325EB52D5EBD305E71985E91065E6C
:20DE9300BD315FB2155FA2705FA26D5FB2325FB3115FA3655FA35B5FB32E5FB52D61FF046D
:20DEB3005EA2665EA3695EA46D5EBD215EBD205FA2705FA35F61D2045EA2695EA3685EA4BC
:20DED300705FA2745FA36261FF045EC2385EA2665EA3695EA46D5FA2705FA35F61FF045E57
:20DEF300A2625EA36C5EA4695FA26D5FA35B61D3045EA2665EA3695EA46D5EB50D5FA27060
:20DF13005FA35F5FB50D61FF045EB2125EC2285EA2695EA2255EB2365EB3155EA3685EA33A
:20DF33005F5EB3325EB4125EA4705EA42C5EB4365EA5B15EB5295EBD305EBD385EBD3C5EDD
:20DF530071F85E91CA5EBD3D5FB2125FA2745FA22F5FB2365FB30E5FA3625FA31F5FB3323C
:20DF73005FA5AE5FB52961D3045EA2225EA3625EA4295EBD355EBD315EBD305FA22C5FA3A1
:20DF93001C61FF045EA21F5EA3665EA4255FA2295FA31961D2045EC2385EA2225EA3625E8A
:20DFB300A4295EBD205EBD305EBD385EBD3C5FA22C5FA31C61FF045EA2255EA35F5EA42CEF
:20DFD3005EBD345EBD305FA22F5FA31F61D3045EA2225EA3625EA4295EB5095FA22C5FA310
:20DFF3001C5FB50961FF045EB2165EC2185EA21F5EA2625EB2365EB3125EA3665EA3225E41
:20E01300B3365EB4165EA4255EA4695EB4365EA5E65EB5295EBD205EBD305EBD385EBD3CAD
:20E033005E71985E91065EBD3D5FB2165FA2295FA26D5FB2365FB3125FA3195FA35B5FB365
:20E05300325FA5E35FB52961FF045EA2665EA31F5EA46D5EBD355EBD315EBD305FA2705F47
:20E07300A35F61D3045EA2695EA31C5EA4705FA2745FA36261FF045EC2385EA2665EA31F40
:20E093005EA46D5EBD205EBD305EBD385EBD3C5FA2705FA35F61D2045EA2625EA3225EA43E
:20E0B300695EBD345EBD305FA26D5FA35B61FF045EA2665EA31F5EA46D5EB5095FA2705F3A
:20E0D300A35F5FB50961D3045EB00D5EA0225EB02E5EB10D5EA1985EB12D5EB2165EC22802
:20E0F3005EA2695EA2255EB2365EB3165EA31C5EA35F5EB3365EB4165EA4705EA42C5EB474
:20E11300365EA5225EB52A5EBD205EBD305EBD385EBD3C5EBD3E5FB00D5FA0225FB02E5FF2
:20E13300B10D5FA1985FB12D5FB2165FA2745FA22F5FB2365FB3125FA3625FA31F5FB33239
:20E153005FA51F5FB52A61FF045EA2225EA3625EA4295EBD365EBD325EBD305FA22C5FA31F
:20E173001C61D3045EA21F5EA3665EA4255FA2295FA31961FF045EC2385EA2225EA3625EA7
:20E19300A4295EBD205FA22C5FA31C61FF045EA2255EA35F5EA42C5FA22F5FA31F61D2047A
:20E1B3005EA2225EA3625EA4295EB50A5FA22C5FA31C5FB50A61FF045EB00E5EB02A5EB14F
:20E1D3000D5EB1295EB2165EC2185EA21F5EA2965EB2355EB3165EA3665EA3225EB3365E39
:20E1F300B4165EA4255EA49A5EB4355EA5985EB5295EBD305E71F85E91CA5EBD315FB00E2D
:20E213005FB02A5FB10D5FB1295FB2165FA2295FA29D5FB2355FB3125FA3195FA3915FB343
:20E23300315FA5965FB52961D3045EA2985EA31F5EA49D5EBD215EBD205FA29F5FA3946126
:20E25300FF045EA29A5EA31C5EA49F5EB5095FA2A25FA3965FB50961D3045EB00A5EB10974
:20E273005EC2385EA2985EA31F5EA49D5FB00A5FB1095FA29F5FA39461FF045EA2965EA379
:20E29300225EA49A5FA29D5FA39161FF045EA2985EA31F5EA49D5FA29F5FA39461D2045EF6
:20E2B300B02A5EB1295EB2155EC2285EA29A5EA28D5EB2325EB3165EA31C5EA3945EB33544
:20E2D3005EB4155EA49F5EA4955EB4325EB5295EBD305EBD315FB02A5FB1295FB2155FA21C
:20E2F300A25FA29A5FB2325FB3115FA3965FA3865FB32E5FB52961FF045EA28A5EA3965EE8
:20E31300A4925EBD215EBD205FA2955FA38361D3045EA2865EA3985EA48D5EB5095FA2928D
:20E333005FA37F5FB50961FF045EB00A5EB1095EC2385EA28A5EA3965EA4925FB00A5FB162
:20E35300095FA2955FA38361D3045EA28D5EA3945EA4955FA29A5FA38661FF045EA28A5E26
:20E37300A3965EA4925FA2955FA38361D2045EB02E5EB12D5EB2125EC2185EA2865EA21FF4
:20E393005EB2365EB3155EA3985EA38A5EB3325EB4125EA48D5EA4255EB4365EA5225EB53D
:20E3B3002A5EBD305EBD385EBD3C5EC8115EBD3E5FB02E5FB12D5FB2125FA2925FA2295FE2
:20E3D300B2365FB30E5FA37F5FA3195FB3325FA51F5FB52A61FF045EA2225EA3865EA429A9
:20E3F3005EBD365EBD325EBD305FA22C5FA31C61FF045EA2255EA3835EA42C5FA22F5FA369
:20E413001F61D3045EC2385EA2225EA3865EA4295EBD205FA22C5FA31C61FF045EA21F5EFF
:20E43300A38A5EA4255FA2295FA31961D3045EA2225EA3865EA4295FA22C5FA31C61FF0475
:20E453005EB2165EC2285EA2255EA29A5EB2355EB3125EA3835EA31C5EB3365EB4165EA402
:20E473002C5EA49F5EB4355EBD305EBD315FB2165FA22F5FA2A25FB2355FB3125FA31F5FFA
:20E49300A3965FB33161D2045EA2985EA31F5EA49D5EBD215EBD205FA29F5FA39461FF044E
:20E4B3005EA2965EA3225EA49A5FA29D5FA39161FF045EC2385EA2985EA31F5EA49D5FA2AF
:20E4D3009F5FA39461D3045EA29A5EA31C5EA49F5FA2A25FA39661FF045EA2985EA31F5EAF
:20E4F300A49D5EB50A5FA29F5FA3945FB50A61D3045EB2155EC2185EA2965EA2865EB23264
:20E513005EB3165EA3225EA3985EB3355EB4155EA49A5EA48D5EB4325EB52E5EBD305EBD82
:20E53300315FB2155FA29D5FA2925FB2325FB3115FA3915FA37F5FB32E5FB52E61FF045E82
:20E55300A28A5EA3965EA4925EBD215EBD205FA2955FA38361D2045EA28D5EA3945EA495CF
:20E573005FA29A5FA38661FF045EC2385EA28A5EA3965EA4925FA2955FA38361D3045EA2A1
:20E59300865EA3985EA48D5FA2925FA37F61FF045EA28A5EA3965EA4925EB50E5FA2955F77
:20E5B300A3835FB50E61FF045EB2125EC2285EA28D5EA29A5EB2355EB3155EA3945EA38387
:20E5D3005EB3325EB4125EA4955EA49F5EB4355EA5E65EB5295EC6185E30325E50445E7061
:20E5F300F85EC61E5E33115E937F5EB60D5EBD305EBD385EBD3C5EBD3D5FB2125FA29A5F31
:20E61300A2A25FB2355FB30E5FA3865FA3965FB3315FA5E35FB52961D3045EA2985EA3865F
:20E633005EA49D5EBD355EBD315EBD305FA29F5FA39461FF045EA2965EA38A5EA49A5FA2E9
:20E653009D5FA39161D2045EC2385EA2985EA3865EA49D5EBD205FA29F5FA39461FF045EF7
:20E67300A29A5EA3835EA49F5FA2A25FA39661D3045EA2985EA3865EA49D5EB5095FA29F39
:20E693005FA3945FB50961FF045EB2155EC2185EA2965EA21F5EB2365EB3125EA38A5EA349
:20E6B300985EB3355EB4155EA49A5EA4255EB4365EA5225EB52A5EC62E5EA6035EB60A5E00
:20E6D300BD305EBD385EBD3C5EBD3D5FB2155FA29D5FA2295FB2365FB3115FA3915FA31932
:20E6F3005FB3325FA51F5FB52A61D3045EA2225EA3965EA4295EBD355EBD315EBD305FA25E
:20E713002C5FA31C61FF045EA2255EA3945EA42C5FA22F5FA31F61FF045EC2385EA2225EC3
:20E73300A3965EA4295EBD205FA22C5FA31C61D2045EA21F5EA3985EA4255FA2295FA31981
:20E7530061FF045EA2225EA3965EA4295EB50A5FA22C5FA31C5FB50A61D3045EB00E5EA086
:20E77300E65EB02D5EB10D5EA16C5EB12D5EB2165EC2285EA2255EA2E95EB2355EB3155E5D
:20E79300A3945EA31C5EB3365EB4165EA42C5EA4EF5EB4355EA5E65EB5295EC63E5E300028
:20E7B3005E50075E70D85EC6385E33005E93F05EA6575EB6095EBD305EBD385EBD3C5EBD95
:20E7D3003E5FB00E5FA0E65FB02D5FB10D5FA16C5FB12D5FB2165FA22F5FA2F25FB2355FF5
:20E7F300B3125FA31F5FA3E35FB3315FA5E35FB52961FF045EA2E65EA31F5EA4EC5EBD362B
:20E813005EBD325EBD305FA2EF5FA3E161D3045EA2E35EA3225EA4E95FA2EC5FA3DE61FF24
:20E83300045EC2385EA2E65EA31F5EA4EC5EBD205FA2EF5FA3E161FF045EA2E95EA31C5E9F
:20E85300A4EF5FA2F25FA3E361D2045EA2E65EA31F5EA4EC5EB5095FA2EF5FA3E15FB50903
:20E8730061FF045EB00D5EB0295EB10D5EB1295EB2155EC2185EA2E35EA2695EB2355EB37C
:20E89300165EA3225EA3E65EB3355EB4155EA4E95EA46D5EB4355EA56C5EB5295EBD305EE3
:20E8B300BD315FB00D5FB0295FB10D5FB1295FB2155FA2EC5FA2705FB2355FB3115FA3DEE0
:20E8D3005FA3655FB3315FA5695FB52961D3045EA26C5EA3E35EA4705EBD215EBD205FA25F
:20E8F300725FA36861FF045EA26D5EA3E15EA4725EB5095FA2745FA3695FB50961D3045E53
:20E91300B0095EB1095EC2385EA26C5EA3E35EA4705FB0095FB1095FA2725FA36861FF0487
:20E933005EA2695EA3E65EA46D5FA2705FA36561D3045EA26C5EA3E35EA4705FA2725FA3BE
:20E953006861FE045EB0295EB1295EB2155EC2285EA26D5EA2695EB2325EB3155EA3E15E7F
:20E97300A3685EB3355EB4155EA4725EA4705EB4325EB5295EBD305EBD315FB0295FB1299E
:20E993005FB2155FA2745FB2325FB3115FA3695FA3625FB32E5FB52961FF045EA2665EA34C
:20E9B300695EA46D5EBD215EBD205FA2705FA35F61D3045EA2625EA36C5EA4695EB5095F36
:20E9D300A26D5FA35B5FB50961FF045EB0095EB1095EC2385EA2665EA3695EA46D5FB00959
:20E9F3005FB1095FA2705FA35F61D3045EA2695EA3685EA4705FA2745FA36261FF045EA260
:20EA1300665EA3695EA46D5FA2705FA35F61D3045EB02D5EB12D5EB2125EC2185EA2625E09
:20EA3300A2E35EB2355EB3155EA36C5EA3665EB3325EB4125EA4695EA4E95EB4355EA5E612
:20EA53005EB5295EBD305EBD385EBD3C5EC8215EBD3E5FB02D5FB12D5FB2125FA26D5FA2C7
:20EA7300EC5FB2355FB30E5FA35B5FA3DE5FB3315FA5E35FB52961FE045EA2E65EA3625E83
:20EA9300A4EC5EBD365EBD325EBD305FA2EF5FA3E161D3045EA2E95EA35F5EA4EF5FA2F2B2
:20EAB3005FA3E361FF045EC2385EA2E65EA3625EA4EC5EBD205FA2EF5FA3E161FF045EA2F9
:20EAD300E35EA3665EA4E95FA2EC5FA3DE61D3045EA2E65EA3625EA4EC5FA2EF5FA3E1617E
:20EAF300FF045EB2155EC2285EA2E95EA26D5EB2355EB3125EA35F5EA3E15EB3355EB41526
:20EB13005EA4EF5EA4725EB4355EBD305EBD315FB2155FA2F25FA2745FB2355FB3115FA3A6
:20EB3300E35FA3695FB33161D3045EA26C5EA3E35EA4705EBD215EBD205FA2725FA3686182
:20EB5300FE045EA2695EA3E65EA46D5FA2705FA36561D3045EC2385EA26C5EA3E35EA470B7
:20EB73005FA2725FA36861FF045EA26D5EA3E15EA4725FA2745FA36961FF045EA26C5EA3CD
:20EB9300E35EA4705EB5095FA2725FA3685FB50961D3045EB2155EC2185EA2695EA2625E39
:20EBB300B2325EB3155EA3E65EA36C5EB3355EB4155EA46D5EA4695EB4325EB52D5EBD30CE
:20EBD3005E71985E91065EBD315FB2155FA2705FA26D5FB2325FB3115FA3655FA35B5FB339
:20EBF3002E5FB52D61FF045EA2665EA3695EA46D5EBD215EBD205FA2705FA35F61D3045E11
:20EC1300A2695EA3685EA4705FA2745FA36261FE045EC2385EA2665EA3695EA46D5FA270B7
:20EC33005FA35F61D3045EA2625EA36C5EA4695FA26D5FA35B61FF045EA2665EA3695EA4ED
:20EC53006D5EB50D5FA2705FA35F5FB50D61D3045EB2125EC2285EA2695EA26D5EB2355E06
:20EC7300B3155EA3685EA35F5EB3325EB4125EA4705EA4725EB4355EA5B15EB5295EBD3021
:20EC93005EBD385EBD3C5E71F85E91CA5EBD3D5FB2125FA2745FB2355FB30E5FA3625FA37B
:20ECB300695FB3315FA5AE5FB52961FF045EA26C5EA3625EA4705EBD355EBD315EBD305FBB
:20ECD300A2725FA36861FF045EA2695EA3665EA46D5FA2705FA36561D3045EC2385EA26C2C
:20ECF3005EA3625EA4705EBD205FA2725FA36861FE045EA26D5EA35F5EA4725FA2745FA3F9
:20ED13006961D3045EA26C5EA3625EA4705EB5095FA2725FA3685FB50961FF045EB2155E01
:20ED3300C2185EA2695EA2E35EB2355EB3125EA3665EA36C5EB3355EB4155EA46D5EA4E997
:20ED53005EB4355EA5E65EB5295EBD305E71985E91065EBD315FB2155FA2705FA2EC5FB2AC
:20ED7300355FB3115FA3655FA3DE5FB3315FA5E35FB52961D3045EA2E65EA3695EA4EC5EA6
:20ED9300BD215EBD205FA2EF5FA3E161FF045EA2E95EA3685EA4EF5FA2F25FA3E361FF0491
:20EDB3005EC2385EA2E65EA3695EA4EC5FA2EF5FA3E161D3045EA2E35EA36C5EA4E95FA263
:20EDD300EC5FA3DE61FE045EA2E65EA3695EA4EC5EB5095FA2EF5FA3E15FB50961D3045E11
:20EDF300B00D5EA0B15EB02D5EB10D5EA18A5EB12A5EB2155EC2285EA2E95EA2B35EB2352D
:20EE13005EB3155EA3685EA3E15EB3355EB4155EA4EF5EA4B85EB4355EA5B15EB5295EBD04
:20EE3300305EBD385EBD3C5EBD3E5FB00D5FA0B15FB02D5FB10D5FA18A5FB12A5FB2155F1E
:20EE5300A2F25FA2BB5FB2355FB3115FA3E35FA3AE5FB3315FA5AE5FB52961FF045EA2B10A
:20EE73005EA3E35EA4B65EBD365EBD325EBD305FA2B85FA3AC61D3045EA2AE5EA3E65EA4C4
:20EE9300B35FA2B65FA3A961FF045EC2385EA2B15EA3E35EA4B65EBD205FA2B85FA3AC613E
:20EEB300D3045EA2B35EA3E15EA4B85FA2BB5FA3AE61FF045EA2B15EA3E35EA4B65EB509E0
:20EED3005FA2B85FA3AC5FB50961FE045EB00D5EB0295EB10A5EB1265EB2155EC2185EA23B
:20EEF300AE5EA2865EB2325EB3155EA3E65EA3B15EB3355EB4155EA4B35EA48D5EB4325E77
:20EF1300A58A5EB5265EBD305E71F85E91CA5EBD315FB00D5FB0295FB10A5FB1265FB21595
:20EF33005FA2B65FA2925FB2325FB3115FA3A95FA37F5FB32E5FA5865FB52661D3045EA2A6
:20EF53008A5EA3AE5EA4925EBD215EBD205FA2955FA38361FF045EA28D5EA3AC5EA4955EAC
:20EF7300B5065FA29A5FA3865FB50661D3045EB0095EB1065EC2385EA28A5EA3AE5EA492FD
:20EF93005FB0095FB1065FA2955FA38361FF045EA2865EA3B15EA48D5FA2925FA37F61D3A2
:20EFB300045EA28A5EA3AE5EA4925FA2955FA38361FF045EB0295EB1265EB2125EC2285EBA
:20EFD300A28D5EA2255EB2325EB3155EA3AC5EA3835EB3325EB4125EA4955EA42C5EB432C1
:20EFF3005EB5265EBD305EBD315FB0295FB1265FB2125FA29A5FA22F5FB2325FB30E5FA36D
:20F01300865FA31F5FB32E5FB52661D2045EA2225EA3865EA4295EBD215EBD205FA22C5FAE
:20F03300A31C61FF045EA21F5EA38A5EA4255EB5065FA2295FA3195FB50661FF045EB009D6
:20F053005EB1065EC2385EA2225EA3865EA4295FB0095FB1065FA22C5FA31C61D3045EA2AB
:20F07300255EA3835EA42C5FA22F5FA31F61FF045EA2225EA3865EA4295FA22C5FA31C6171
:20F09300D3045EB02D5EB12A5EB2125EC2185EA21F5EA2AE5EB2355EB3125EA38A5EA322D5
:20F0B3005EB3325EB4125EA4255EA4B35EB4355EA5B15EB5295EBD305EBD385EBD3C5EC8A8
:20F0D300115EBD3E5FB02D5FB12A5FB2125FA2295FA2B65FB2355FB30E5FA3195FA3A95FAE
:20F0F300B3315FA5AE5FB52961FF045EA2B15EA31F5EA4B65EBD365EBD325EBD305FA2B89B
:20F113005FA3AC61D2045EA2B35EA31C5EA4B85FA2BB5FA3AE61FF045EC2385EA2B15EA393
:20F133001F5EA4B65EBD205FA2B85FA3AC61FF045EA2AE5EA3225EA4B35FA2B65FA3A96196
:20F15300D3045EA2B15EA31F5EA4B65FA2B85FA3AC61FF045EB2155EC2285EA2B35EA28DC4
:20F173005EB2325EB3125EA31C5EA3AC5EB3355EB4155EA4B85EA4955EB4325EBD305EBDE5
:20F19300315FB2155FA2BB5FA29A5FB2325FB3115FA3AE5FA3865FB32E61D3045EA28A5EB0
:20F1B300A3AE5EA4925EBD215EBD205FA2955FA38361FF045EA2865EA3B15EA48D5FA29207
:20F1D3005FA37F61D2045EC2385EA28A5EA3AE5EA4925FA2955FA38361FF045EA28D5EA332
:20F1F300AC5EA4955FA29A5FA38661D3045EA28A5EA3AE5EA4925EB5095FA2955FA3835FFB
:20F21300B50961FF045EB2125EC2185EA2865EA21F5EB2325EB3155EA3B15EA38A5EB332D2
:20F233005EB4125EA48D5EA4255EB4325EB52D5EBD305EBD315FB2125FA2925FA2295FB2D5
:20F25300325FB30E5FA37F5FA3195FB32E5FB52D61FF045EA2225EA3865EA4295EBD215E5A
:20F27300BD205FA22C5FA31C61D3045EA2255EA3835EA42C5FA22F5FA31F61FF045EC23837
:20F293005EA2225EA3865EA4295FA22C5FA31C61D2045EA21F5EA38A5EA4255FA2295FA308
:20F2B3001961FF045EA2225EA3865EA4295EB50D5FA22C5FA31C5FB50D61D3045EB2125EA6
:20F2D300C2285EA2255EA2B35EB2355EB3125EA3835EA31C5EB3325EB4125EA42C5EA4B801
:20F2F3005EB4355EA5985EB5295EC6185E30325E50445E70F85EC61E5E33115E937F5EB6C1
:20F313000D5EBD305EBD385EBD3C5EBD3D5FB2125FA22F5FA2BB5FB2355FB30E5FA31F5F8B
:20F33300A3AE5FB3315FA5965FB52961FF045EA2B15EA31F5EA4B65EBD355EBD315EBD307B
:20F353005FA2B85FA3AC61D3045EA2AE5EA3225EA4B35FA2B65FA3A961FF045EC2385EA257
:20F37300B15EA31F5EA4B65EBD205FA2B85FA3AC61FF045EA2B35EA31C5EA4B85FA2BB5F46
:20F39300A3AE61D2045EA2B15EA31F5EA4B65EB5095FA2B85FA3AC5FB50961FF045EB21520
:20F3B3005EC2185EA2AE5EA2E35EB2355EB3125EA3225EA3B15EB3355EB4155EA4B35EA410
:20F3D300E95EB4355EA5B15EB5295EC62E5EA6035EB60A5EBD305EBD385EBD3C5EBD3D5FD7
:20F3F300B2155FA2B65FA2EC5FB2355FB3115FA3A95FA3DE5FB3315FA5AE5FB52961D30431
:20F413005EA2E65EA3AE5EA4EC5EBD355EBD315EBD305FA2EF5FA3E161FF045EA2E95EA34E
:20F43300AC5EA4EF5FA2F25FA3E361D3045EC2385EA2E65EA3AE5EA4EC5EBD205FA2EF5FA7
:20F45300A3E161FF045EA2E35EA3B15EA4E95FA2EC5FA3DE61FF045EA2E65EA3AE5EA4EC7D
:20F473005EB5095FA2EF5FA3E15FB50961D2045EB00D5EA0985EB02D5EB10A5EA1665EB1BD
:20F493002A5EB2155EA2E95EA29A5EB2355EB3155EA3AC5EA3E15EB3355EB4155EA4EF5ED1
:20F4B300A49F5EB4355EA5985EB5295EC63E5E30005E50075E70D85EC6385E33005E93F0BF
:20F4D3005EA6575EB6095EBD305EBD385EBD3C5EBD3E5FB00D5FA0985FB02D5FB10A5FA14A
:20F4F300665FB12A5FB2155FA2F25FA2A25FB2355FB3115FA3E35FA3965FB3315FA5965F7B
:20F51300B52961FF045EA2985EA3E35EA49D5EBD365EBD325EBD305FA29F5FA39461D30424
:20F533005EA2965EA3E65EA49A5FA29D5FA39161FF045EB2155EA2985EA2B15EB2355EA356
:20F55300E35EB4155EA49D5EA4B65EB4355EBD205FB2155FA29F5FA2B85FB2355FB3115F6E
:20F57300A3945FA3AC5FB33161D3045EA2B35EA3E15EA4B85FA2BB5FA3AE61FF045EA2B148
:20F593005EA3E35EA4B65EB5095FA2B85FA3AC5FB50961D2045EB00D5EB10A5EA2AE5EB3F2
:20F5B300155EA3E65EA3985EB3355EA4B35EBD305EBD315FB00D5FB10A5FA2B65FA3A96118
:20F5D300FF045EA2B15EA3965EA4B65EBD215EBD205FA2B85FA3AC61FF045EA2B35EA3948B
:20F5F3005EA4B85FA2BB5FA3AE61D3045EA2B15EB3155EA3965EA3AE5EB3355EA4B65FA27E
:20F61300B85FA3AC61FF045EA2AE5EA3B15EA4B35FA2B65FA3A961D3045EA2B15EA3AE5EA0
:20F63300A4B65FA2B85FA3AC61FF045EA2B35EA3AC5EA4B85EBD305EBD315FA2BB5FA3AE75
:20F6530061D2045EA2B15EA3AE5EA4B65EBD215EBD205FA2B85FA3AC61FF045EA2AE5EA357
:20F67300B15EA4B35FA2B65FA3A961FF045EA2B15EA3AE5EA4B65FA2B85FA3AC61D3045E36
:20F69300A2B35EA3AC5EA4B85FA2BB5FA3AE61FF045EA2B15EA3AE5EA4B65FA2B85FA3AC4C
:20F6B30061D3045EB02D5EB12A5EB2155EA2AE5EA2965EB2355EA3B15EB4155EA4B35EA44D
:20F6D3009A5EB4355EB5295EBD305EBD385EBD3C5FB02D5FB12A5FB2155FA2B65FA29D5FB5
:20F6F300B2355FB3115FA3A95FA3915FB3315FB52961FF045EA2985EA3AE5EA49D5EBD3496
:20F713005EBD305FA29F5FA39461D2045EA29A5EA3AC5EA49F5FA2A25FA39661FF045EA297
:20F73300985EA3AE5EA49D5EBD205FA29F5FA39461D3045EA2965EA3B15EA49A5FA29D5F46
:20F75300A39161FF045EA2985EA3AE5EA49D5FA29F5FA39461FF045EA29A5EB3155EA3AC11
:20F773005EA3945EB3355EA49F5EBD305EBD315FA2A25FA39661D3045EA2985EA3965EA4BF
:20F793009D5EBD215EBD205FA29F5FA39461FF045EA2965EA3985EA49A5FA29D5FA391614B
:20F7B300D2045EA2985EA3965EA49D5FA29F5FA39461FF045EA29A5EA3945EA49F5FA2A285
:20F7D3005FA39661D3045EA2985EA3965EA49D5FA29F5FA39461FF045EA2965EA3985EA4AD
:20F7F3009A5EBD215FA29D5FA39161D3045EA2985EA3965EA49D5EBD205FA29F5FA3946117
:20F81300FF045EA29A5EA3945EA49F5FA2A25FA39661FF045EA2985EA3965EA49D5FA29FF5
:20F833005FA39461D2045EA2965EA3985EA49A5FA29D5FA39161FF045EA2985EA3965EA457
:20F853009D5FA29F5FA39461D3045EA29A5EA3945EA49F5EBD305EBD385EBD3C5EBD3D5F0E
:20F87300A2A25FA39661FF045EA2985EA3965EA49D5EBD2D5EBD3D5EBD355EBD3D5EBD39CB
:20F893005EBD3D5EBD3C5FA29F5FA39461D3045EA2965EA3985EA49A5EBD345EBD305FA2D2
:20F8B3009D5FA39161FF045EA2985EA3965EA49D5FA29F5FA39461FF045EA29A5EA3945EAC
:20F8D300A49F5EBD205FA2A25FA39661D2045EA2985EA3965EA49D5FA29F5FA39461FF04BD
:20F8F3005EA2965EA3985EA49A5FA29D5FA39161D3045EA2985EA3965EA49D5FA29F5FA351
:20F913009461FF045EA29A5EA3945EA49F5FA2A25FA39661D3045EA2985EA3965EA49D5F6C
:20F93300A29F5FA39461FF045EA2965EA3985EA49A5FA29D5FA39161D3045EA2985EA39616
:20F953005EA49D5EB5095FA29F5FA3945FB50961FE045EB00D5EB02D5EB10A5EA1225EB184
:20F973002A5EB2155EA2965EA2865EB2325EA3945E4B0B5EA31C5EB32A5EB4155EA4965E09
:20F99300A41F5EB4325EA5225EB52A5EBD305EBD385EC8315EBD3C5EC8115EBD3E5E7198A8
:20F9B3005E91065FB00D5FB02D5FB10A5FA1225FB12A5FB2155FA2985FA28A5FB2325FB3D2
:20F9D300115FA3985FA3225FB32E5FC4365F29015F49805F69925F898A5FC4385F2CE55F05
:20F9F3006CC15F8C9E5FEC005FA4035F4C145FA51F5FB52A61FF045EA28A5EA4225EBD2E72
:20FA13005EBD3E5EBD365EBD3E5EBD3A5EBD3E5EBD3C61D3045EA28D5EA4255EBD2C5EBD7D
:20FA3300245EBD2061FF045EA28A5EA42261D3045EA2865EA41F61FF045EA28A5EA4225EF3
:20FA5300B50A5FB50A61D3045EB00D5EB0295EB10A5EB12A5EA28D5EB30A5EA3195EA37F98
:20FA73005EB3325EA4255EB52A5EBD305E71F85E91CA5EBD315FB00D5FB0295FB10A5FB137
:20FA93002A5FB52A61FE045EA28A5EA3835EA4225EBD215EBD2061D3045EA2865EA3865E3C
:20FAB300A41F5EB50A5FB50A61FF045EB0095EB10A5EA28A5EA3835EA4225FB0095FB10A3D
:20FAD30061FF045EA28D5EA37F5EA42561D3045EA28A5EA3835EA42261FF045EA0665EB03B
:20FAF3002E5EA1985EB12D5EA2835EA3865EA41C5EA5985EB52D5EBD305EBD385EBD3C5E9C
:20FB130071985E91065EBD3D5FA0665FB02E5FA1985FB12D5FA5965FB52D61D3045EA28A68
:20FB33005EA3835EA4225EBD355EBD315EBD3061FE045EA2925EA37F5EA42961D3045EA24B
:20FB53008A5EA3835EA4225EBD2061FF045EA2835EA3865EA41C61FF045EA28A5EA3835EC9
:20FB7300A4225EB50D5FB50D61D3045EB00E5EA0985EB0295EB10D5EA1225EB12A5EA29242
:20FB93005EA37C5EA4295EA5225EB52A5EBD305E71F85E91CA5EBD315FB00E5FA0985FB06E
:20FBB300295FB10D5FA1225FB12A5FA51F5FB52A61FF045EA28A5EA3835EA4225EBD215EFF
:20FBD300BD2061D3045EA2835EA38A5EA41C5EB50A5FB50A61FE045EB0095EB10A5EA28A79
:20FBF3005EA3835EA4225FB0095FB10A61D3045EA2925EA37C5EA42961FF045EA28A5EA3B7
:20FC1300835EA42261D3045EA08A5EB02E5EA1B15EB12D5EA2835EA38A5EA41C5EA5B15E04
:20FC3300B52D5EBD305EBD385EBD3C5E71985E91065EBD3D5FA08A5FB02E5FA1B15FB12D72
:20FC53005FA5AE5FB52D61FF045EA28A5EA3835EA4225EBD355EBD315EBD3061FF045EA2BD
:20FC7300925EA37C5EA42961D3045EA28A5EA3835EA4225EBD2061FE045EA2835EA38A5EC3
:20FC9300A41C61D3045EA28A5EA3835EA4225EB50D5FB50D61FF045EB00E5EA0985EB02999
:20FCB3005EB10D5EA1225EB12A5EA2925EA37C5EA4295EA5225EB52A5EBD305E71F85E911E
:20FCD300CA5EBD315FB00E5FA0985FB0295FB10D5FA1225FB12A5FA51F5FB52A61D3045E9F
:20FCF300A28A5EA3835EA4225EBD215EBD2061FF045EA2835EA38A5EA41C5EB50A5FB50ADB
:20FD130061FF045EB0095EB10A5EA28A5EA3835EA4225FB0095FB10A61D3045EA2925EA30D
:20FD33007C5EA42961FE045EA28A5EA3835EA42261D3045EA0225EB02E5EA16C5EB12D5EDB
:20FD5300A27F5EA38A5EA4195EA56C5EB52D5EBD305EBD385EBD3C5E71985E91065EBD3D71
:20FD73005FA0225FB02E5FA16C5FB12D5FA5695FB52D61FF045EA28A5EA3835EA4225EBD0A
:20FD9300355EBD315EBD3061D3045EA2955EA37C5EA42C61FF045EA28A5EA3835EA4225E18
:20FDB300BD2061D3045EA27F5EA38A5EA41961FF045EA28A5EA3835EA4225EB50D5FB50D1F
:20FDD30061FE045EB00E5EA0985EB0295EB10D5EA1225EB12A5EA2955EA3775EA42C5EA510
:20FDF300225EB52A5EBD305E71F85E91CA5EBD315FB00E5FA0985FB0295FB10D5FA1225FF0
:20FE1300B12A5FA51F5FB52A61D3045EA28A5EA3835EA4225EBD215EBD2061FF045EA27FCF
:20FE33005EA38D5EA4195EB50A5FB50A61D3045EB0095EB10A5EA28A5EA3835EA4225FB022
:20FE5300095FB10A61FF045EA2955EA3775EA42C61D3045EA28A5EA3835EA42261FF045EA1
:20FE7300A0665EB02E5EA1985EB12D5EA27F5EA38D5EA4195EA5985EB52D5EBD305EBD38B9
:20FE93005EBD3C5E71985E91065EBD3D5FA0665FB02E5FA1985FB12D5FA5965FB52D61D2BF
:20FEB300045EA28A5EA3835EA4225EBD355EBD315EBD3061FF045EA2955EA3775EA42C6112
:20FED300FF045EA28A5EA3835EA4225EBD2061D3045EA27F5EA38D5EA41961FF045EA28A51
:20FEF3005EA3835EA4225EB50D5FB50D61D3045EB00E5EA0985EB0295EB10D5EA1225EB199
:20FF13002A5EA2955EA3775EA42C5EA5225EB52A5EBD305E71F85E91CA5EBD315FB00E5F74
:20FF3300A0985FB0295FB10D5FA1225FB12A5FA51F5FB52A61FF045EA28A5EA3835EA422CE
:20FF53005EBD215EBD2061D2045EA27F5EA38D5EA4195EB50A5FB50A61FF045EB0095EB1F3
:20FF73000A5EA28A5EA3835EA4225FB0095FB10A61FF045EA2955EA3775EA42C61D3045ECB
:20FF9300A28A5EA3835EA42261FF045EA0E65EB02D5EA18A5EB12A5EA27C5EA38D5EA41613
:20FFB3005EA58A5EB52A5EBD305EBD385EBD3C5E71985E91065EBD3D5FA0E65FB02D5FA19A
:20FFD3008A5FB12A5FA5865FB52A61D3045EA28A5EA3835EA4225EBD355EBD315EBD3061D0
:0DFFF300FF045EA29A5EA3775EA42F61D288
:020000040017E3
:13000000045EA28A5EA3835EA4225EBD2061FF045EA27C9C
:200013005EA38D5EA41661D3045EA28A5EA3835EA4225EB50A5FB50A61FF045EB00D5EA005
:20003300985EB0295EB10A5EA1225EB12A5EA29A5EA3745EA42F5EA5225EB52A5EBD305E20
:2000530071F85E91CA5EBD315FB00D5FA0985FB0295FB10A5FA1225FB12A5FA51F5FB52A5D
:2000730061FF045EA28A5EA3835EA4225EBD215EBD2061D3045EA27C5EA3925EA4165EB5EE
:200093000A5FB50A61FF045EB0095EB10A5EA28A5EA3835EA4225FB0095FB10A61D2045E98
:2000B300A29A5EA3745EA42F61FF045EA28A5EA3835EA42261D3045EA0225EB02E5EA16CB6
:2000D3005EB12D5EA27C5EA3925EA4165EA56C5EB52D5EBD305EBD385EBD3C5E71985E91B0
:2000F300065EBD3D5FA0225FB02E5FA16C5FB12D5FA5695FB52D61FF045EA28A5EA3835E0A
:20011300A4225EBD355EBD315EBD3061D3045EA29A5EA3745EA42F61FF045EA28A5EA38335
:200133005EA4225EBD2061FF045EA27C5EA3925EA41661D2045EA28A5EA3835EA4225EB546
:200153000D5FB50D61FF045EB00E5EA0985EB0295EB10D5EA1225EB12A5EA29A5EA3745E2E
:20017300A42F5EA5225EB52A5EBD305E71F85E91CA5EBD315FB00E5FA0985FB0295FB10D17
:200193005FA1225FB12A5FA51F5FB52A61D3045EA28A5EA3835EA4225EBD215EBD2061FF4E
:2001B300045EA27C5EA3925EA4165EB50A5FB50A61D3045EB0095EB10A5EA28A5EA3835EF2
:2001D300A4225FB0095FB10A61FF045EA29A5EA3745EA42F61FF045EA28A5EA3835EA422DA
:2001F30061D2045EA0CB5EB02D5EA1665EB12A5EA2775EA3925EA4125EA5665EB52A5EBD34
:20021300305EBD385EBD3C5E71985E91065EBD3D5FA0CB5FB02D5FA1665FB12A5FA5625FD2
:20023300B52A61FF045EA28A5EA3835EA4225EBD355EBD315EBD3061D3045EA29D5EA37405
:200253005EA43261FF045EA28A5EA3835EA4225EBD2061D3045EA2775EA3925EA41261FFD0
:20027300045EA28A5EA3835EA4225EB50A5FB50A61D2045EB00D5EA0985EB0295EB10A5E64
:20029300A1225EB12A5EA29D5EA3705EA4325EA5225EB52A5EBD305E71F85E91CA5EBD3194
:2002B3005FB00D5FA0985FB0295FB10A5FA1225FB12A5FA51F5FB52A61FF045EA28A5EA37A
:2002D300835EA4225EBD215EBD2061FF045EA2775EA3955EA4125EB50A5FB50A61D3045E97
:2002F300B0095EB10A5EA28A5EA3835EA4225FB0095FB10A61FF045EA29D5EA3705EA4320F
:2003130061D3045EA28A5EA3835EA42261FF045EB02D5EB12A5EB2125EA3955EB4125EB599
:200333002A5EBD305EBD385EBD3C5E71985E91065EBD3D5FB02D5FB12A5FB2125FB30E5FBF
:20035300B52A61D2045EA3835EBD2D5EBD3D5EBD355EBD3D5EBD395EBD3D5EBD3C61FF0441
:200373005EA3705EBD2C5EBD245EBD2061FF045EA38361D3045EA39561FF045EA3835EB587
:200393000A5FB50A61D3045EB00D5EB0295EB10A5EB12A5EB3125EB52A5EBD305E71F85E76
:2003B30091CA5EBD315FB00D5FB0295FB10A5FB12A5FB52A61FF045EBD215EBD2061D2048B
:2003D3005EB50A5FB50A61FF045EB0095EB10A5FB0095FB10A61D10E5EA0665EB02E5EA12A
:2003F300985EB12D5EA5985EB52D5EBD305EBD385EBD3C5E71985E91065EBD3D5FA0665FCE
:20041300B02E5FA1985FB12D5FA5965FB52D61D3045EBD355EBD315EBD3061D1095EBD20A6
:2004330061D2095EB50D5FB50D61FF045EB00E5EA0985EB0295EB10D5EA1225EB12A5EA566
:20045300225EB52A5EBD305E71F85E91CA5EBD315FB00E5FA0985FB0295FB10D5FA1225F89
:20047300B12A5FA51F5FB52A61D3045EBD215EBD2061FF045EB50A5FB50A61FF045EB00964
:200493005EB10A5FB0095FB10A61A40E5EA08A5EB02E5EA1B15EB12D5EA5B15EB52D5EBD2C
:2004B300305EBD385EBD3C5E71985E91065EBD3D5FA08A5FB02E5FA1B15FB12D5FA5AE5FD6
:2004D300B52D61FF045EBD355EBD315EBD3061D2095EBD2061D1095EB50D5FB50D61FF0485
:2004F3005EB00E5EA0985EB0295EB10D5EA1225EB12A5EA5225EB52A5EBD305E71F85E9127
:20051300CA5EBD315FB00E5FA0985FB0295FB10D5FA1225FB12A5FA51F5FB52A61D3045E56
:20053300BD215EBD2061FF045EB50A5FB50A61D3045EB0095EB10A5FB0095FB10A61D00E17
:200553005EA0225EB02E5EA16C5EB12D5EA56C5EB52D5EBD305EBD385EBD3C5E71985E918B
:20057300065EBD3D5FA0225FB02E5FA16C5FB12D5FA5695FB52D61FF045EBD355EBD315EF7
:20059300BD3061D2095EBD2061D2095EB50D5FB50D61D3045EB00E5EA0985EB0295EB10D2A
:2005B3005EA1225EB12A5EA5225EB52A5EBD305E71F85E91CA5EBD315FB00E5FA0985FB092
:2005D300295FB10D5FA1225FB12A5FA51F5FB52A61FE045EBD215EBD2061D3045EB50A5F77
:2005F300B50A61FF045EB0095EB10A5FB0095FB10A61D10E5EA0665EB02E5EA1985EB12DB0
:200613005EA5985EB52D5EBD305EBD385EBD3C5E71985E91065EBD3D5FA0665FB02E5FA1A1
:20063300985FB12D5FA5965FB52D61D3045EBD355EBD315EBD3061D1095EBD2061FE095E9C
:20065300B50D5FB50D61D3045EB00E5EA0985EB0295EB10D5EA1225EB12A5EA5225EB52AAB
:200673005EBD305E71F85E91CA5EBD315FB00E5FA0985FB0295FB10D5FA1225FB12A5FA5E7
:200693001F5FB52A61FF045EBD215EBD2061D3045EB50A5FB50A61FE045EB0095EB10A5FAA
:2006B300B0095FB10A61A50E5EA0E65EB02D5EA18A5EB12A5EA58A5EB52A5EBD305EBD38F7
:2006D3005EBD3C5E71985E91065EBD3D5FA0E65FB02D5FA18A5FB12A5FA5865FB52A61FFEF
:2006F300045EBD355EBD315EBD3061D2095EBD2061D1095EB50A5FB50A61FF045EB00D5E32
:20071300A0985EB0295EB10A5EA1225EB12A5EA5225EB52A5EBD305E71F85E91CA5EBD316B
:200733005FB00D5FA0985FB0295FB10A5FA1225FB12A5FA51F5FB52A61D3045EBD215EBD55
:200753002061FF045EB50A5FB50A61FF045EB0095EB10A5FB0095FB10A61A40E5EA0225E70
:20077300B02E5EA16C5EB12D5EA56C5EB52D5EBD305EBD385EBD3C5E71985E91065EBD3D89
:200793005FA0225FB02E5FA16C5FB12D5FA5695FB52D61FF045EBD355EBD315EBD3061D213
:2007B300095EBD2061D2095EB50D5FB50D61FE045EB00E5EA0985EB0295EB10D5EA1225E7E
:2007D300B12A5EA5225EB52A5EBD305E71F85E91CA5EBD315FB00E5FA0985FB0295FB10DA9
:2007F3005FA1225FB12A5FA51F5FB52A61D3045EBD215EBD2061FF045EB50A5FB50A61D3A7
:20081300045EB0095EB10A5FB0095FB10A61D10E5EA0CB5EB02D5EA1665EB12A5EA5665EB6
:20083300B52A5EBD305EBD385EBD3C5E71985E91065EBD3D5FA0CB5FB02D5FA1665FB12A77
:200853005FA5625FB52A61D2045EBD355EBD315EBD3061FE095EBD2061D2095EB50A5FB5B3
:200873000A61D3045EB00D5EA0985EB0295EB10A5EA1225EB12A5EA5225EB52A5EBD305EBD
:2008930071F85E91CA5EBD315FB00D5FA0985FB0295FB10A5FA1225FB12A5FA51F5FB52A15
:2008B30061FF045EBD215EBD2061D2045EB50A5FB50A61FF045EB0095EB10A5FB0095FB11C
:2008D3000A61D10E5EB02D5EB12A5EB52A5EBD305EBD385EBD3C5E71985E91065EBD3D5F02
:2008F300B02D5FB12A5FB52A61D3045EBD2D5EBD3D5EBD355EBD3D5EBD395EBD3D5EBD3C0D
:2009130061FF045EBD2C5EBD245EBD2061A40E5EB50A5FB50A61FF045EB00D5EB0295EB18C
:200933000A5EB12A5EB52A5EBD305E71F85E91CA5EBD315FB00D5FB0295FB10A5FB12A5F06
:20095300B52A61FF045EBD215EBD2061D3045EB50A5FB50A61FF045EB0095EB10A5FB009AB
:200973005FB10A61A40E5EA0665EB02E5EA1985EB12D5EA5985EB52D5EBD305EBD385EBD30
:200993003C5E71985E91065EBD3D5FA0665FB02E5FA1985FB12D5FA5965FB52D61FF045E40
:2009B300BD355EBD315EBD3061D2095EBD2061D1095EB50D5FB50D61FF045EB00E5EA09892
:2009D3005EB0295EB10D5EA1225EB12A5EA5225EB52A5EBD305E71F85E91CA5EBD315FB0CF
:2009F3000E5FA0985FB0295FB10D5FA1225FB12A5FA51F5FB52A61D3045EBD215EBD20611D
:200A1300FF045EB50A5FB50A61D3045EB0095EB10A5FB0095FB10A61D00E5EA08A5EB02EE8
:200A33005EA1B15EB12D5EA5B15EB52D5EBD305EBD385EBD3C5E71985E91065EBD3D5FA01B
:200A53008A5FB02E5FA1B15FB12D5FA5AE5FB52D61FF045EBD355EBD315EBD3061D2095EF6
:200A7300BD2061D2095EB50D5FB50D61D2045EB00E5EA0985EB0295EB10D5EA1225EB12A73
:200A93005EA5225EB52A5EBD305E71F85E91CA5EBD315FB00E5FA0985FB0295FB10D5FA1C1
:200AB300225FB12A5FA51F5FB52A61FF045EBD215EBD2061FF045EB50A5FB50A61D3045E56
:200AD300B0095EB10A5FB0095FB10A61D10E5EA0225EB02E5EA16C5EB12D5EA56C5EB52D0D
:200AF3005EBD305EBD385EBD3C5E71985E91065EBD3D5FA0225FB02E5FA16C5FB12D5FA52F
:200B1300695FB52D61D2045EBD355EBD315EBD3061FE095EBD2061D2095EB50D5FB50D6179
:200B3300D3045EB00E5EA0985EB0295EB10D5EA1225EB12A5EA5225EB52A5EBD305E71F8F8
:200B53005E91CA5EBD315FB00E5FA0985FB0295FB10D5FA1225FB12A5FA51F5FB52A61FF57
:200B7300045EBD215EBD2061D2045EB50A5FB50A61FF045EB0095EB10A5FB0095FB10A614E
:200B9300D10E5EA0665EB02E5EA1985EB12D5EA5985EB52D5EBD305EBD385EBD3C5E7198B9
:200BB3005E91065EBD3D5FA0665FB02E5FA1985FB12D5FA5965FB52D61D3045EBD355EBDE0
:200BD300315EBD3061D1095EBD2061D2095EB50D5FB50D61FF045EB00E5EA0985EB0295EE8
:200BF300B10D5EA1225EB12A5EA5225EB52A5EBD305E71F85E91CA5EBD315FB00E5FA0989D
:200C13005FB0295FB10D5FA1225FB12A5FA51F5FB52A61D3045EBD215EBD2061FF045EB589
:200C33000A5FB50A61FF045EB0095EB10A5FB0095FB10A61A40E5EA0E65EB02D5EA18A5E9A
:200C5300B12A5EA58A5EB52A5EBD305EBD385EBD3C5E71985E91065EBD3D5FA0E65FB02D12
:200C73005FA18A5FB12A5FA5865FB52A61FF045EBD355EBD315EBD3061D2095EBD2061D1E1
:200C9300095EB50A5FB50A61FF045EB00D5EA0985EB0295EB10A5EA1225EB12A5EA5225EBB
:200CB300B52A5EBD305E71F85E91CA5EBD315FB00D5FA0985FB0295FB10A5FA1225FB12ACA
:200CD3005FA51F5FB52A61D3045EBD215EBD2061FF045EB50A5FB50A61D3045EB0095EB1F4
:200CF3000A5FB0095FB10A61D00E5EA0225EB02E5EA16C5EB12D5EA56C5EB52D5EBD305E0B
:200D1300BD385EBD3C5E71985E91065EBD3D5FA0225FB02E5FA16C5FB12D5FA5695FB52D0B
:200D330061FF045EBD355EBD315EBD3061D2095EBD2061D2095EB50D5FB50D61D3045EB01B
:200D53000E5EA0985EB0295EB10D5EA1225EB12A5EA5225EB52A5EBD305E71F85E91CA5EA4
:200D7300BD315FB00E5FA0985FB0295FB10D5FA1225FB12A5FA51F5FB52A61FE045EBD210D
:200D93005EBD2061D3045EB50A5FB50A61FF045EB0095EB10A5FB0095FB10A61D10E5EA08E
:200DB300CB5EB02D5EA1665EB12A5EA5665EB52A5EBD305EBD385EBD3C5E71985E91065E27
:200DD300BD3D5FA0CB5FB02D5FA1665FB12A5FA5625FB52A61D3045EBD355EBD315EBD309D
:200DF30061D1095EBD2061FE095EB10A5EB50A5FB10A5FB50A61D3045EB00D5EA0985EB09D
:200E1300295EA1225EB12A5EA5225EB52A5EBD305E71F85E91CA5EBD315FB00D5FA0985FB1
:200E3300B0295FA1225FB12A5FA51F5FB52A61FF045EBD215EBD2061D3045EB50A5FB50ABB
:200E530061FE045EB0095EB10A5FB0095FB10A61A50E5EB02D5EB12A5EB52A5EBD305EBD8F
:200E7300385EBD3C5E71985E91065EBD3D5FB02D5FB12A5FB52A61FF045EBD355EBD3D5EFE
:200E9300BD395EBD3D5EBD3C61FF045EBD345EBD3061D3045EBD2061D1095EB50A5FB50AB3
:200EB30061FF045EB00D5EB0295EB10A5EB12A5EB52A5EBD305E71F85E91CA5EBD315FB0B4
:200ED3000D5FB0295FB10A5FB12A5FB52A61D3045EBD215EBD2061FF045EB50A5FB50A6179
:200EF300FF045EB0095EB10A5FB0095FB10A61A40E5EA0665EB02E5EA1985EB12D5EA59859
:200F13005EB52D5EBD305EBD385EBD3C5E71985E91065EBD3D5FA0665FB02E5FA1985FB18B
:200F33002D5FA5965FB52D61FF045EBD355EBD315EBD3061D2095EBD2061D2095EB50D5F19
:200F5300B50D61FE045EB00E5EA0985EB0295EB10D5EA1225EB12A5EA5225EB52A5EBD304D
:200F73005E71F85E91CA5EBD315FB00E5FA0985FB0295FB10D5FA1225FB12A5FA51F5FB5F6
:200F93002A61D3045EBD215EBD2061FF045EB50A5FB50A61D3045EB0095EB10A5FB0095FE7
:200FB300B10A61D10E5EA08A5EB02E5EA1B15EB12D5EA5B15EB52D5EBD305EBD385EBD3C8A
:200FD3005E71985E91065EBD3D5FA08A5FB02E5FA1B15FB12D5FA5AE5FB52D61D2045EBD51
:200FF300355EBD315EBD3061FE095EBD2061D2095EB50D5FB50D61D3045EB00E5EA0985EAA
:20101300B0295EB10D5EA1225EB12A5EA5225EB52A5EBD305E71F85E91CA5EBD315FB00ED8
:201033005FA0985FB0295FB10D5FA1225FB12A5FA51F5FB52A61FF045EBD215EBD2061D2E6
:20105300045EB50A5FB50A61FF045EB0095EB10A5FB0095FB10A61D10E5EA0225EB02E5E7E
:20107300A16C5EB12D5EA56C5EB52D5EBD305EBD385EBD3C5E71985E91065EBD3D5FA0229B
:201093005FB02E5FA16C5FB12D5FA5695FB52D61D3045EBD355EBD315EBD3061D1095EBD34
:2010B3002061D2095EB50D5FB50D61FF045EB00E5EA0985EB0295EB10D5EA1225EB12A5E5F
:2010D300A5225EB52A5EBD305E71F85E91CA5EBD315FB00E5FA0985FB0295FB10D5FA122B7
:2010F3005FB12A5FA51F5FB52A61FF045EBD215EBD2061D3045EB50A5FB50A61FF045EB082
:20111300095EB10A5FB0095FB10A61A40E5EA0225EB02E5EA1985EB12D5EB52A5EBD305E40
:20113300BD385EBD3C5EC8215EBD3E5FA0225FB02E5FA1985FB12D5FB52A61FF045EBD2E92
:201153005EBD3E5EBD365EBD3E5EBD3A5EBD3E5EBD3C61D3045EBD345EBD3061FE095EBD1F
:201173002061D2045EB50A5FB50A61FF045EB00E5EB10D5EBD305EBD315FB00E5FB10D61FC
:20119300D3045EBD215EBD2061A2185EBD305EBD3161FF045EBD215EBD206176185EB02E36
:2011B3005EB12D5EB52A5EBD305EBD385EBD3C5EC8115EBD3E5FB02E5FB12D5FB52A61FF06
:2011D300045EBD365EBD325EBD3061D2095EBD2061D10E5EC6285E30325E50445E70F85E36
:2011F300C62E5E33115E937F5EB60D5EBD305E34325E54495E74F85E94FF5EF4005EBD384B
:201213005EBD3C5E71985E91065EBD3D61D2045EBD3C61FE095EBD3461A50E5EA2865EA2D1
:201233001F5EB2325E29215E49145E89AE5EC43A5EE9005E2C315E6CF05E8CFC5EEC015E9B
:201253004C0B5EB4325EBD245EC63E5EA6435EB60A5EBD345EBD3C5EBD385EBD3C5FA292F7
:201273005FA2295FB2325FA3195FB32E61FF045EA2225EA4255FA22C5FA31C61D2045EA264
:20129300255EA4295FA22F5FA31F61FF045EA2225EA4255EBD345FA22C5FA31C61D3045EBD
:2012B300A21F5EA4225FA2295FA31961FF045EA2225EA4255FA22C5FA31C61FF045EB21273
:2012D3005EA2255EA2695EB2325E4B105EA31C5EB3325EB4125EA4295EA46D5EB4325EBDF5
:2012F300245EC61E5EA6B15EB6095EBD345EBD3C5EBD385EBD3C5FB2125FA22F5FA2745F2C
:20131300B2325FB30E5FA31F5FA3625FB32E61D3045EA2665EA31F5EA4695FA2705FA35FF6
:2013330061FF045EA2625EA3225EA4665FA26D5FA35B61D2045EA2665EA31F5EA4695EBD3B
:20135300345FA2705FA35F61FF045EA2695EA31C5EA46D5FA2745FA36261D3045EA2665E46
:20137300A31F5EA4695FA2705FA35F61FF045EB2125EA2625EA2865EB2325EB3125EA32265
:201393005EA3665EB3325EB4125EA4665EA48A5EB4325EBD245EC63E5E30005E50075E7082
:2013B300D85EC6385E33005E93F05EA6575EBD345EBD305FB2125FA26D5FA2925FB2325FB9
:2013D300B30E5FA35B5FA37F5FB32E61D3045EA28A5EA3625EA48D5EBD205FA2955FA38311
:2013F30061FF045EA28D5EA35F5EA4925FA29A5FA38661FF045EA28A5EA3625EA48D5FA2F1
:20141300955FA38361D2045EA2865EA3665EA48A5FA2925FA37F61FF045EA28A5EA3625E2C
:20143300A48D5EB50A5FA2955FA3835FB50A61D3045EB00E5EB02E5EB10D5EB12D5EB21208
:201453005EA28D5EA2255EB2325EB3125EA35F5EA3835EB3325EB4125EA4925EA4295EB446
:20147300325EB52A5EBD305EC8215EBD325FB00E5FB02E5FB10D5FB12D5FB2125FA29A5F3A
:20149300A22F5FB2325FB30E5FA3865FA31F5FB32E5FB52A61FF045EA2225EA3865EA425AA
:2014B3005EBD225EBD205FA22C5FA31C61D3045EA21F5EA38A5EA4225FA2295FA31961FFAB
:2014D300045EA2225EA3865EA4255FA22C5FA31C61FF045EA2255EA3835EA4295FA22F5F13
:2014F300A31F61D2045EA2225EA3865EA4255EB50A5FA22C5FA31C5FB50A61FF045EB00E0A
:201513005EB02A5EB10D5EB1295EA21F5EB3125EA38A5EA3225EB3325EA4225EB52A5E71C9
:20153300F85E91CA5EBD215FB00E5FB02A5FB10D5FB1295FA2295FA3195FB52A61D3045EE6
:20155300A2225EA31F5EA4255EBD205FA22C5FA31C61FF045EA2255EA31C5EA4295FA22FE6
:201573005FA31F61D3045EB00A5EB1095EA2225EA31F5EA4255FB00A5FB1095FA22C5FA305
:201593001C61FF045EA21F5EA3225EA4225FA2295FA31961D3045EA2225EA31F5EA4255E0E
:2015B300B50A5FA22C5FA31C5FB50A61FE045EB02A5EB1295EA2255EA31C5EA4295EB52A73
:2015D3005EBD305E341E5E54055E74F55E94D75EF4025EBD385EBD3C5EBD3D5FB02A5FB117
:2015F300295FA22F5FA31F5FB52A61FF045EA2225EA31F5EA4255EBD355EBD315EBD305F0D
:20161300A22C5FA31C61D3045EA21F5EA3225EA4225FA2295FA31961FF045EB00A5EB10954
:201633005EA2225EA31F5EA4255EBD205FB00A5FB1095FA22C5FA31C61D3045EA2255EA318
:201653001C5EA4295FA22F5FA31F61FF045EA2225EA31F5EA4255EB50A5FA22C5FA31C5F4B
:20167300B50A61D3045EB02E5EB12D5EB2125EA21F5EA2625EB2325EA3225EB4125EA42298
:201693005EA4665EB4325EB52A5EBD305EBD315FB02E5FB12D5FB2125FA2295FA26D5FB271
:2016B300325FB30E5FA3195FA35B5FB32E5FB52A61FE045EA2665EA31F5EA4695EBD215EE1
:2016D300BD205FA2705FA35F61D3045EA2695EA31C5EA46D5FA2745FA36261FF045EA26678
:2016F3005EA31F5EA4695FA2705FA35F61FF045EA2625EA3225EA4665FA26D5FA35B61D32A
:20171300045EA2665EA31F5EA4695EB50A5FA2705FA35F5FB50A61FF045EB00E5EB02A5E9E
:20173300B10D5EB1295EA2695EB3125EA31C5EA35F5EB3325EA46D5EB52A5EBD215FB00E4F
:201753005FB02A5FB10D5FB1295FA2745FA3625FB52A61D3045EA2665EA3625EA4695EBD49
:20177300205FA2705FA35F61FE045EA2625EA3665EA4665FA26D5FA35B61D3045EB00A5E57
:20179300B1095EA2665EA3625EA4695FB00A5FB1095FA2705FA35F61FF045EA2695EA35F17
:2017B3005EA46D5FA2745FA36261FF045EA2665EA3625EA4695EB50A5FA2705FA35F5FB533
:2017D3000A61D3045EB02A5EB1295EA2625EA3665EA4665EB52A5EBD305EBD315FB02A5FA7
:2017F300B1295FA26D5FA35B5FB52A61FF045EA2665EA3625EA4695EBD215EBD205FA27073
:201813005FA35F61D3045EA2695EA35F5EA46D5FA2745FA36261FE045EB00A5EB1095EA278
:20183300665EA3625EA4695FB00A5FB1095FA2705FA35F61D3045EA2625EA3665EA4665F95
:20185300A26D5FA35B61FF045EA2665EA3625EA4695EB50A5FA2705FA35F5FB50A61D3042C
:201873005EB02E5EB12D5EB2125EA2695EA28D5EB2325EA35F5EB4125EA46D5EA4925EB4EA
:20189300325EB52A5EBD305EBD385EBD3C5EBD3D5FB02E5FB12D5FB2125FA2745FA29A5F6D
:2018B300B2325FB30E5FA3625FA3865FB32E5FB52A61FF045EA28A5EA3625EA48D5EBD3577
:2018D3005EBD315EBD305FA2955FA38361FF045EA2865EA3665EA48A5FA2925FA37F61D31E
:2018F300045EA28A5EA3625EA48D5EBD205FA2955FA38361FE045EA28D5EA35F5EA4925FBC
:20191300A29A5FA38661D3045EA28A5EA3625EA48D5EB50A5FA2955FA3835FB50A61FF0482
:201933005EB00E5EB02A5EB10D5EB1295EA2865EB3125EA3665EA38A5EB3325EA48A5EB56F
:201953002A5EBD215FB00E5FB02A5FB10D5FB1295FA2925FA37F5FB52A61D3045EA28A5EF0
:20197300A3865EA48D5EBD205FA2955FA38361FF045EA28D5EA3835EA4925FA29A5FA3861A
:2019930061FF045EB00A5EB1095EA28A5EA3865EA48D5FB00A5FB1095FA2955FA38361D37F
:2019B300045EA2865EA38A5EA48A5FA2925FA37F61FE045EA28A5EA3865EA48D5EB50A5FE0
:2019D300A2955FA3835FB50A61D3045EB02A5EB1295EA2835EA3835EA4865EB52A5EBD305B
:2019F3005EBD315FB02A5FB1295FA28D5FA37C5FB52A61FF045EA28A5EA3865EA48D5EBDAD
:201A1300215EBD205FA2955FA38361D3045EA2925EA38A5EA4955FA29D5FA38A61FF045E64
:201A3300B00A5EB1095EA28A5EA3865EA48D5FB00A5FB1095FA2955FA38361D3045EA28319
:201A53005EA3835EA4865FA28D5FA37C61FF045EA28A5EA3865EA48D5EB50A5FA2955FA3A2
:201A7300835FB50A61FE045EB02E5EB12D5EA2925EA37F5EA4955EB52A5EBD305EBD315FFB
:201A9300B02E5FB12D5FA29D5FA38A5FB52A61D3045EA28A5EA3865EA48D5EBD215EBD2061
:201AB3005FA2955FA38361FF045EA2835EA38D5EA4865FA28D5FA37C61D3045EA28A5EA32C
:201AD300865EA48D5FA2955FA38361FF045EA2925EA37F5EA4955FA29D5FA38A61D3045EF6
:201AF300A28A5EA3865EA48D5EB50A5FA2955FA3835FB50A61FF045EB00E5EB02A5EB10D67
:201B13005EB1295EA27F5EA38D5EA4835EB52A5EBD305EBD385EBD3C5EBD3D5FB00E5FB032
:201B33002A5FB10D5FB1295FA28A5FA3775FB52A61D2045EA28A5EA3865EA48D5EBD355E4B
:201B5300BD315EBD305FA2955FA38361FF045EA2955EA37F5EA49A5FA2A25FA38D61FF0473
:201B73005EB00A5EB1095EA28A5EA3865EA48D5EBD205FB00A5FB1095FA2955FA38361D3C6
:201B9300045EA27F5EA38D5EA4835FA28A5FA37761FF045EA28A5EA3865EA48D5EB50A5F18
:201BB300A2955FA3835FB50A61D3045EB02A5EB1295EA2955EA37C5EA49A5EB52A5EBD305A
:201BD3005EBD315FB02A5FB1295FA2A25FA38D5FB52A61FF045EA28A5EA3865EA48D5EBDA5
:201BF300215EBD205FA2955FA38361D2045EA27F5EA3925EA4835FA28A5FA37761FF045EC7
:201C1300B00A5EB1095EA28A5EA3865EA48D5FB00A5FB1095FA2955FA38361FF045EA295F9
:201C33005EA37C5EA49A5FA2A25FA38D61D3045EA28A5EA3865EA48D5EB50A5FA2955FA3B9
:201C5300835FB50A61FF045EB02E5EB12D5EA27C5EA3925EA47F5EA5985EB52D5EBD215FEE
:201C7300B02E5FB12D5FA2865FA3745FA5965FB52D61D3045EA28A5EA3865EA48D5EBD204B
:201C93005FA2955FA38361FF045EA29A5EA37C5EA49D5FA2A55FA39261D2045EA28A5EA300
:201CB300865EA48D5FA2955FA38361FF045EA27C5EA3925EA47F5FA2865FA37461D3045E5A
:201CD300A28A5EA3865EA48D5EB50D5FA2955FA3835FB50D61FF045EB00E5EB02A5EB10D7F
:201CF3005EB1295EA29A5EA3775EA49D5EA5225EB52A5EBD305EBD315FB00E5FB02A5FB189
:201D13000D5FB1295FA2A55FA3925FA51F5FB52A61FF045EA28A5EA3865EA48D5EBD215E31
:201D3300BD205FA2955FA38361D3045EA27C5EA3955EA47F5FA2865FA37461FF045EB00A54
:201D53005EB1095EA28A5EA3865EA48D5FB00A5FB1095FA2955FA38361D2045EA29A5EA399
:201D7300775EA49D5FA2A55FA39261FF045EA28A5EA3865EA48D5EB50A5FA2955FA3835F65
:201D9300B50A61D3045EA0E65EB02D5EA16C5EB12D5EB2125EA28D5EA2695EB2325EA39583
:201DB3005EB4125EA4925EA46D5EB4325EA58A5EB52A5EBD305EBD385EBD3C5EBD3D5FA08F
:201DD300E65FB02D5FA16C5FB12D5FB2125FA29A5FA2745FB2325FB30E5FA3865FA3625F44
:201DF300B32E5FA5865FB52A61FF045EA2665EA3865EA4695EBD355EBD315EBD305FA27013
:201E13005FA35F61D3045EA2625EA3775EA4665FA26D5FA35B61FF045EA2665EA3865EA4B6
:201E3300695EBD205FA2705FA35F61FF045EA2695EA3955EA46D5FA2745FA36261D2045ED9
:201E5300A2665EA3865EA4695EB50A5FA2705FA35F5FB50A61FF045EB00D5EA0225EB02E8D
:201E73005EB10D5EA1985EB12D5EB2125EA2625EA2865EB2325EB3125EA38A5EA3665EB3EE
:201E9300325EB4125EA4665EA48A5EB4325EA5225EB52A5EBD305E71985E91065EBD315FED
:201EB300B00D5FA0225FB02E5FB10D5FA1985FB12D5FB2125FA26D5FA2925FB2325FB30E7B
:201ED3005FA35B5FA37F5FB32E5FA51F5FB52A61D3045EA28A5EA3625EA48D5EBD215EBD65
:201EF300205FA2955FA38361FF045EA28D5EA35F5EA4925FA29A5FA38661D3045EA28A5E6C
:201F1300A3625EA48D5FA2955FA38361FF045EA2865EA3665EA48A5FA2925FA37F61FF04AA
:201F33005EA28A5EA3625EA48D5EB50A5FA2955FA3835FB50A61D2045EB00E5EA0E65EB077
:201F53002D5EB10D5EA16C5EB12D5EB2125EA28D5EA2695EB2325EB3125EA35F5EA3835EBF
:201F7300B3325EB4125EA4925EA46D5EB4325EA5E65EB5295EBD305FB00E5FA0E65FB02D50
:201F93005FB10D5FA16C5FB12D5FB2125FA29A5FA2745FB2325FB30E5FA3865FA3625FB3D4
:201FB3002E5FA5E35FB52961FF045EA2665EA3865EA4695EBD205FA2705FA35F61D3045E5D
:201FD300A2625EA38A5EA4665FA26D5FA35B61FF045EA2665EA3865EA4695FA2705FA35F9E
:201FF30061D3045EA2695EA3835EA46D5FA2745FA36261FF045EA2665EA3865EA4695EB592
:20201300095FA2705FA35F5FB50961D2045EB00D5EB0295EB10D5EB1295EA2625EB3125EF5
:20203300A38A5EA3665EB3325EA4665EB5295E71F85E91CA5EBD215FB00D5FB0295FB10DE5
:202053005FB1295FA26D5FA35B5FB52961FF045EA2665EA3625EA4695EBD205FA2705FA3E6
:202073005F61FF045EA2695EA35F5EA46D5FA2745FA36261D3045EB0095EB1095EA2665E4E
:20209300A3625EA4695FB0095FB1095FA2705FA35F61FF045EA2625EA3665EA4665FA26DB7
:2020B3005FA35B61D3045EA2665EA3625EA4695EB5095FA2705FA35F5FB50961FF045EB0C7
:2020D300295EB1295EA2695EA35F5EA46D5EB5295EBD305EBD385EBD3C5EBD3D5FB0295F34
:2020F300B1295FA2745FA3625FB52961D2045EA2665EA3625EA4695EBD355EBD315EBD308B
:202113005FA2705FA35F61FF045EA2625EA3665EA4665FA26D5FA35B61FF045EB0095EB1F0
:20213300095EA2665EA3625EA4695EBD205FB0095FB1095FA2705FA35F61D3045EA2695E12
:20215300A35F5EA46D5FA2745FA36261FF045EA2665EA3625EA4695EB5095FA2705FA35F9C
:202173005FB50961D3045EB02D5EB12D5EB2125EA2625EA21F5EB2325EA3665EB4125EA40E
:20219300665EA4225EB4325EB5295EBD305EBD315FB02D5FB12D5FB2125FA26D5FA2295FF8
:2021B300B2325FB30E5FA35B5FA3195FB32E5FB52961FF045EA2225EA3625EA4255EBD21C7
:2021D3005EBD205FA22C5FA31C61D2045EA2255EA35F5EA4295FA22F5FA31F61FF045EA2CA
:2021F300225EA3625EA4255FA22C5FA31C61D3045EA21F5EA3665EA4225FA2295FA319614D
:20221300FF045EA2225EA3625EA4255EB5095FA22C5FA31C5FB50961FF045EB00D5EB029C2
:202233005EB10D5EB1295EA2255EB3125EA35F5EA31C5EB3325EA4295EB5295EBD215FB07D
:202253000D5FB0295FB10D5FB1295FA22F5FA31F5FB52961D3045EA2225EA31F5EA4255E43
:20227300BD205FA22C5FA31C61FF045EA21F5EA3225EA4225FA2295FA31961D2045EB009C6
:202293005EB1095EA2225EA31F5EA4255FB0095FB1095FA22C5FA31C61FF045EA2255EA3A4
:2022B3001C5EA4295FA22F5FA31F61D3045EA2225EA31F5EA4255EB5095FA22C5FA31C5F0C
:2022D300B50961FF045EB0295EB1295EA21F5EA3225EA4225EB5295EBD305EBD315FB029E9
:2022F3005FB1295FA2295FA3195FB52961D3045EA2225EA31F5EA4255EBD215EBD205FA2F7
:202313002C5FA31C61FF045EA2255EA31C5EA4295FA22F5FA31F61FF045EB0095EB1095E4D
:20233300A2225EA31F5EA4255FB0095FB1095FA22C5FA31C61D2045EA21F5EA3225EA42266
:202353005FA2295FA31961FF045EA2225EA31F5EA4255EB5095FA22C5FA31C5FB50961D3A0
:20237300045EB02D5EB12D5EB2125EA2255EA2E95EB2315EA31C5EB4125EA4295EA4EC5EA6
:20239300B4315EB5295EBD305EBD385EBD3C5EBD3D5FB02D5FB12D5FB2125FA22F5FA2F2FD
:2023B3005FB2315FB30E5FA31F5FA3E35FB32D5FB52961FF045EA2E65EA31F5EA4E95EBDB6
:2023D300355EBD315EBD305FA2EF5FA3E161D3045EA2E35EA3225EA4E65FA2EC5FA3DE61F7
:2023F300FF045EA2E65EA31F5EA4E95EBD205FA2EF5FA3E161FF045EA2E95EA31C5EA4EC70
:202413005FA2F25FA3E361D2045EA2E65EA31F5EA4E95EB5095FA2EF5FA3E15FB50961FF3D
:20243300045EB00D5EB0295EB10D5EB1295EA2E35EB3125EA3225EA3E65EB3315EA4E65E47
:20245300B5295EBD215FB00D5FB0295FB10D5FB1295FA2EC5FA3DE5FB52961D3045EA2E67D
:202473005EA3E35EA4E95EBD205FA2EF5FA3E161FF045EA2E95EA3E15EA4EC5FA2F25FA35A
:20249300E361D3045EB0095EB1095EA2E65EA3E35EA4E95FB0095FB1095FA2EF5FA3E161C5
:2024B300FF045EA2E35EA3E65EA4E65FA2EC5FA3DE61D3045EA2E65EA3E35EA4E95EB5097E
:2024D3005FA2EF5FA3E15FB50961FE045EB0295EB1295EA2E15EA3E15EA4E35EB5295EBD28
:2024F300305EBD315FB0295FB1295FA2E95FA3DB5FB52961FF045EA2E65EA3E35EA4E95E61
:20251300BD215EBD205FA2EF5FA3E161D3045EA2EC5EA3E65EA4EF5FA2F45FA3E661FF047F
:202533005EB0095EB1095EA2E65EA3E35EA4E95FB0095FB1095FA2EF5FA3E161D3045EA268
:20255300E15EA3E15EA4E35FA2E95FA3DB61FF045EA2E65EA3E35EA4E95EB5095FA2EF5F75
:20257300A3E15FB50961D3045EB02D5EB12D5EA2EC5EA3DE5EA4EF5EB5295EBD305EBD3169
:202593005FB02D5FB12D5FA2F45FA3E65FB52961FE045EA2E65EA3E35EA4E95EBD215EBD26
:2025B300205FA2EF5FA3E161D3045EA2E15EA3E95EA4E35FA2E95FA3DB61FF045EA2E65EBE
:2025D300A3E35EA4E95FA2EF5FA3E161FF045EA2EC5EA3DE5EA4EF5FA2F45FA3E661D3046F
:2025F3005EA2E65EA3E35EA4E95EB5095FA2EF5FA3E15FB50961FF045EB00D5EB0295EB142
:202613000D5EB1295EA2DE5EA3E95EA4E15EB5295EBD305EBD385EBD3C5EBD3D5FB00D5FB3
:20263300B0295FB10D5FB1295FA2E65FA3D85FB52961D3045EA2E65EA3E35EA4E95EBD351D
:202653005EBD315EBD305FA2EF5FA3E161FE045EA2EF5EA3DE5EA4F25FA2F85FA3E961D3C0
:20267300045EB0095EB1095EA2E65EA3E35EA4E95EBD205FB0095FB1095FA2EF5FA3E161BF
:20269300FF045EA2DE5EA3E95EA4E15FA2E65FA3D861FF045EA2E65EA3E35EA4E95EB50983
:2026B3005FA2EF5FA3E15FB50961D3045EB0295EB1295EA2EF5EA3DB5EA4F25EB5295EBD5A
:2026D300305EBD315FB0295FB1295FA2F85FA3E95FB52961FF045EA2E65EA3E35EA4E95E62
:2026F300BD215EBD205FA2EF5FA3E161D3045EA2DE5EA3EC5EA4E15FA2E65FA3D861FE04D1
:202713005EB0095EB1095EA2E65EA3E35EA4E95FB0095FB1095FA2EF5FA3E161D3045EA286
:20273300EF5EA3DB5EA4F25FA2F85FA3E961FF045EA2E65EA3E35EA4E95EB5095FA2EF5F5F
:20275300A3E15FB50961D3045EB02D5EB12D5EB2115EA2E95EA3EC5EB4115EA4EC5EA56C9F
:202773005EB52D5EBD215FB02D5FB12D5FB2115FA2F25FB30D5FA3E35FA5695FB52D61FF2A
:20279300045EA2E65EA3E35EA4E95EBD205FA2EF5FA3E161FF045EA2E35EA3DB5EA4E65FF5
:2027B300A2EC5FA3DE61D3045EA2E65EA3E35EA4E95FA2EF5FA3E161FE045EA2E95EA3EC9F
:2027D3005EA4EC5FA2F25FA3E361D3045EA2E65EA3E35EA4E95EB50D5FA2EF5FA3E15FB52C
:2027F3000D61FF045EB00D5EB0295EB10D5EB1295EA2E35EB2315EB3115EA3E65EA4E65E3C
:20281300B4315EA5E65EB5295EBD305EBD315FB00D5FB0295FB10D5FB1295FA2EC5FB2312B
:202833005FA3DE5FB32D5FA5E35FB52961D3045EA2E65EA3E35EA4E95EBD215EBD205FA2DD
:20285300EF5FA3E161FF045EA2E95EA3E15EA4EC5FA2F25FA3E361FF045EB0095EB1095EAD
:20287300A2E65EA3E35EA4E95FB0095FB1095FA2EF5FA3E161D3045EA2E35EA3E65EA4E600
:202893005FA2EC5FA3DE61FE045EA2E65EA3E35EA4E95EB5095FA2EF5FA3E15FB50961D300
:2028B300045EA0B15EB02D5EA18A5EB12A5EB2115EA2E95EA2255EB2325EA3E15EB3315E62
:2028D300B4115EA4EC5EA4295EB4325EA5225EB52A5EBD305EBD385EBD3C5EBD3D5FA0B164
:2028F3005FB02D5FA18A5FB12A5FB2115FA2F25FA22F5FB2325FB30D5FA3E35FA31F5FB306
:202913002E5FA51F5FB52A61FF045EA2225EA3E35EA4255EBD355EBD315EBD305FA22C5F11
:20293300A31C61D3045EA21F5EA3E65EA4225FA2295FA31961FF045EA2225EA3E35EA4258D
:202953005EBD205FA22C5FA31C61D3045EA2255EA3E15EA4295FA22F5FA31F61FF045EA2BF
:20297300225EA3E35EA4255EB50A5FA22C5FA31C5FB50A61FE045EB00D5EA0E65EB02D5E96
:20299300B10A5EA16C5EB12D5EB2125EA21F5EA2625EB2325EB3115EA3E65EA3225EB3326E
:2029B3005EB4125EA4225EA4665EB4325EA5E65EB5295E71985E91065EBD215FB00D5FA038
:2029D300E65FB02D5FB10A5FA16C5FB12D5FB2125FA2295FA26D5FB2325FB30E5FA3195F67
:2029F300A35B5FB32E5FA5E35FB52961D3045EA2665EA31F5EA4695EBD205FA2705FA35F2C
:202A130061FF045EA2695EA31C5EA46D5FA2745FA36261D3045EA2665EA31F5EA4695FA247
:202A3300705FA35F61FF045EA2625EA3225EA4665FA26D5FA35B61D3045EA2665EA31F5E7A
:202A5300A4695EB5095FA2705FA35F5FB50961FF045EB00D5EA0B15EB02D5EB10D5EA18A3D
:202A73005EB12A5EB2125EA2695EA28D5EB2325EB3125EA31C5EA35F5EB3325EB4125EA4A7
:202A93006D5EA4925EB4325EA5B15EB5295EBD305FB00D5FA0B15FB02D5FB10D5FA18A5F95
:202AB300B12A5FB2125FA2745FA29A5FB2325FB30E5FA3625FA3865FB32E5FA5AE5FB52977
:202AD30061D2045EA28A5EA3625EA48D5EBD205FA2955FA38361FF045EA2865EA3665EA487
:202AF3008A5FA2925FA37F61FF045EA28A5EA3625EA48D5FA2955FA38361D3045EA28D5E07
:202B1300A35F5EA4925FA29A5FA38661FF045EA28A5EA3625EA48D5EB5095FA2955FA383D2
:202B33005FB50961D3045EB00D5EB0295EB10A5EB1265EA2865EB3125EA3665EA38A5EB3E1
:202B5300325EA48A5EB5295E71F85E91CA5EBD215FB00D5FB0295FB10A5FB1265FA2925F16
:202B7300A37F5FB52961FF045EA28A5EA3865EA48D5EBD205FA2955FA38361D2045EA28DC5
:202B93005EA3835EA4925FA29A5FA38661FF045EB0095EB1065EA28A5EA3865EA48D5FB0A8
:202BB300095FB1065FA2955FA38361FF045EA2865EA38A5EA48A5FA2925FA37F61D3045E1D
:202BD300A28A5EA3865EA48D5EB5095FA2955FA3835FB50961FF045EB0295EB1265EA28DEF
:202BF3005EA3835EA4925EB5295EBD305EBD385EBD3C5EBD3D5FB0295FB1265FA29A5FA316
:202C1300865FB52961D3045EA28A5EA3865EA48D5EBD355EBD315EBD305FA2955FA38361A3
:202C3300FF045EA2865EA38A5EA48A5FA2925FA37F61D2045EB0095EB1065EA28A5EA38659
:202C53005EA48D5EBD205FB0095FB1065FA2955FA38361FF045EA28D5EA3835EA4925FA244
:202C73009A5FA38661D3045EA28A5EA3865EA48D5EB5095FA2955FA3835FB50961FF045E31
:202C9300B02D5EB12A5EB2125EA2865EA2695EB2355EA38A5EB4125EA48A5EA46C5EB435C5
:202CB3005EB5295EBD305EBD315FB02D5FB12A5FB2125FA2925FA2705FB2355FB30E5FA329
:202CD3007F5FA3655FB3315FB52961FF045EA26C5EA3865EA46D5EBD215EBD205FA2725F6C
:202CF300A36861D3045EA26D5EA3835EA4705FA2745FA36961FF045EA26C5EA3865EA46D75
:202D13005FA2725FA36861D2045EA2695EA38A5EA46C5FA2705FA36561FF045EA26C5EA381
:202D3300865EA46D5EB5095FA2725FA3685FB50961D3045EB00D5EB0295EB10A5EB1265E3F
:202D5300A26D5EB3125EA3835EA3685EB3355EA4705EB5295EBD215FB00D5FB0295FB10AA3
:202D73005FB1265FA2745FA3695FB52961FF045EA26C5EA3695EA46D5EBD205FA2725FA394
:202D93006861D3045EA2695EA36C5EA46C5FA2705FA36561FF045EB0095EB1065EA26C5E0A
:202DB300A3695EA46D5FB0095FB1065FA2725FA36861FF045EA26D5EA3685EA4705FA27459
:202DD3005FA36961D2045EA26C5EA3695EA46D5EB5095FA2725FA3685FB50961FF045EB071
:202DF300295EB1265EA2695EA36C5EA46C5EB5295EBD305EBD315FB0295FB1265FA2705F0D
:202E1300A3655FB52961D3045EA26C5EA3695EA46D5EBD215EBD205FA2725FA36861FF0425
:202E33005EA26D5EA3685EA4705FA2745FA36961D3045EB0095EB1065EA26C5EA3695EA41B
:202E53006D5FB0095FB1065FA2725FA36861FF045EA2695EA36C5EA46C5FA2705FA3656106
:202E7300FF045EA26C5EA3695EA46D5EB5095FA2725FA3685FB50961D2045EB02D5EB12A36
:202E93005EB2155EA26D5EA2835EB2355EA3685EB4155EA4705EA4865EB4355EB5295EBD9D
:202EB300305EBD385EBD3C5EBD3D5FB02D5FB12A5FB2155FA2745FA28B5FB2355FB3115F68
:202ED300A3695FA37F5FB3315FB52961FF045EA2815EA3695EA4835EBD355EBD315EBD3017
:202EF3005FA2885FA37D61D3045EA27F5EA36C5EA4815FA2865FA37B61FF045EA2815EA326
:202F1300695EA4835EBD205FA2885FA37D61D3045EA2835EA3685EA4865FA28B5FA37F6153
:202F3300FF045EA2815EA3695EA4835EB5095FA2885FA37D5FB50961D2045EB00D5EB02941
:202F53005EB10A5EB1265EA27F5EB3155EA36C5EA3815EB3355EA4815EB5295EBD215FB02C
:202F73000D5FB0295FB10A5FB1265FA2865FA37B5FB52961FF045EA2815EA37F5EA4835E20
:202F9300BD205FA2885FA37D61FF045EA2835EA37D5EA4865FA28B5FA37F61D3045EB009F0
:202FB3005EB1065EA2815EA37F5EA4835FB0095FB1065FA2885FA37D61FF045EA27F5EA349
:202FD300815EA4815FA2865FA37B61D3045EA2815EA37F5EA4835EB5095FA2885FA37D5F95
:202FF300B50961FF045EB0295EB1265EB2155EA2835EA29A5EB2355EA37D5EB4155EA4867C
:203013005EA49D5EB4355EB5295EBD305EBD315FB0295FB1265FB2155FA28B5FA2A25FB210
:20303300355FB3115FA37F5FA3965FB3315FB52961D2045EA2985EA37F5EA49A5EBD215E07
:20305300BD205FA29F5FA39461FF045EA2965EA3815EA4985FA29D5FA39161FF045EB00988
:203073005EB1065EA2985EA37F5EA49A5FB0095FB1065FA29F5FA39461D3045EA29A5EA33D
:203093007D5EA49D5FA2A25FA39661FF045EA2985EA37F5EA49A5EB5095FA29F5FA3945FFD
:2030B300B50961D3045EB02D5EB12A5EA2965EB3155EA3815EA3985EB3355EA4985EB529A0
:2030D3005EBD305EBD315FB02D5FB12A5FA29D5FA3915FB52961FF045EA2985EA3965EA4CD
:2030F3009A5EBD215EBD205FA29F5FA39461D2045EA29A5EA3945EA49D5FA2A25FA39661D5
:20311300FF045EA2985EA3965EA49A5FA29F5FA39461D3045EA2965EA3985EA4985FA29DF9
:203133005FA39161FF045EA2985EA3965EA49A5EB5095FA29F5FA3945FB50961FF045EB0D9
:203153000D5EB0295EB10A5EB1265EA29A5EA3945EA49D5EB5295EBD305EBD385EBD3C5E6D
:20317300BD3D5FB00D5FB0295FB10A5FB1265FA2A25FA3965FB52961D3045EA2985EA396BF
:203193005EA49A5EBD355EBD315EBD305FA29F5FA39461FF045EA2965EA3985EA4985FA235
:2031B3009D5FA39161D2045EB0095EB1065EA2985EA3965EA49A5EBD205FB0095FB1065FD6
:2031D300A29F5FA39461FF045EA29A5EA3945EA49D5FA2A25FA39661D3045EA2985EA39631
:2031F3005EA49A5EB5095FA29F5FA3945FB50961FF045EB0295EB1265EB2155EA2965EA226
:20321300695EB2355EA3985EB4155EA4985EA46C5EB4355EB5295EBD305EBD315FB0295F74
:20323300B1265FB2155FA29D5FA2705FB2355FB3115FA3915FA3655FB3315FB52961D30454
:203253005EA26C5EA3965EA46D5EBD215EBD205FA2725FA36861FF045EA26D5EA3945EA42D
:20327300705FA2745FA36961FF045EB0095EB1065EA26C5EA3965EA46D5FB0095FB1065F5C
:20329300A2725FA36861D2045EA2695EA3985EA46C5FA2705FA36561FF045EA26C5EA396B7
:2032B3005EA46D5EB5095FA2725FA3685FB50961D3045EB02D5EB12A5EA26D5EB3155EA336
:2032D300945EA3685EB3355EA4705EA58A5EB52A5EBD305EBD315FB02D5FB12A5FA2745F7B
:2032F300A3695FA5865FB52A61FF045EA26C5EA3695EA46D5EBD215EBD205FA2725FA368EA
:2033130061D3045EA2695EA36C5EA46C5FA2705FA36561FF045EA26C5EA3695EA46D5FA29C
:20333300725FA36861FF045EA26D5EA3685EA4705FA2745FA36961D2045EA26C5EA3695EA7
:20335300A46D5EB50A5FA2725FA3685FB50A61FF045EB00D5EB0295EB10A5EB1265EA269C4
:203373005EA36C5EA46C5EA5B15EB5295EBD305EBD315FB00D5FB0295FB10A5FB1265FA233
:20339300705FA3655FA5AE5FB52961D3045EA26C5EA3695EA46D5EBD215EBD205FA2725F8E
:2033B300A36861FF045EA26D5EA3685EA4705FA2745FA36961D3045EB0095EB1065EA26C93
:2033D3005EA3695EA46D5FB0095FB1065FA2725FA36861FF045EA2695EA36C5EA46C5FA24D
:2033F300705FA36561D3045EA26C5EA3695EA46D5EB5095FA2725FA3685FB50961FE045E8F
:20341300A0985EB02D5EA1665EB12A5EB2155EA26D5EA28D5EB2325EA3685EB4155EA47025
:203433005EA4925EB4325EA5665EB52A5EBD305EBD385EBD3C5EBD3D5FA0985FB02D5FA1DB
:20345300665FB12A5FB2155FA2745FA29A5FB2325FB3115FA3695FA3865FB32E5FA5625F25
:20347300B52A61FF045EA28A5EA3695EA48D5EBD355EBD315EBD305FA2955FA38361D30439
:203493005EA2865EA36C5EA48A5FA2925FA37F61FF045EA28A5EA3695EA48D5EBD205FA263
:2034B300955FA38361D3045EA28D5EA3685EA4925FA29A5FA38661FF045EA28A5EA3695E44
:2034D300A48D5EB50A5FA2955FA3835FB50A61D3045EB00D5EA0B15EB02D5EB10A5EA18A73
:2034F3005EB12A5EA2865EB3155EA36C5EA38A5EB3325EA48A5EA5B15EB5295EBD305E7103
:20351300985E91065EBD315FB00D5FA0B15FB02D5FB10A5FA18A5FB12A5FA2925FA37F5F66
:20353300A5AE5FB52961FE045EA28A5EA3865EA48D5EBD215EBD205FA2955FA38361D3041B
:203553005EA28D5EA3835EA4925FA29A5FA38661FF045EA28A5EA3865EA48D5FA2955FA3F4
:203573008361FF045EA2865EA38A5EA48A5FA2925FA37F61D3045EA28A5EA3865EA48D5E6A
:20359300B5095FA2955FA3835FB50961FF045EB00D5EA0CB5EB02D5EB10A5EA1665EB12AE8
:2035B3005EB2125EA28D5EA2695EB2325EA3835EB4125EA4925EA46D5EB4325EA5665EB533
:2035D3002A5EBD305EBD385EBD3C5EBD3D5FB00D5FA0CB5FB02D5FB10A5FA1665FB12A5F26
:2035F300B2125FA29A5FA2745FB2325FB30E5FA3865FA3625FB32E5FA5625FB52A61D30479
:203613005EA2665EA3865EA4695EBD2D5EBD3D5EBD355EBD3D5EBD395EBD3D5EBD3C5FA2F3
:20363300705FA35F61FE045EA2625EA38A5EA4665EBD345EBD305FA26D5FA35B61D3045EF3
:20365300A2665EA3865EA4695FA2705FA35F61FF045EA2695EA3835EA46D5EBD205FA2741B
:203673005FA36261FF045EA2665EA3865EA4695EB50A5FA2705FA35F5FB50A61D3045EB0C4
:203693000D5EA0225EB0265EB10A5EA1985EB1295EA2625EB3125EA38A5EA3665EB3325EB6
:2036B300A4665EA5225EB52A5EBD305E71F85E91CA5EBD315FB00D5FA0225FB0265FB10AE8
:2036D3005FA1985FB1295FA26D5FA35B5FA51F5FB52A61FF045EA2665EA3625EA4695EBD27
:2036F300215EBD205FA2705FA35F61D3045EA2695EA35F5EA46D5FA2745FA36261FE045E7F
:20371300B0065EB1095EA2665EA3625EA4695FB0065FB1095FA2705FA35F61D3045EA262FA
:203733005EA3665EA4665FA26D5FA35B61FF045EA2665EA3625EA4695EB50A5FA2705FA3B4
:203753005F5FB50A61D3045EA0665EB02E5EB12D5EA25F5EA35F5EA4625EA5985EB52D5E69
:20377300BD305EBD385EBD3C5E71985E91065EBD3D5FA0665FB02E5FB12D5FA2695FA35848
:203793005FA5965FB52D61FF045EA2665EA3625EA4695EBD355EBD315EBD305FA2705FA349
:2037B3005F61FF045EA26D5EA3665EA4705FA2775FA36661D3045EA2665EA3625EA4695E43
:2037D300BD205FA2705FA35F61FE045EA25F5EA35F5EA4625FA2695FA35861D3045EA2663F
:2037F3005EA3625EA4695EB50D5FA2705FA35F5FB50D61FF045EB00E5EA0225EB0265EB1F2
:203813000D5EB1295EA26D5EA35B5EA4705EA5225EB52A5EBD305E71F85E91CA5EBD315F3D
:20383300B00E5FA0225FB0265FB10D5FB1295FA2775FA3665FA51F5FB52A61D3045EA2662C
:203853005EA3625EA4695EBD215EBD205FA2705FA35F61FF045EA25F5EA3695EA4625FA2AC
:20387300695FA35861FF045EB0065EB1095EA2665EA3625EA4695FB0065FB1095FA2705FB0
:20389300A35F61D3045EA26D5EA35B5EA4705FA2775FA36661FE045EA2665EA3625EA46929
:2038B3005EB50A5FA2705FA35F5FB50A61D3045EA08A5EB02E5EA1B15EB12D5EA25B5EA3A4
:2038D300695EA45F5EA5B15EB52D5EBD305EBD385EBD3C5E71985E91065EBD3D5FA08A5F86
:2038F300B02E5FA1B15FB12D5FA2665FA3545FA5AE5FB52D61FF045EA2665EA3625EA469A1
:203913005EBD355EBD315EBD305FA2705FA35F61D3045EA2705EA35B5EA4745FA27C5FA3E2
:203933006961FF045EA2665EA3625EA4695EBD205FA2705FA35F61D3045EA25B5EA3695E0B
:20395300A45F5FA2665FA35461FF045EA2665EA3625EA4695EB50D5FA2705FA35F5FB50DE9
:2039730061FE045EB00E5EA0225EB0265EB10D5EA1985EB1295EA2705EA3585EA4745EA534
:20399300225EB52A5EBD305E71F85E91CA5EBD315FB00E5FA0225FB0265FB10D5FA1985F17
:2039B300B1295FA27C5FA3695FA51F5FB52A61D3045EA2665EA3625EA4695EBD215EBD20EE
:2039D3005FA2705FA35F61FF045EA25B5EA36D5EA45F5FA2665FA35461D3045EB0065EB15C
:2039F300095EA2665EA3625EA4695FB0065FB1095FA2705FA35F61FF045EA2705EA3585EEC
:203A1300A4745FA27C5FA36961D3045EA2665EA3625EA4695EB50A5FA2705FA35F5FB50A1A
:203A330061FF045EB02E5EA16C5EB12D5EB2125EA2695EA2255EB2325EA36D5EB4125EA4A6
:203A53006D5EA4295EB4325EA56C5EB52D5EBD305EBD385EBD3C5E71985E91065EBD3D5FC0
:203A7300B02E5FA16C5FB12D5FB2125FA2745FA22F5FB2325FB30E5FA3625FA31F5FB32EBC
:203A93005FA5695FB52D61D2045EA2225EA3625EA4255EBD355EBD315EBD305FA22C5FA36C
:203AB3001C61FF045EA21F5EA3585EA4225FA2295FA31961FF045EA2225EA3625EA4255E24
:203AD300BD205FA22C5FA31C61D3045EA2255EA36D5EA4295FA22F5FA31F61FF045EA222DE
:203AF3005EA3625EA4255EB50D5FA22C5FA31C5FB50D61D3045EB00E5EB0265EB10D5EA1FA
:203B1300985EB1295EA21F5EB3125EA3665EA3225EB3325EA4225EA5225EB52A5EBD305E84
:203B330071F85E91CA5EBD315FB00E5FB0265FB10D5FA1985FB1295FA2295FA3195FA51F5C
:203B53005FB52A61FF045EA2225EA31F5EA4255EBD215EBD205FA22C5FA31C61D2045EA24E
:203B7300255EA31C5EA4295FA22F5FA31F61FF045EB0065EB1095EA2225EA31F5EA4255F1C
:203B9300B0065FB1095FA22C5FA31C61FF045EA21F5EA3225EA4225FA2295FA31961D304B1
:203BB3005EA2225EA31F5EA4255EB50A5FA22C5FA31C5FB50A61FF045EA0665EB02E5EB1F0
:203BD3002D5EB2125EA2255EA2065EB2325EA31C5EB4125EA4295EA40A5EB4325EA5985E61
:203BF300B52D5EBD305EBD385EBD3C5E71985E91065EBD3D5FA0665FB02E5FB12D5FB21225
:203C13005FA22F5FA2105FB2325FB30E5FA31F5FA3005FB32E5FA5965FB52D61D3045EA277
:203C3300035EA31F5EA4065EBD355EBD315EBD305FA20C5FA3FE5FB32D61FF045EA2005E51
:203C5300A3225EA4035FA20A5FA3FA61D2045EA2035EA31F5EA4065EBD205FA20C5FA3FED6
:203C730061FF045EA2065EA31C5EA40A5FA2105FA3005FB32E61D3045EA2035EA31F5EA4EE
:203C9300065EB50D5FA20C5FA3FE5FB32D5FB50D61FF045EB00E5EA0225EB0265EB10D5E30
:203CB300B1295EA2005EB3125EA3225EA3035EB3325EA4035EA5225EB52A5EBD305E71F811
:203CD3005E91CA5EBD315FB00E5FA0225FB0265FB10D5FB1295FA20A5FA3FA5FA51F5FB5C5
:203CF3002A61FF045EA2035EA3005EA4065EBD215EBD205FA20C5FA3FE61D3045EA2065EF7
:203D1300A3FE5EB3315EA40A5FA2105FA3005FB32E61FF045EB0065EB1095EA2035EA300BA
:203D33005EB3325EA4065FB0065FB1095FA20C5FA3FE5FB32D61D2045EA2005EA3035EA46E
:203D5300035FA20A5FA3FA61FF045EA2035EA3005EA4065EB50A5FA20C5FA3FE5FB50A612D
:203D7300D3045EA0E65EB02D5EA18A5EB12A5EA2FE5EB2315EA3FE5EB3315EA4005EA58A69
:203D93005EB52A5EBD305EBD385EBD3C5E71985E91065EBD3D5FA0E65FB02D5FA18A5FB16F
:203DB3002A5FA2065FA3F85FA5865FB52A61FF045EA2035EB2325EA3005EB3325EA4065EAA
:203DD300BD355EBD315EBD305FA20C5FA3FE61D3045EA20A5EA3035EA40C5FA2125FA303CE
:203DF3005FB32E61FF045EA2035EA3005EA4065EBD205FA20C5FA3FE5FB32D61FF045EA215
:203E1300FE5EB2315EA3FE5EB3315EA4005FA2065FA3F861D2045EA2035EB2325EA3005E31
:203E3300B3325EA4065EB50A5FA20C5FA3FE5FB50A61FF045EB00D5EA0225EB0265EB10A4E
:203E53005EA1985EB1295EA20A5EA3FA5EB3315EA40C5EA5225EB52A5EBD305E71F85E91C8
:203E7300CA5EBD315FB00D5FA0225FB0265FB10A5FA1985FB1295FA2125FA3035FB32E5F05
:203E9300A51F5FB52A61D3045EA2035EA3005EB3325EA4065EBD215EBD205FA20C5FA3FE02
:203EB3005FB32D61FF045EA2FE5EB2315EA3065EA4005FA2065FA3F861D3045EB0065EB1A8
:203ED300095EA2035EB2325EA3005EA4065FB0065FB1095FA20C5FA3FE61FF045EA20A5E71
:203EF300A3FA5EB3315EA40C5FA2125FA3035FB32E61FF045EA2035EA3005EB3325EA406B7
:203F13005EB50A5FA20C5FA3FE5FB32D5FB50A61D2045EB02E5EA16C5EB12D5EA2FA5EB2E3
:203F3300315EA3065EA4FE5EB4315EA56C5EB52D5EBD305EBD385EBD3C5E71985E91065E95
:203F5300BD3D5FB02E5FA16C5FB12D5FA2035FA3F45FA5695FB52D61FF045EA2035EB2321D
:203F73005EA3005EA4065EB4325EBD355EBD315EBD305FA20C5FA3FE61D3045EA20C5EA3A8
:203F9300FA5EB3315EA4105FA2165FA3065FB32E61FF045EA2035EA3005EB3325EA4065E50
:203FB300BD205FA20C5FA3FE5FB32D61D3045EA2FA5EB2315EA3065EA4FE5EB4315FA20304
:203FD3005FA3F461FF045EA2035EB2325EA3005EA4065EB4325EB50D5FA20C5FA3FE5FB5A1
:203FF3000D61D2045EB00E5EB0265EB10D5EA1985EB1295EA20C5EA3F85EB3315EA4105E78
:20401300A5225EB52A5EBD305E71F85E91CA5EBD315FB00E5FB0265FB10D5FA1985FB12932
:204033005FA2165FA3065FB32E5FA51F5FB52A61FF045EA2035EA3005EB3325EA4065EBDDF
:20405300215EBD205FA20C5FA3FE5FB32D61FF045EA2FA5EB2315EA30A5EA4FE5EB4315F59
:20407300A2035FA3F461D3045EB0065EB1095EA2035EB2325EA3005EA4065EB4325FB00687
:204093005FB1095FA20C5FA3FE61FF045EA20C5EA3F85EB3315EA4105FA2165FA3065FB3F9
:2040B3002E61D3045EA2035EA3005EB3325EA4065EB50A5FA20C5FA3FE5FB32D5FB50A6150
:2040D300FF045EA0CB5EB02D5EA1665EB12A5EA2F85EB2315EA30A5EA4FA5EB4315EA5663C
:2040F3005EB52A5EC6185E30325E50445E70F85EC61E5E33115E937F5EB60D5EBD305E346A
:20411300325E54495E74F85E94FF5EF4005EBD385EBD3C5FA0CB5FB02D5FA1665FB12A5FA3
:20413300A2005FA3F25FA5625FB52A61D2045EA2035EB2325EA3005EA4065EB4325FA20C5C
:204153005FA3FE61FF045EA2105EA3F85EB3315EA4125FA2195FA30A5FB32E61FF045EA2BF
:20417300035EA3005EB3325EA4065EBD2C5EC63E5EA6035EB60A5EBD3C5EBD345EBD3C5EB4
:20419300BD385EBD3C5FA20C5FA3FE5FB32D61D3045EA2F85EB2315EA30A5EA4FA5EB431B9
:2041B3005FA2005FA3F261FF045EA2035EB2325EA3005EA4065EB4325EB50A5FA20C5FA3D5
:2041D300FE5FB50A61D3045EB00D5EA0225EB0265EB10A5EA1985EB1295EA2105EA3F45EBE
:2041F300B3315EA4125EA5225EB52A5EBD2C5EC62E5EA6815EB6095EBD3C5EBD345EBD3C1A
:204213005EBD385EBD3C5FB00D5FA0225FB0265FB10A5FA1985FB1295FA2195FA30A5FB34C
:204233002E5FA51F5FB52A61FF045EA2035EA3005EB3325EA4065FA20C5FA3FE5FB32D617C
:20425300D2045EA2F85EB2315EA30C5EA4FA5EB4315FA2005FA3F261FF045EB0065EB1096B
:204273005EA2035EB2325EA3005EA4065EB4325EBD2C5EBD245EBD205FB0065FB1095FA2A9
:204293000C5FA3FE61D3045EA2105EA3F45EB3315EA4125FA2195FA30A5FB32E61FF045E44
:2042B300A2035EA3005EB3325EA4065EB50A5FA20C5FA3FE5FB32D5FB50A61FF045EB02ED3
:2042D3005EB12D5EB2125EA2065EA2255EB2325EA30C5EB4125E29F15E49C05E69005E8942
:2042F300EE5EC43C5EE9025E2CF15E8CD95EEC005E4C095EA49A5EB4315EB52A5EC63E5EFF
:2043130030005E50075E70D85EC6385E33005E93F05EA6575EBD305E341E5E54055E74F55D
:204333005E94D75EF4025EC8115EBD325FB02E5FB12D5FB2125FA2105FA22F5FB2325FB396
:204353000D5FA3005FB30E5FA31F5FB32E5FC4185F29B15F49AF5F69005F89F15FC4165FB6
:204373002CA25F6C705F8C155FEC015FA40C5F4C0D5FA49F5FB42D5FB52A61D3045EA22294
:204393005EA3005EA4985EBD225EBD205FA22C5FA31C5FA49D61FF045EA21F5EA3F45EB383
:2043B300315EA4965FA2295FA3195FA49A61D2045EA2225EA3005EB3325EA4985FA22C5F7C
:2043D300A31C5FA49D61FF045EA2255EA30C5EA49A5FA22F5FA31F5FA49F61D3045EA222EC
:2043F3005EA3005EA4985EB50A5FA22C5FA31C5FA49D5FB50A61FF045EB00E5EB02A5EB122
:204413000D5EB1295EA21F5EB3125EA3035EA3225EB3325EA4965EB52A5EBD215FB00E5F0B
:20443300B02A5FB10D5FB1295FA2295FA3195FA49A5FB52A61D3045EA2225EA31F5EA49805
:204453005EBD205FA22C5FA31C5FA49D61FF045EA2255EA31C5EA49A5FA22F5FA31F5FA48D
:204473009F61FF045EB00A5EB1095EA2225EA31F5EA4985FB00A5FB1095FA22C5FA31C5F3E
:20449300A49D61D2045EA21F5EA3225EA4965FA2295FA3195FA49A61FF045EA2225EA31F2F
:2044B3005EA4985EB50A5FA22C5FA31C5FA49D5FB50A61D3045EB02A5EB1295EA2255EA35B
:2044D3001C5EA49A5EB52A5EBD305EBD385EBD3C5EBD3D5FB02A5FB1295FA22F5FA31F5F65
:2044F300A49F5FB52A61FF045EA2225EA31F5EA4985EBD355EBD315EBD305FA22C5FA31CB6
:204513005FA49D61D3045EA21F5EA3225EA4965FA2295FA3195FA49A61FF045EB00A5EB169
:20453300095EA2225EA31F5EA4985EBD205FB00A5FB1095FA22C5FA31C5FA49D61FF045E69
:20455300A2255EA31C5EA49A5FA22F5FA31F5FA49F61D2045EA2225EA31F5EA4985EB50AA5
:204573005FA22C5FA31C5FA49D5FB50A61FF045EB02E5EB12D5EB2125EA21F5EA2625EB290
:20459300325EA3225EB4115EA4965EA4E35EB4315EB52A5EBD305EBD315FB02E5FB12D5F23
:2045B300B2125FA2295FA26D5FB2325FB30E5FA3195FA35B5FB32E5FB40D5FA49A5FA4E9C8
:2045D3005FB42D5FB52A61D3045EA2665EA31F5EA4E65EBD215EBD205FA2705FA35F5FA458
:2045F300EC61FF045EA2695EA31C5EA4E95FA2745FA3625FA4EF61D3045EA2665EA31F5E00
:20461300A4E65FA2705FA35F5FA4EC61FF045EA2625EA3225EA4E35FA26D5FA35B5FA4E9B7
:2046330061D3045EA2665EA31F5EA4E65EB50A5FA2705FA35F5FA4EC5FB50A61FE045EB054
:204653000E5EB02A5EB10D5EB1295EA2695EB3125EA31C5EA35F5EB3325EA4E95EB52A5EDB
:20467300BD215FB00E5FB02A5FB10D5FB1295FA2745FA3625FA4EF5FB52A61FF045EA266CA
:204693005EA3625EA4E65EBD205FA2705FA35F5FA4EC61D3045EA2625EA3665EA4E35FA2D9
:2046B3006D5FA35B5FA4E961FF045EB00A5EB1095EA2665EA3625EA4E65FB00A5FB1095F5B
:2046D300A2705FA35F5FA4EC61D3045EA2695EA35F5EA4E95FA2745FA3625FA4EF61FF044A
:2046F3005EA2665EA3625EA4E65EB50A5FA2705FA35F5FA4EC5FB50A61D3045EB02A5EB17B
:20471300295EA2625EA3665EA4E35EB52A5EBD305EBD315FB02A5FB1295FA26D5FA35B5F3F
:20473300A4E95FB52A61FE045EA2665EA3625EA4E65EBD215EBD205FA2705FA35F5FA4EC4F
:2047530061D3045EA2695EA35F5EA4E95FA2745FA3625FA4EF61FF045EB00A5EB1095EA2FB
:20477300665EA3625EA4E65FB00A5FB1095FA2705FA35F5FA4EC61FF045EA2625EA3665EF7
